:020000040800F2
:1000000000000110F19F03081946030879C7000892
:10001000F5A00308F5A00308F5A003080000000000
:10002000000000000000000000000000614C030818
:100030005D4C030800000000594C030859EA000811
:10004000F5A00308F5A00308F5A00308F5A0030830
:10005000F5A00308F5A00308699C0008599D000855
:10006000F5A003081D9D0008E19C0008B1BB000835
:10007000A1BB000891BB000881BB000871BB000850
:100080005DBB000849BB0008F5A00308F5A0030804
:10009000F5A00308F5A00308F5A00308A59C000837
:1000A000F5A0030861CD0008F1CC000889CD000857
:1000B00051CD000841CD000831CD000849C20008EB
:1000C00051C200083DC2000845C20008F5A003085F
:1000D000F5A003088D920008F1910008E5EA0008F8
:1000E0002D9C0008F5A003087D4C0308E1CC000816
:1000F00001CD0008F5A0030811CD000835BB0008AC
:10010000F5A00308F5A0030821CD0008F5A0030819
:10011000F5A00308F5A00308F5A00308F5A003085F
:1001200021BB00080DBB0008F9BA0008E5BA0008B9
:10013000D1BA0008F5A00308F5A00308F5A003084C
:10014000F5A00308F5A00308F5A003081D46030861
:10015000BDBA0008A9BA000895BA0008F5A00308BE
:1001600031C2000839C20008F5A00308F5A0030851
:10017000F5A00308F5A00308F5A00308F5A00308FF
:08018000F5A00308F5A0030837
:1001880002020300701E00206C1E00200000000008
:100198000000000016000800741E00207C1E0020CD
:1001A80000000000C005000803000100E023002053
:1001B800E823002000000000000000001D000100EE
:1001C800002400209424002000000000C805000836
:1001D800100003008C240020982400200000000058
:1001E800CA05000819000500F82300209C240020F7
:1001F80000000000CE05000800010400882400204B
:10020800A424002000000000D405000827000400F2
:1002180020240020A824002000000000D8050008A1
:1002280001010400F42400209033002000000000A5
:100238000000000008020900383300209433002031
:1002480000000000D981000806020C00413300209C
:10025800A033002000000000398F000807020200C8
:1002680074330020AC33002000000000DC050008D7
:10027800FA01010088330020B0330020000000009C
:10028800DE05000802000C0050330020B4330020C3
:10029800000000000000000003123200D6350020E4
:1002A800A4350020000000000000000025005A00CE
:1002B800F03400204A350020000000000000000053
:1002C800F6010800C0330020E834002000000000D8
:1002D8000000000023000E00F83600204C3A0020F1
:1002E80000000000D917020828000C00FC39002083
:1002F8005C3A002000000000E00500082600080025
:10030800103A0020683A002000000000EC050008C0
:100318002900500094390020703A002000000000A5
:10032800000000001400020090390020C03A0020AC
:1003380000000000F40500082C0010004C3E0020CE
:100348003C3E002000000000DD3602082B0024009F
:10035800803E00205C3E002000000000AD36020810
:1003680000020500A43E002000420020000000001A
:10037800000000001E000400E83F002008420020A2
:1003880000000000F605000822000C00683F00206D
:100398000C42002000000000FA05000801000A00D5
:1003A8004C500020585000200000000006060008AD
:1003B8001A0008003450002064500020000000009B
:1003C80010060008F8010100284F00206C5000209A
:1003D80000000000180600082A006000D050002025
:1003E8007050002000000000B9830208150070005A
:1003F800F0480020305100200000000000000000FC
:100408000B100C007C540020445500200000000014
:100418001A0600081F000E007052002050550020D8
:10042800000000002606000805020100B85200205E
:100438006055002000000000340600081200160075
:10044800955500205C560020000000003606000884
:100458000C002400AC550020745600200000000059
:1004680081D101080A0012009C5E0020E466002089
:10047800000000004C0600080D003400685E0020F3
:10048800F866002000000000196D0208FD01240034
:10049800E45600202C670020000000005981000865
:1004A80018002C00B0720020DC7200200000000050
:1004B8007D40020806001A00D46D00200873002051
:1004C800000000004584020834001000006D002080
:1004D8002473002000000000E1830208FB010100F2
:1004E800DC6B0020347300200000000051C30008BA
:1004F800FC010900A46A00203873002000000000F5
:100508001DC30008F70106009C6A00204473002000
:10051800000000005E0600080400C0004C8E0020A9
:10052800409000200000000000000000F9010400D5
:10053800748300200091002000000000C981000899
:100548001B00F4000C9100204493002000000000E0
:100558009553020803010600F895002040960020F4
:10056800000000006406000805000500C997002087
:10057800B8A40020000000006C0600080E00DE0091
:10058800B4960020C0A400200000000025840208C2
:1005980013000400C4970020A0A50020000000005C
:1005A8007406000802010300A3960020A4A50020F9
:0805B80000000000A9D10108B8
:1005C000C4090000190128280000000105000000EE
:1005D000280100009001000020030000013C2C00D5
:1005E0000000000131000000000000000115580269
:1005F000D903C503030000000100C800141E010058
:1006000064002C0128000A0AE803000064000100CD
:100610007E05EA05B405320004002B21231E0002EA
:10062000000001000A0100000000000001000000BD
:1006300000050000000000000001000000000000B4
:100640000000000000000000000000000030010079
:10065000005A0000000090012C01C8006400350021
:100660000100000004010100000000000101010080
:08067000010000000801000078
:100678000000803F0000803F0000803F50010000E4
:100688000700000002000000000000000000000059
:10069800010203040607080901FF00000000803F6B
:1006A8000000803F64CF0308050804000000000034
:1006B8000CF40308A4F3030850CF0308000000005B
:1006C80090CF030805080A00000000000CF4030896
:1006D800A4F30308F4F2030800000000FFFFFFFF83
:1006E800010000000101000045310208000000007F
:1006F80000000000300E0408C80F040800000000C5
:1007080000000000400E0408480E04080000000025
:10071800012000004C0E0408540E040800000000DC
:1007280001400000580E040894FA03080000000075
:1007380001200000640E0408700E04080000000088
:1007480004000000740E0408800E04080000000075
:1007580004000000840E04081C19040800000000AE
:1007680001000000010200000000803FB5440308BA
:100778006D440308BD43030800000000AD400308B2
:1007880031420308B1420308994103080000000000
:1007980000000000A14003088540030881400308C9
:1007A8007D400308714003086D4003087940030841
:1007B8007540030895400308894003087141030800
:1007C800854103085D410308494103083541030891
:1007D8000000803F01010100000000000102030445
:1007E80001020304060708090101000000010101D4
:1007F800010000000060024010600240000000009C
:10080800000B0000000020000000000000000000B5
:10081800006002402860024000000000060C000052
:1008280000002000000000000000000000600240FE
:100838004060024000000000100D00000000200091
:100848000000000000000000006002405860024004
:1008580000000000160E000000002000000000004C
:1008680000000000006002407060024000000000CC
:10087800200F000000002000000000000000000021
:10088800006002408860024000000000261000005E
:10089800000020000000000000000000006002408E
:1008A800A06002400000000030110000000020009D
:1008B800000000000000000000600240B860024034
:1008C80000000000362F000000002000000000009B
:1008D80000000000006402401064024000000000B4
:1008E8000038000000004000000000000000000088
:1008F800006402402864024000000000063900003D
:1009080000004000000000000000000000640240F9
:100918004064024000000000103A0000000040005F
:10092800000000000000000000640240586402401B
:1009380000000000163B000000004000000000001E
:1009480000000000006402407064024000000000E3
:10095800203C0000000040000000000000000000F3
:100968000064024088640240000000002644000041
:100978000000400000000000000000000064024089
:10098800A064024000000000304500000000400064
:10099800000000000000000000640240B86402404B
:1009A8000000000036460000000040000000000083
:1009B8000000000000000101FFFF0000000A040819
:1009C8000000000000000000BDD10108A086010061
:1009D800040000000000000000000000000000000B
:1009E80000000000000000000000000000000000FF
:1009F80008FB03086409040800000000014B010813
:100A08007D0000000600000000000000000000005B
:100A180000000000000000000000000000000000CE
:100A2800000000003026040800000000000000005C
:100A3800DD8A0308E803000003000000000000004E
:100A4800000000000000000000000000000000009E
:100A58000000000000000000382604080000000024
:100A68000000000055850208102700000300000060
:100A7800000000000000000000000000000000006E
:100A8800000000000000000000000000A80E04089C
:100A98000000000035350208DD2A0108204E00005C
:100AA8000500000000000000000000000000000039
:100AB800000000000000000000000000000000002E
:100AC800580B040800000000000000009985030886
:100AD80010270000010000000000000000000000D6
:100AE80000000000000000000000000000000000FE
:100AF8000000000044260408000000000000000078
:100B0800E9C20008E803000005000000000000003A
:100B180000000000000000000000000000000000CD
:100B2800000000000000000050260408000000003B
:100B3800000000004DD40108204E00000300000012
:100B4800000000000000000000000000000000009D
:100B580000000000000000000000000060260408FB
:100B680000000000000000007DD20108204E0000B7
:100B7800030000000000000000000000000000006A
:100B8800000000000000000000000000000000005D
:100B98007026040800000000000000005949010800
:100BA800400D0300030000000000000000000000EA
:100BB800000000000000000000000000000000002D
:100BC8000000000004F80308000000000000000016
:100BD800CD7F02081027000001000000000000007F
:100BE80000000000000000000000000000000000FD
:100BF8000000000000000000700904080000000068
:100C080000000000396402081027000003000000FB
:100C180000000000000000000000000000000000CC
:100C2800000000000000000000000000802604080A
:100C3800000000000000000041940308A0860100A5
:100C4800010000000000000000000000000000009B
:100C5800000000000000000000000000000000008C
:100C6800A4F70308000000000000000069930308CF
:100C780050C3000001000000000000000000000058
:100C8800000000000000000000000000000000005C
:100C980000000000601104080000000000000000CF
:100CA800D98E0308A86100000100000000000000C0
:100CB800000000000000000000000000000000002C
:100CC8000000000000000000882604080000000062
:100CD8000000000083680208A086010001000000EF
:100CE80000000000000000000000000000000000FC
:100CF80000000000000000000000000048F80308A1
:100D0800000000000000000025040108A00F0000FA
:100D180001000000000000000000000000000000CA
:100D280000000000000000000000000000000000BB
:100D3800942604080000000000000000F1210308C8
:100D48001027000001000000000000000000000063
:100D5800000000000000000000000000000000008B
:100D680000000000B80B04080000000000000000AC
:100D7800FDB5020810270000010000000000000077
:100D8800000000000000000000000000000000005B
:100D980000000000000000005809040800000000DE
:100DA80000000000DD3403081A41000001000000C3
:100DB800000000000000000000000000000000002B
:100DC800000000000000000000000000A026040849
:100DD8000000000000000000F56C0208400D030050
:100DE80000000000000000000000000000000000FB
:100DF80000000000000000000000000000000000EB
:100E0800A8260408000000000000000021D6010800
:100E1800A0860100030000000000000000000000A0
:100E280000000000000000000000000000000000BA
:100E3800000000000C2B04080E0000000000000059
:100E48000000000000000000B8140020FFFFFFFFB2
:100E5800FA0000000100000001000000C826040894
:100E6800000000000000000000000000000000007A
:100E7800C0260408040000004BA802080000000077
:100E880000000000D0260408010000000000000057
:100E98000000000000000000000000000D0000003D
:100EA800000000000000000000000000BE8F0020CD
:100EB8000100C40900000000BC8F00200100C40923
:100EC80000000000BA8F00200100C40900000000E3
:100ED800B88F00200100C40900000000B48F002072
:100EE8000100C40900000000B68F00200100C409F9
:100EF80000000000B28F00200100C40900000000BB
:100F0800B08F00200100C40900000000F02604088A
:100F18000E000000000000000000000000000000BB
:100F2800EC070020349600209CFF2C0100000000F4
:100F3800640100200A000000F4F20308C8950020AC
:100F4800E0150C17000000006501002008000000F3
:100F5800A4F3030866010020050000000CF4030850
:100F6800AF510020020000000CF30308CF970020C7
:100F780001200100CE9700200200000018F30308AA
:100F88009A9700200000F4010100000098970020C3
:100F98000000F40101000000969700200000F40111
:100FA80001000000949700200000F40101000000F7
:100FB8009297002000FF0100AE970020E803D007B9
:100FC8000A000000AC970020006401000A0000003D
:100FD800AD970020006401000A000000A6970020D9
:100FE800006401000A000000AB97002000640100C3
:100FF8000A000000AA970020006401000A0000000F
:10100800A9970020006401000A000000A5970020AD
:1010180000FF01000A000000A497002000FF010063
:101028000A000000B09600200000F4010100000052
:10103800AE9600200000F40101000000AC960020EC
:101048000000F40101000000AA9600200000F4014D
:1010580001000000A197002000C80100A09700200F
:1010680000C801009F97002000C801009E9700203B
:10107800006401000A0000009D97002000FF0100A5
:101088000A000000B997002000C80100B8970020A6
:1010980000C80100B797002000C80100B6970020DB
:1010A80000C80100B597002000C80100B4970020CF
:1010B80000C80100B397002000C80100B2970020C3
:1010C80000C80100B197002000C80100F8260408F4
:1010D8000000000000000000000000000000000008
:1010E80008270408090000000000000090080020FC
:1010F8000400000010270408090000000000000098
:101108008408002004000000CC290408090000001D
:101118000000000078080020040000001C260408D5
:1011280009000000000000006C0800200400000016
:1011380018270408090000000000000060080020CB
:101148000400000020270408090000000000000037
:1011580054080020040000002827040809000000A3
:1011680000000000480800200400000030270408A0
:1011780009000000000000003C08002004000000F6
:10118800D026040801000000000000000000000054
:1011980000000000000000000D000000000000003A
:1011A80000000000000000003827040800000000CC
:1011B80000000000000000000000000048270408AC
:1011C8000500000000000000A996002000000000B3
:1011D800D026040801000000000000000000000004
:1011E80000000000000000000D00000000000000EA
:1011F8000000000000000000502704080000000064
:10120800000000000000000000000000C80F0408F3
:1012180000000000000000002A1800200400000060
:10122800182604080C00000005A80208F008002091
:10123800000000005C2C04080C000000F9A802085B
:10124800E4080020000000005C2704080C000000EF
:10125800DDA80208D8080020000000006427040860
:101268000800000000000000CC0800200400000076
:101278006C2704080C000000C1A70208C008002061
:1012880000000000742704080900000000000000A6
:10129800B4080020040000007C27040803000000B4
:1012A800B53303089C08002000000000D02604087D
:1012B8000100000000000000000000000000000025
:1012C800000000000D000000000000000000000009
:1012D8000000000080270408000000000000000053
:1012E8000000000000000000902704080C00000027
:1012F80000000000040900200000000098270408EE
:101308000A00000000000000D09700200000000044
:10131800A42704080A00000000000000D897002055
:1013280000000000AC2704080A00000000000000CC
:10133800E097002000000000B42704080700000020
:1013480000000000FC08002000000000C02704087E
:1013580004000000616E03080000000000000000A7
:10136800D026040801000000000000000000000072
:1013780000000000000000000D0000000000000058
:101388000000000000000000CC2704080000000056
:10139800000000000000000000000000E027040832
:1013A80007000000000000004009002000000000C5
:1013B800EC270408080000000000000034090020A1
:1013C80000000000F82704080800000000000000E2
:1013D8002809002000000000042804080800000074
:1013E800000000001C09002000000000102804086C
:1013F80008000000000000001009002000000000A4
:10140800D0260408010000000000000000000000D1
:1014180000000000000000000D00000000000000B7
:1014280000000000000000001C2804080000000064
:1014380000000000671C00200000000028280408A5
:101448000B00000000000000A809002000000000B8
:10145800302804080B000000000000009C09002050
:10146800000000003C2804080B00000000000000F9
:101478009009002000000000482804080B00000024
:10148800000000008409002000000000542804081F
:101498000B00000000000000780900200000000098
:1014A800602804080B000000000000006C09002000
:1014B80000000000682804080B000000000000007D
:1014C8006009002000000000742804080B000000D8
:1014D80000000000540900200000000080280408D3
:1014E800080000000000000048090020000000007B
:1014F800D0260408010000000000000000000000E1
:1015080000000000000000000D00000000000000C6
:1015180000000000000000008C2804080000000003
:10152800000000000000000000000000A0280408DF
:101538000800000000000000D8090020000000009A
:10154800AC2804080800000000000000CC090020B6
:1015580000000000B828040808000000000000008F
:10156800C009002000000000C4280408080000008A
:1015780000000000B409002000000000D026040884
:101588000100000000000000000000000000000052
:10159800000000000D000000000000000000000036
:1015A80000000000CC280408000000000000000033
:1015B800641C002000000000DC2804080B00000068
:1015C80000000000080A002000000000E8280408C5
:1015D8000B00000000000000FC09002000000000D3
:1015E800F42804080700000000000000F4090020A7
:1015F80000000000002904080700000000000000A7
:10160800EC090020000000000C2904080700000075
:1016180000000000E409002000000000D0260408B3
:1016280001000000000000000000000000000000B1
:10163800000000000D000000000000000000000095
:101648000000000018290408000000000000000045
:10165800641C002000000000242904080700000082
:1016680000000000540A0020000000002C29040893
:1016780007000000000000004C0A002000000000E5
:10168800342904080700000000000000440A002074
:10169800000000003C2904080700000000000000CA
:1016A8003C0A00200000000044290408070000004C
:1016B80000000000340A0020000000004C29040843
:1016C80007000000000000002C0A002000000000B5
:1016D800542904080700000000000000240A002024
:1016E800000000005C29040807000000000000005A
:1016F8001C0A0020000000006429040807000000FC
:1017080000000000140A002000000000D026040891
:1017180001000000000000000000000000000000C0
:10172800000000000D0000000000000000000000A4
:10173800000000006C2904080E00000000000000F2
:10174800296A0308000000005C0A0020A796002010
:101758000A320100A696002001FA0100A296002094
:1017680000C80100A0960020E803D007010000008F
:10177800434F4C4942524900742904080E000000A6
:101788003F6A0308000000008F6C0308380B002034
:101798007C2904080E00000085A80208000000004B
:1017A80000000000880B0020842904080E000000B7
:1017B800416E0308856D03085D6C0308640C002006
:1017C8008C2904080E000000D96A0308A96A0308D6
:1017D80000000000180D0020942904080E000000E5
:1017E800516B0308956B030800000000B80D00203A
:1017F800A297002001030100A02904080E000000A0
:10180800856A0308616A030800000000A80E00202A
:10181800A82904080E000000096B0308B96C030826
:1018280000000000340F0020B42904080E00000056
:10183800C56B0308016D030800000000D40F0020E9
:101848009C97002001030100BC2904080000000047
:10185800000000000000000000000000C829040883
:101868000800000000000000F41000200000000044
:10187800D02904080700000000000000EC10002038
:1018880000000000E0290408070000000000000034
:10189800E410002000000000EC2904080700000004
:1018A80000000000DC10002000000000F8290408F7
:1018B80003000000B5330308C41000200000000036
:1018C800D02604080100000000000000000000000D
:1018D80000000000000000000D00000000000000F3
:1018E8000000000000000000002A040800000000BA
:1018F800000000000000000000000000102A04089A
:101908000A000000000000005CF703080000000067
:10191800182A04080A0000000000000070F90308F3
:1019280000000000202A04080A000000000000004F
:10193800BA97002000000000282A04080A000000C6
:10194800000000000011002000000000D02604085C
:10195800010000000000000000000000000000007E
:10196800000000000D000000000000000000000062
:1019780000000000302A04080000000000000000F9
:1019880000000000000000007CF8030803000000CD
:10199800B53303083811002000000000442A040869
:1019A80003000000B5330308F8150020000000000C
:1019B8004C2A040803000000B53303082011002056
:1019C80000000000542A040803000000B53303088F
:1019D8000811002000000000D026040801000000C3
:1019E80000000000000000000000000000000000EF
:1019F8000D000000000000000000000000000000D2
:101A0800602A040800000000000000000000000038
:101A1800000000006C2A0408070000004D6D030850
:101A2800D01100200000000008FB0308030000009C
:101A3800B5330308B811002000000000782A040814
:101A480003000000B5330308A011002000000000C7
:101A5800802A040803000000B53303088811002019
:101A680000000000882A040807000000316D030800
:101A78008011002000000000782C040803000000FA
:101A8800B53303086811002000000000942A0408F8
:101A980003000000B53303085011002000000000C7
:101AA800D02604080100000000000000000000002B
:101AB80000000000000000000D0000000000000011
:101AC8000000000000000000A02A04080E0000002A
:101AD800FD690308D169030800000000D81100203F
:101AE800A82A04080E000000316C0308000000005A
:101AF8000000000078120020B42A04080E0000003C
:101B08000000000000000000000000000413002096
:101B1800C42A04080E000000096C0308696D030854
:101B28000000000090130020CC2A040800000000E8
:101B3800000000000000000000000000A00E0408E3
:101B480003000000B5330308A014002000000000C3
:101B5800B82A040803000000B533030888140020DD
:101B680000000000D82A040803000000B533030869
:101B78007014002000000000E42A0408030000009C
:101B8800B53303085814002000000000EC2A0408AC
:101B980002000000CD320308000000000000000031
:101BA800F42A040802000000CD32030801000000F6
:101BB80000000000002B040802000000CD320308DA
:101BC8000200000000000000000000000D000000FE
:101BD80000000000000000000000000004030904E9
:101BE8001201000202020040830440570002010271
:101BF8000301000009024300020100C03209040089
:101C08000001020201000524001001052401000161
:101C1800042402020524060001070582030800FFC8
:101C280009040100020A0000000705010240000043
:101C38000705810240000000FF0000009D450308E1
:101C4800DD42030821AB0208F140030849450308B7
:101C5800014103081D410308E1400308D14003087E
:101C68000000000000000000FC2C04080E0000002A
:101C7800F14C030800000000000000007817002065
:101C8800D02C040800000000000000000000000044
:101C980000000000C80F0408000000000000000059
:101CA800E4170020040000005C2C04080C0000006D
:101CB80025520308401C0020000000005C2704088F
:101CC8000C000000FB510308341C00200000000039
:101CD800642704080800000000000000281C0020F9
:101CE800040000006C2704080C0000009950030849
:101CF8001C1C0020000000007C27040803000000D2
:101D0800B5330308041C002000000000E02C040880
:101D180003000000B5330308EC1B0020000000009E
:101D2800D0260408010000000000000000000000A8
:101D380000000000000000000D000000000000008E
:101D48000000000000000000D02C04080000000083
:101D5800000000000000000000000000C80F040898
:101D68000000000000000000E4170020040000004C
:101D7800082C040803000000914E0308D41B00201F
:101D8800080000006C2704080C00000099500308A4
:101D98001C1C0020000000007C2704080300000031
:101DA800B5330308041C002000000000E02C0408E0
:101DB80003000000B5330308EC1B002000000000FE
:101DC800D026040801000000000000000000000008
:101DD80000000000000000000D00000000000000EE
:101DE8000000000000000000E82C040800000000CB
:101DF800000000000000000000000000C80F0408F8
:101E08000000000000000000E417002004000000AB
:101E1800102C040803000000B53303084C1C0020F4
:101E280000000000D02604080100000000000000A7
:101E38000000000000000000000000000D0000008D
:101E480000000000000000000000000000FFFF008C
:101E5800000000002D202D2D202D2D2D2D202D2D85
:101E68002D0000000000000000000000000000003D
:101E7800000000AA5505010000AA550B010000AAA0
:101E88005507010000AA550902000000AA550300E1
:101E98009F00000001000000C0122D202D2D202DD4
:101EA8002D2D2D202D2D2D2D0000000000000000CF
:101EB800000000000000000000000000B6950020AF
:101EC80088130C1701000000B895002088130C1720
:101ED80000000000602B0408000000000000000063
:101EE8000000000000000000702B0408080000003B
:101EF8000000000058180020040000007C2B040893
:101F080008000000000000004C180020000000003D
:101F18007C270408040000007D520308000000002C
:101F280000000000D02604080100000000000000A6
:101F38000000000000000000000000000D0000008C
:101F4800000000000000000000000000B495002020
:101F580088130C1701000000B295002088130C1795
:101F680000000000B82B04080E000000414D0308D3
:101F7800000000000000000064180020C595002043
:101F880001000000CCF30308B19500200100000017
:101F9800D8F30308BA95002002000000E0F3030814
:101FA80006900020000000000000000004900020BF
:101FB8000000000000000000029000200000000067
:101FC8000000000000900020000000000000000059
:101FD800FE8F00200000000000000000FC8F0020A1
:101FE8000000000000000000281800200000000089
:101FF80000000000B095002002000000ECF3030888
:10200800C02B0408000000000000000000000000D1
:1020180000000000702B0408080000000000000009
:10202800E8180020040000007C2B040808000000C9
:1020380000000000DC180020000000007C270408D5
:1020480004000000214D030800000000000000000B
:10205800D026040801000000000000000000000075
:1020680000000000000000000D000000000000005B
:102078000000000000000000D02B04080000000051
:10208800000000000000000000000000E02B040831
:102098000C0000003D510308241900200400000032
:1020A800EC2B04080C000000654D030818190020EB
:1020B80004000000F82B04080C0000000951030874
:1020C8000C19002000000000042C04080300000084
:1020D800B14E0308F418002008000000102C040872
:1020E80003000000B53303084C1C0020000000006A
:1020F800D0260408010000000000000000000000D5
:1021080000000000000000000D00000000000000BA
:102118000000000000000000C826040800000000BD
:10212800000000000000000000000000182C040857
:1021380004000000DD520308000000000000000059
:10214800D026040801000000000000000000000084
:1021580000000000000000000D000000000000006A
:102168000000000000000000642C040800000000CB
:102178000000000000000000000000004C0C0408F3
:102188000C0000000000000084190020040000007A
:10219800742C0408080000000000000078190020D2
:1021A80004000000802C0408080000000000000063
:1021B8006C19002004000000882C040808000000A6
:1021C800000000006019002004000000902C0408A2
:1021D800080000000000000054190020040000005E
:1021E800982C04080800000000000000481900208E
:1021F80004000000A02C04080800000000000000F3
:102208003C19002004000000A82C04080800000065
:10221800000000003019002004000000D026040847
:1022280001000000000000000000000000000000A5
:10223800000000000D000000000000000000000089
:1022480000000000B02C04080E000000314D030807
:10225800000000000000000090190020B82C0408BD
:102268000E00000000000000000000000000000058
:10227800081A0020C02C04080E000000000000000E
:102288000000000000000000A81A0020C7950020E8
:1022980004000000F8F30308AC950020E0150C17C3
:1022A80000000000AF95002008000000A4F3030818
:1022B800AE950020050000000CF40308C82C0408A3
:1022C8000E000000000000000000000000000000F8
:1022D800F81A002020700020702D72000000000005
:1022E80000010000000000000000000001000000E4
:1022F800685E0C00430000000000000000000000C1
:1023080000000000000000000000000000000000C5
:102318000000000043000000000000000000000072
:1023280000000000000000000000000000000000A5
:102338000000000043000000000000000000000052
:102348000000000000000000000000000000000085
:102358000000000043000000000000000000000032
:102368000000000000000000000000000000000065
:102378000000000043000000000000000000000012
:102388000000000000000000000000000000000045
:1023980000000000430000000000000000000000F2
:1023A8000000000000000000000000000000000025
:1023B80000000000430000000000000000000000D2
:1023C8000000000000000000000000000000000005
:1023D8000000000015A3030855A103080000000031
:1023E800DC2D0408BB260408B9010408B901040857
:1023F800B9010408B9010408B9010408B9010408BD
:10240800B9010408B9010408B9010408FFFFFFFF76
:10241800FFFFFFFFFFFFFFFFFFFF00000100415329
:1024280043494900000000000000000000000000CF
:102438000000000000000000000000000000415300
:1024480043494900000000000000000000000000AF
:102458000000000000000000000000000000000074
:10246800F41D002000000000000000000000000033
:102478000000000000000000000000000000000054
:102488000000000000000000000000000000000044
:102498000000000000000000000000000000000034
:1024A8000000000000000000000000000000000024
:1024B8000000000000000000000000000000000014
:0824C80000000000010000000B
:10800000436B826A816930B41C68456A24F00104BC
:108010001144AA421C60D9600DD3016900248A1A58
:108020005A6084621A68002142F0010280F84C1004
:1080300030BC1A607047AA1A5A608562F2E700BF26
:10804000436A8269F0B4D154436A0469426B0133D4
:10805000A34228BF00234362FAB1116811F0010165
:1080600001D0F0BC7047856A1768866927F0010760
:108070002E449D421760D6600BD3641B546081620E
:108080001368002143F0010380F84C10F0BC13602A
:1080900070475D1B55608362F2E7826DD36843F0E1
:1080A0008003D360DDE700BF026B10B462B1836C64
:1080B000C2684469D11A013B615C5DF8044B08BF9A
:1080C00013468364C8B27047016A4369C4685B5C45
:1080D0000131A14228BF114601625DF8044BD8B2BC
:1080E000704700BF436B13B190F84C007047836A30
:1080F000406A181AB0FA80F040097047416A836AF2
:1081000099420AD3CB1A416B026961B14968501E8A
:108110000B4483420AD2C01A704702691144CB1A39
:10812000416B0029F2D1501EC01A704700207047E1
:10813000036B43B1826C5B6893422FBF981AC0688F
:108140009B1AC0187047C269036A9A422FBFD01A9F
:10815000C0688018C01A70470A4B30B503F1140488
:1081600093F900205D78072AC8BF143A81180433B8
:108170000D7313F8025C855413F8012C0A76A342A0
:10818000EED130BDE4C7030803682DE9F041DF6993
:108190001FB13B46BDE8F0411847002A164611DDE5
:1081A00004460D460E4400E023689B68204698472D
:1081B0000028F9D0236815F8011B1B682046984752
:1081C000AE42F1D1BDE8F08100233E213D22017095
:1081D00042708370C3707047152303701623C370F9
:1081E000172383712D234370322303713323C3710B
:1081F000704700BF40F2E93300E0A3B10289013BC0
:1082000012F0020F9BB2F8D089B2818140F2E933BB
:1082100000E043B10289013B12F0010F9BB2F8D09C
:108220008089C0B27047094A904205D0084B9842F5
:1082300001D0FF2070470123064A02EB03135A893D
:10824000013292B25A815889C0B270470030014061
:108250000038004018A60020F0B5446814B1256825
:10826000A4886C8341F08001046840F2E93501E0A4
:10827000002D54D02689013D16F0020FADB2F7D083
:1082800089B2A18140F2E93101E0002958D0258965
:10829000013915F0010F89B2F7D0A189A1894FF0FA
:1082A000000C4FF47A714FF6FF764FF0FF0E6245E7
:1082B00002D12DE0B1421BD02589013915F002050C
:1082C00089B2F7D0A4F80CE04FF47A7102E0B9B2A9
:1082D000B1420DD0258915F0010501F1FF37F6D027
:1082E000A589ADB20BB11D7001330CF1010CDEE7B5
:1082F0001B4B9C4204D0A3F578439C4208D1012536
:10830000184B03EB05156B8901339BB26B816B89AD
:10831000436813B11A689B8813830120F0BD10498C
:108320008C4204D0A1F578418C42B7D101250D498A
:1083300001EB05156989013189B269816989ADE768
:10834000074DAC4203D008498C42A7D10121054D0D
:1083500005EB01114D890135ADB24D8149899DE78C
:108360000030014018A600200038004030B44468B6
:1083700014B12368A5885D83036840F2E93001E009
:10838000002832D01D89013815F0020F80B2F7D0D5
:1083900089B2998140F2E93101E0002947D018897A
:1083A000013910F0010F89B2F7D0998940F2E93113
:1083B00000E059B31889013910F0020F89B2F8D0E2
:1083C00092B29A8140F2E93201E0002A3FD0198945
:1083D000013A11F0010F92B2F7D09B8914B12368D2
:1083E000A2881A83012030BC704721498B4204D0F7
:1083F000A1F578418B42D9D101201E4901EB001033
:108400004189013189B241814189CFE7184A9342BC
:1084100004D0A2F578429342E0D10121154B03EB41
:1084200001114B8901339BB24B814B89D6E7104830
:10843000834203D010498B42B8D101210D4800EB93
:1084400001114889013080B248814989AEE7084965
:108450008B4203D0084A9342C0D10122054B03EB63
:108460000212538901339BB253815389B6E700BF8F
:108470000030014018A6002000380040002870B5E8
:108480001EDB0928044620DD012303EB83035B0088
:10849000B0FBF3F2092AF8D87BB10E4EB4FBF3F02F
:1084A0000928CCBF57223022A6FB03E5024403FB78
:1084B0001044EB0801F8012BF0D100230B7070BDC4
:1084C0002D230B7040420131DBE7303001F8010B06
:1084D000F3E700BFCDCCCCCC884230B44FF00104E0
:1084E0002ED301FB04F4B0FBF4F58D42F9D284B134
:1084F000AAB901E0B0FBF4F5092DCCBF5722302218
:108500002A4404FB150003F8012BB4FBF1F4002C02
:10851000F0D100221A7030BC7047B0FBF4F5092D81
:10852000CCBF372230222A4404FB150003F8012B6C
:10853000B4FBF1F4002CF0D100221A7030BC70476B
:108540000546002AEBD1D7E703685A1C0260197070
:10855000704700BF2DE9F047089C2578002B804626
:1085600089460CBF4FF0200A4FF0300A661C35B325
:10857000002A29DD334601E0024698B113F8011BB9
:10858000501E0029F8D1971E60B13D46013D51466D
:108590004046C8476B1C002BF8DC257827EAE770BB
:1085A000013055B1041B29464046C847301916F81A
:1085B000015B002DF7D1BDE8F087BDE8F087002A08
:1085C00004DC2846BDE8F0870020EBE7571EDCE717
:1085D0000A44914251D030B441F2210411F8013BD8
:1085E00080EA0320430010F4004F84EA03059BB2A5
:1085F000ADB208BF1D466B0015F4004F84EA0300BE
:108600009BB280B208BF1846430010F4004F84EAC2
:1086100003059BB2ADB208BF1D466B0015F4004FB9
:1086200084EA03009BB280B208BF1846430010F4EE
:10863000004F84EA03059BB2ADB208BF1D466B0034
:1086400015F4004F84EA03009BB280B208BF1846BD
:10865000430010F4004F84EA03059BB2ADB208BF9B
:108660001D466B0084EA030015F4004F85B298B2F2
:1086700018BF28468A42B1D130BC7047836842682F
:10868000D0ED037A00EB83010133934281ED040ABC
:10869000836004BF0023836000EB830393ED047ABF
:1086A000036870EE277A9A42C0ED037A77EEC77AB4
:1086B000C0ED037A0CDA013307EE103AF8EEC76A20
:1086C000B7EE007A87EEA60A036030EE070A70471D
:1086D00007EE102AB8EEC77A87EE870A704700BF08
:1086E00090ED097A90ED004AD0ED0A6AD0ED014A8A
:1086F000D0ED047A90ED035AD0ED025AA4EE007A40
:10870000B0EE406AB0EE470AB0EE667AA6EE247A82
:1087100067EEC07AA0EE457AE6EE257A80ED097A1A
:10872000C0ED0A7A704700BFD0ED057A90ED013AAE
:10873000D0ED003AD0ED064A90ED024A90ED077A6E
:1087400090ED035A90ED086AD0ED045AC0ED067A18
:10875000F0EE406A27EE830AC0ED056AA3EEA60A92
:1087600080ED087AA4EE240AA5EE470AA5EEC60A13
:1087700080ED070A704700BFD0ED007A90ED017AD6
:1087800030EE670AE7EE007AB0EE670AC0ED007AD5
:10879000704700BF704700BF704700BF2DE9F04F22
:1087A000DFF8F8C1DFF8F8E1BCF80A70DEF8006025
:1087B000BCF80C30BCF808A03C028BB0361B4FF064
:1087C0000004CDE90034009CBCF806304FEA176580
:1087D0004FF0000767EB0507B946B046A4FB0667F4
:1087E0000024CDE90634009C002304FB0977002413
:1087F000CDE90034AAFB0823CDE90223039AF30D47
:1088000000930AFB09230393009B43EA4723009349
:10881000029B4FEAD31AFB150193039B4AEA436A72
:10882000DDE9002344464D46CDE90845069C12F596
:10883000FA62A4FB086743F1000304FB0977CDE962
:108840000623BCF80440039BBCF802204FEAE31B5C
:10885000230C059323040493340A44EA07643D126D
:10886000DDE904674FEAC23816EB0A0647EB0B074F
:1088700018EB0408DDE906344FEA524949EB0509D3
:10888000B3F5FA6F74F10004B246BB463CDADDE999
:108890000067BC00B20044EA9673B41847EB0305C6
:1088A00022463C462B4602FB04F406FB0344A2FB93
:1088B00006232344940844EA83749D105B104FEA16
:1088C0003202B8EB040869EB0509BAEB020A6BEB5C
:1088D000030BDDE90623304C4FF0FF35A242AB41DC
:1088E0002CDBDDE90856A5FB052305FB06F403EBAD
:1088F0004403D40F44EA4304DD17DDE90623121BC9
:1089000063EB0503CDE90623DEF80440A4FB08234E
:1089100004FB0933540D44EAC3245D15B4EB0A0A81
:1089200065EB0B0B4FEADA3343EA4B4300B10360CC
:1089300009B1069B0B600BB0BDE8F08F40F6AC525E
:10894000B4184FF0000347EB03052246A2FB0223B5
:1089500004FB05F403EB4403941843EB0305A4184C
:108960005D414FEA850CA6004CEA947CB41A6CEB8E
:108970000305DF00D6006D104FEA340447EA527752
:10898000921B63EB0703B8EB040869EB05091AEBCC
:10899000020A4BEB030BA4E724FAFFFF183A00206E
:1089A000581E00204FF480530382704750F8043C57
:1089B000012280F83520143803B11847704700BFF2
:1089C000BFF34F8F0549064BCA6802F4E0621343B8
:1089D000CB60BFF34F8F00BFFDE700BF00ED00E0AD
:1089E0000400FA05F8B5027B466903681F2A2DD9F1
:1089F000A2F120055F682024AC402742114617D021
:108A00001022AA40DC60DA605A68EA40D40749D4F0
:108A1000716B756A0A68B46A22F00102A5420A60A5
:108A200037D1012286F84C20027B11461F2A20D91B
:108A30002039082258688A40024200D0DA600422B5
:108A4000586802FA01F1014221D1F8BD20241D68C5
:108A50009440254211460CD0102191409C609960B1
:108A60001968D140C907D3D5012101FA02F29A60F1
:108A7000CEE7082218688A40024200D09A60042299
:108A8000186802FA01F101420BD09960F8BDD96073
:108A9000F8BD04463046FFF7B3FA227B236811463F
:108AA000C4E7F8BD012202FA05F5DD60B0E700BFBA
:108AB00070B4037B04681F2B08D9203B2021626817
:108AC00001FA03F31A421CD170BC704720212268BE
:108AD00001FA03F31A42F7D042691449582000FB07
:108AE000021251685689CD680868296821F0010191
:108AF0002960828992B222EA06028281A36070BC58
:108B0000704742690949582000FB02125168568992
:108B1000CD680868296821F001012960828992B234
:108B200022EA06028281E36070BC7047006E00207A
:108B300030B4094B1C786CB1084A002502EBC40420
:108B4000116893884D628889083203439BB2A24220
:108B50008B81F5D130BC7047207200202472002038
:108B600010B4037B01681F2B09D9203B20224C68DD
:108B700002FA03F31C4214D15DF8044B7047202223
:108B80000C6802FA03F31C42F6D00C4A4068002439
:108B9000147002685DF8044B22F0010202608B60E1
:108BA0007047064A40680024147002685DF8044B60
:108BB00022F001020260CB60704700BF0F920020DC
:108BC000F0B5C40022189200AE498B585B689D8AAC
:108BD000ADB2EEB2F7070A445CD4B70732D5BFF3A3
:108BE0005F8F167EF6B2012E00F0C780A64D1A8B5D
:108BF000BFF35F8F221801EB8202167E022E00F077
:108C0000D580221801EB8202167E032E00F08880A8
:108C10009A8895F9086092B242F480629A8022188C
:108C200001EB8202127E013296425BD1AA7A0026C3
:108C30006E72002A40F09580204401EB80000023F2
:108C40004375F0BD77074ED416F0400600F0C9809A
:108C50008D4D1E8A95F908E0176AF6B207F80E6086
:108C60005FFA8EFE0EF1010C4FFA8CFC177E85F830
:108C700008C00CF103029742664600F01C812218DE
:108C800001EB8202127E9445C9D10EF1020676B242
:108C90002E72C4E71E887C4D26F400663604360C1E
:108CA0001E801E88B6B246F480661E80967E00271F
:108CB0002F72002E48D06E7A002E42D0221801EB7F
:108CC00082020126127E6E72022A00F0B9802218FA
:108CD00001EB8202927D42F001021A82204401EBF4
:108CE0008000037EF0BD684D967E0127AF72002E96
:108CF00073D06E7A002E7BD1221801EB8202527E55
:108D0000002A00F0A3801A882E7A92B2013642F42B
:108D1000007276B21A802E721A88D205FCD47EE7D1
:108D2000927E002A3FF474AF6A7A002A3FF470AF53
:108D30009A8895F9086022F480621204120C9A80D5
:108D40006DE7D27DFF2AB9D0221801EB8202967D11
:108D500006F0FE061E82D37DFF2BBFD0FF232B72B1
:108D6000BCE79A8822F4407212042044120C01EBF2
:108D700080009A8000234375F0BD927E424D002A08
:108D80003FF435AF6A7A002A3FF431AF1A8822F4F3
:108D900080621204120C1A80BFF35F8F1A8B1A883C
:108DA000AE7292B242F400721A8031E7927E002ACB
:108DB0003FF427AF6A7A002A3FF423AF1A8895F967
:108DC000086022F480621204120C1A809A8822F43D
:108DD00080621204120C9A8021E76A7A002A8BD0F2
:108DE00091E715F0800F284D3AD195F9086016E704
:108DF000167ED2F820E01F88022E95F9086045D92A
:108E000027F480673F043F0C1F801F8AFFB20EF8D3
:108E100006701F88D2F820E0BFB247F400771F80A9
:108E2000F2B21F8A561C76B2FFB20EF806709F8807
:108E3000961CBAB276B242F480622E729A806BE7C8
:108E40001A8892B242F400621A8040E71A8895F9B3
:108E5000086092B242F4807201271A806F725BE759
:108E600095F90870B7F1FF3F2CD0D669F65D1E82E8
:108E700092F818E001377AB2964516462A727FF4C6
:108E8000CEAEA3E7A8A50020581E0020BFB247F42D
:108E900000771F801F8AFFB20EF80670F6B21F8A95
:108EA000D2F820E0721C52B20336FFB276B20EF84E
:108EB00002702E7230E79A8822F480621204120C3B
:108EC0009A80DCE6D77D1F822E72957E1DB9127EB8
:108ED000002A7FF403AF9A8822F480621204120CF5
:108EE0009A80FBE690F8493013B1002280F84920BF
:108EF0001846704770B5044682B00830256A6B4644
:108F000006223B21A847A8B19DF804009DF8006007
:108F10009DF801109DF802509DF803209DF8053042
:108F200041EA062143EA002342EA05226182A28245
:108F3000E382012002B070BD00231822036082701A
:108F4000392243604271012283600272C37270470A
:108F5000F8B50468C4F30D0405460E4604B32F6843
:108F600022F046F9092840F08880454C236923F413
:108F700040732361236943F400732361236943F041
:108F8000010323613E6022F033F92369092823F0AD
:108F90000103236171D12B6804332B600020F8BDDD
:108FA000384B394A93422BD902F58042934226D955
:108FB00002F5804293422AD902F58042934228D991
:108FC00002F58032934226D902F50032934224D929
:108FD00002F50032934222D902F50032934220D9A1
:108FE00002F5003293421ED902F5802293421CD929
:108FF000B3F1016F1BD3052004F00AF9FBE7082445
:1090000022F0F6F8092814D04FF0FF30F8BD1024F4
:10901000F6E71824F4E72024F2E72824F0E73024C8
:10902000EEE73824ECE74024EAE74824E8E7582450
:10903000E6E7134F3B6923F440733B613B6943F41C
:1090400000733B613B6923F0F8033B613B6943F0EC
:1090500002031C433C613B6943F480333B6122F0D3
:10906000C7F83B6923F002033B613B69092823F001
:10907000F8033B613FF473AFC6E76FF00100F8BD42
:10908000003C024000400008FF3F0008F8B50446DD
:109090000D468E180027B54201D12069F8BDE3685E
:1090A000591CE160234415F8012B1A720429F2D1EE
:1090B000206918B9A1682046FFF74AFF2061E760E0
:1090C000E9E700BFF0B583B004466B4606220321F2
:1090D0001E202EF073FB00283CD09DF800509DF818
:1090E00001109DF802709DF803209DF804609DF822
:1090F000053041EA052142EA072243EA062309B284
:1091000012B21BB2144D06EE901A07EE102A07EEAB
:10911000903AF8EEE66A95ED005AD5ED025A95EDD3
:10912000016AB8EEC77AF8EEE77A66EE856A27EE4E
:10913000257A67EE867AFDEEE66ABDEEC77AFDEE29
:10914000E77A16EE901A17EE102A17EE903A218061
:10915000A280638003B0F0BD0000002000B583B0A2
:1091600001AB0322002177202EF028FB9DF805306B
:109170009DF804209DF806001B0243EA02431843B1
:1091800003B05DF804FB00BF08B5FFF7E7FF014B34
:10919000586008BD581E002008B5FFF7DFFF014BDF
:1091A000186008BD581E002068202EF007BB00BFC5
:1091B00070B582B004466946183025F05DF8A8B154
:1091C0009DF805009DF801609DF802109DF8035080
:1091D0009DF804209DF8063041EA062143EA002369
:1091E00042EA0522A184E2842385012002B070BDF9
:1091F00038B5254B5C68236B73B1A36D626BCAB144
:10920000998A1A88C90592B201D5D20700D438BD0F
:109210004FF6F7721A8038BDA36D99891A888906AE
:1092200092B2EBD59206E9D5E26ACAB1988880B2CB
:109230009047E2E799891A880D0692B2E0D51006A8
:10924000DED5A26A616A8A4219D0A1692569885C63
:1092500098800132B2FBF5F105FB1122A262CFE743
:109260009B88E2696169DBB28B54E269E068A36DB7
:109270000132B2FBF0F100FB1122E261BEE7DA68D5
:1092800022F08002DA60BBE72033002038B5254B9E
:109290001C68236B73B1A36D626BCAB1998A1A887B
:1092A000C90592B201D5D20700D438BD4FF6F77286
:1092B0001A8038BDA36D99891A88890692B2EBD5B8
:1092C0009206E9D5E26ACAB1988880B29047E2E78F
:1092D00099891A880D0692B2E0D51006DED5A26AE9
:1092E000616A8A4219D0A1692569885C9880013237
:1092F000B2FBF5F105FB1122A262CFE79B88E26980
:109300006169DBB28B54E269E068A36D0132B2FBA4
:10931000F0F100FB1122E261BEE7DA6822F0800280
:10932000DA60BBE72033002003685B6A03B11847AB
:10933000704700BF03681B6A03B11847704700BF3E
:1093400003682DE9F041DF691FB13B46BDE8F041FC
:109350001847002A164611DD04460D460E4400E06B
:1093600023689B68204698470028F9D0236815F8A1
:10937000011B1B6820469847AE42F1D1BDE8F08141
:1093800003689B69184700BF03685B69184700BF03
:1093900003681B69184700BF0368DB68184700BFF4
:1093A00003689B68184700BF03685B68184700BFE5
:1093B00003681B68184700BF014B1868F8E700BF37
:1093C000B0A8002038B50C46097849B105460134EB
:1093D0002B6828461B68984714F8011B0029F7D111
:1093E00038BD00BF064B53F820302BB11A689B885C
:1093F00051690B4201D1138370475383704700BFFB
:109400004CA80020026802F13F4303F57E032DE9DA
:10941000F04F9B0A544DEB5C03F01F055B090124E0
:10942000032B04FA05F400F09980042B00F09180DE
:10943000022B3ED001F00306731E012BC1F3810CF9
:10944000C1F300188588C1F3411137D900242346A0
:1094500001274FF0030E03E0102B04F1020426D085
:1094600007FA03F0A84303F10103F5D1D2F800C0D5
:109470000EFA04F0C04300EA0C0CC2F800C0D2F8A7
:10948000008006FA04FC4CEA080CC2F800C0D2F8CE
:109490000CC000EA0C00D060D2F80CC001FA04F055
:1094A00040EA0C00102BD06004F10204D8D1BDE8D2
:1094B000F08F2E4B5D6C2C435C64BBE700200346B1
:1094C0004FF0010E4FF0030904E00133102B00F1BF
:1094D00002003CD00EFA03F737EA0504F5D1D2F8C2
:1094E00000A009FA00F4E4430AEA040AC2F800A062
:1094F000D2F800B006FA00FA4AEA0B0AC2F800A055
:10950000D2F808A004EA0A0AC2F808A0D2F808B003
:109510000CFA00FA4AEA0B0AC2F808A0D2F804A032
:109520002AEA07075760D2F804A008FA03F747EAC7
:109530000A075760D7683C40D460D76801FA00F446
:1095400001333C43102BD46000F10200C2D1BDE8CE
:10955000F08F064B1D6B2C431C636BE7034B1D6C9C
:109560002C431C6466E700BF08F70308003802407C
:1095700010B50409013C032C17D80D4B33F8142007
:1095800000F00F0042FA00F313F001030DD00123A5
:1095900003FA00F00138104030F016FD054A064B82
:1095A000125D104403EBC00010BD002010BD00BFD1
:1095B00014F7030810F7030848A600202DE9F04F20
:1095C0004A484B494B4B4C4C4FF0010A4FF00209B3
:1095D0004FF004084FF0080C4FF0100E20274026E3
:1095E000802530F8022B12F0010F03D01960A3F888
:1095F00004A0083312F0020F03D01960A3F80490FE
:10960000083312F0040F03D01960A3F80480083364
:1096100012F0080F03D01960A3F804C0083312F049
:10962000100F03D01960A3F804E0083312F0200FE4
:1096300002D019609F80083312F0400F02D01960E9
:109640009E80083312F0800F02D019609D8008338D
:1096500012F4807F05D04FF4807B1960A3F804B02A
:10966000083312F4007F05D04FF4007B1960A3F893
:1096700004B0083312F4806F05D04FF4806B19608A
:10968000A3F804B0083312F4006F05D04FF4006B58
:109690001960A3F804B0083312F4805F05D04FF4CA
:1096A000805B1960A3F804B0083312F4005F05D0A2
:1096B0004FF4005B1960A3F804B0083312F4804F34
:1096C00005D04FF4804B1960A3F804B00833D20BD7
:1096D00004D04FF4004219609A80083301F580618C
:1096E000A1427FF47EAFBDE8F08F00BF14F70308FE
:1096F0000000024048A600200010024000286AD066
:1097000003682DE9F04F03F13F4404F57E045F4EFA
:10971000A40A0125345D04F01F066409032C05FA30
:1097200006F559D0042C00F0AC80022C59D0858865
:10973000B5FA85F0C0F11F0080B2C40803EB8404C1
:1097400000F00700266A80000F27874026EA0706F8
:109750002662276A01F003068240701E3A43012800
:10976000C1F3810CC1F300182262C1F341113DD94C
:109770000024224601274FF0030E03E0102A04F1D3
:10978000020426D007FA02F0A84302F10102F5D143
:10979000D3F800C00EFA04F0C04300EA0C0CC3F882
:1097A00000C0D3F8008006FA04FC4CEA080CC3F8A9
:1097B00000C0D3F80CC000EA0C00D860D3F80CC08D
:1097C00001FA04F040EA0C00102AD86004F1020407
:1097D000D8D1BDE8F08F70472D4C266C35432564F9
:1097E000A5E72B4C666C35436564A0E70020024674
:1097F0004FF0010E4FF0030904E00132102A00F18E
:1098000002003CD00EFA02F737EA0504F5D1D3F88E
:1098100000A009FA00F4E4430AEA040AC3F800A02D
:10982000D3F800B006FA00FA4AEA0B0AC3F800A01F
:10983000D3F808A004EA0A0AC3F808A0D3F808B0CD
:109840000CFA00FA4AEA0B0AC3F808A0D3F804A0FD
:109850002AEA07075F60D3F804A008FA02F747EA8C
:109860000A075F60DF683C40DC60DF6801FA00F4F3
:1098700001323C43102ADC6000F10200C2D1BDE895
:10988000F08F034C266B3543256350E708F7030838
:1098900000380240002855D0026802F13F4303F52A
:1098A0007E032DE9F04F9B0A544DEB5C03F01F053E
:1098B0005B090124032B04FA05F444D0042B00F0C7
:1098C0009780022B44D001F00306731E012BC1F3D5
:1098D000810CC1F300188588C1F341113DD90024E2
:1098E000234601274FF0030E03E0102B04F102047E
:1098F00026D007FA03F0A84303F10103F5D1D2F80B
:1099000000C00EFA04F0C04300EA0C0CC2F800C01C
:10991000D2F8008006FA04FC4CEA080CC2F800C039
:10992000D2F80CC000EA0C00D060D2F80CC001FAEA
:1099300004F040EA0C00102BD06004F10204D8D1EE
:10994000BDE8F08F70472E4B1D6C2C431C64BAE7AA
:109950002B4B5D6C2C435C64B5E7002003464FF055
:10996000010E4FF0030904E00133102B00F1020057
:109970003CD00EFA03F737EA0504F5D1D2F800A07F
:1099800009FA00F4E4430AEA040AC2F800A0D2F893
:1099900000B006FA00FA4AEA0B0AC2F800A0D2F8B0
:1099A00008A004EA0A0AC2F808A0D2F808B00CFA23
:1099B00000FA4AEA0B0AC2F808A0D2F804A02AEA80
:1099C00007075760D2F804A008FA03F747EA0A0726
:1099D0005760D7683C40D460D76801FA00F401337F
:1099E0003C43102BD46000F10200C2D1BDE8F08FDF
:1099F000034B1D6B2C431C6365E700BF08F703088E
:109A000000380240F0B5044690F84D0083B00028BD
:109A100040F0A4805D4EF77A002F40D004F1180585
:109A2000A0692DF06DFF94F846201A212846FEF714
:109A30009DFC012004F018FFA0692DF04DFF284681
:109A400094F85C10256D6B460622A847D0B19DF8AE
:109A500002609DF803309DF800509DF801109DF8BC
:109A600004009DF8052043EA06231BB2E3845BB2A1
:109A700041EA052142EA00220133A184228506D071
:109A800003B0F0BDB4F926305BB20133F8D194F9DC
:109A900024300133F4D1062003F0BAFBF0E7254669
:109AA00055F8180F2DF02CFF80226B212846FEF769
:109AB0005DFC962004F032FF032268212846FEF761
:109AC00055FC962004F02AFF03226B212846FEF75E
:109AD0004DFC0F2004F0C8FE10226A212846FEF734
:109AE00045FC0F2004F0C0FE3A466C212846FEF7E4
:109AF0003DFC0F2004F0B8FE94F8482019212846B8
:109B0000FEF734FC0F2004F0AFFE18221B2128467C
:109B1000FEF72CFC0F2004F0A7FE10221C21284683
:109B2000FEF724FC0F2004F09FFE10223721284668
:109B3000FEF71CFC0F2004F097FE01223821284676
:109B4000FEF714FC0F2004F08FFEA0692DF0C4FE78
:109B5000012004F089FE0123F37261E7FFF708FD9D
:109B6000054618B1202200238271C37128460021C6
:109B7000FFF790FE2146064B41F8143F284624F09B
:109B800011FB284624F0FCFA44E700BF581E0020D1
:109B9000AD89000810B1036882885A83704700BFFE
:109BA00010B1036882881A83704700BF10B5014660
:109BB00000BF064C2068FFF7EDFF0548FEF71AFBD3
:109BC0002068FFF7EDFF00BF10BD00BF8C33002001
:109BD0000038004018B10368828809B95A83704779
:109BE0001A83704710B40A4B0A4A1C780123834039
:109BF000234052F8200029B9B3FA83F149095DF8EE
:109C0000044BE7E7191C18BF01215DF8044BE1E79D
:109C100048A800204CA8002030B1036882881B6946
:109C20001A4214BF01200020704700BF2DE9F04107
:109C30000B4E346873691C400FD0DFF82880012771
:109C4000B4FA84F3C3F11F0307FA03F558F82300AD
:109C500003689847AC437561F2D1BDE8F08100BF5D
:109C6000003C0140985600202DE9F0410B4E34682D
:109C700073691C400FD0DFF828800127B4FA84F301
:109C8000C3F11F0307FA03F558F823000368984748
:109C9000AC437561F2D1BDE8F08100BF003C0140EA
:109CA000985600202DE9F0410B4E346873691C4032
:109CB0000FD0DFF828800127B4FA84F3C3F11F0323
:109CC00007FA03F558F8230003689847AC43756119
:109CD000F2D1BDE8F08100BF003C01409856002061
:109CE0002DE9F0410B4E346873691C400FD0DFF84A
:109CF00028800127B4FA84F3C3F11F0307FA03F5A0
:109D000058F8230003689847AC437561F2D1BDE869
:109D1000F08100BF003C0140985600202DE9F04141
:109D20000B4E346873691C400FD0DFF82880012780
:109D3000B4FA84F3C3F11F0307FA03F558F82300BC
:109D400003689847AC437561F2D1BDE8F08100BF6C
:109D5000003C0140985600202DE9F0410B4E34683C
:109D600073691C400FD0DFF828800127B4FA84F310
:109D7000C3F11F0307FA03F558F823000368984757
:109D8000AC437561F2D1BDE8F08100BF003C0140F9
:109D900098560020084A094808B5536C43F480439C
:109DA00053640021402232F068FC054B4FF0FF3233
:109DB0001A60C3F8032008BD0038024098560020FE
:109DC000D856002003685B6A184700BF2DE9F041B0
:109DD000044618460D46164698462FF04BFC276859
:109DE000E6722844A07229467D69434632462046E1
:109DF000AC46BDE8F0416047036810B504461B68F7
:109E00009847236820469B689847A37B0133A37338
:109E100010BD00BF10B5036804469B689847FF2338
:109E200001226373227310BD08B5FFF7A1FB38B19F
:109E30002C2282710022C2712021BDE8084029E550
:109E400008BD00BF30B4456815B12B68AA885A8395
:109E5000026841F0800140F2E93301E0002B43D079
:109E60001089013B10F0020F9BB2F7D089B29181AB
:109E700040F2E93301E0002B36D01189013B11F0AB
:109E8000010F9BB2F7D09389938940F2E93300E048
:109E9000D3B11189013B11F0020F9BB2F8D0FF231F
:109EA000938140F2E93300E073B11189013B11F075
:109EB000010F9BB2F8D09489E4B215B12B68AA883F
:109EC0001A83204630BC70470F498A4203D00F4B9B
:109ED0009A42F2D101230E4A02EB03135A8901324E
:109EE00092B25A815B89E8E707498A4203D0074B5F
:109EF0009A42C9D10123064901EB03135989013163
:109F000089B259815B89BFE70030014000380040C9
:109F100018A60020F8B5654C0601A7190546387A41
:109F20002DF06AFB3B7A03F01F015B090122032B32
:109F300002FA01F26DD0042B66D0022B5CD0A3197B
:109F400001351879FFF714FBEDB2074610B1122363
:109F5000C5718371A3195879FFF70AFB10B1132358
:109F6000C5718371A3199879FFF702FB10B114230F
:109F7000C5718371A5190A21EA793846FFF7BEFB3E
:109F80006879FFF7F5FAEA790A21FFF7B7FBA879B4
:109F9000FFF7EEFAEA790A21FFF7B0FBA359444A2A
:109FA000934247D0434A934250D0434A934259D0B8
:109FB000424A934262D0424A93426BD0414A934212
:109FC0002CD03444227BE2B901200222198801F40A
:109FD000415141F445710A4302431A809A8B22F49D
:109FE00000621204120C07219A8319821A8892B215
:109FF00042F040021A80F8BD334B596A0A435A6254
:10A000009DE700200246E1E72F4B19690A431A61D8
:10A0100095E72D4B196A0A431A6290E702F56442EC
:10A020004FF40010536A43F40013536221F040F9D7
:10A03000A359C6E702F584324FF48050536A43F4C3
:10A040008053536221F034F9A359BAE702F5003284
:10A050004FF48040136A43F48043136221F030F9D7
:10A06000A359AEE702F5FE324FF40040136A43F401
:10A070000043136221F024F9A359A2E702F58232CA
:10A080004FF40050536A43F40053536221F010F927
:10A09000A35996E702F568424FF48010536A43F4DF
:10A0A0008013536221F004F9A3598AE718A600200F
:10A0B0000030014000380040003C004000340140C6
:10A0C000005001400054014000380240427A02B979
:10A0D000704710B504460368406804F10A019847C8
:10A0E0000023637210BD00BF437A5A1C0344D2B2EE
:10A0F00042729972037A934200D802B9704710B540
:10A1000004460368406804F10A019847002363721B
:10A1100010BD70B5448806460D46C4F30B042246B4
:10A120000021284632F0A9FA33690A4A934209D33A
:10A13000094A934206D2224628461946BDE8704095
:10A1400030F01AB823B121462846BDE870401847C0
:10A1500070BD00BFC005000878060008064B07491F
:10A160008B4202D30023184670471A88C2F30B02B1
:10A170009042F8D01433F3E788010008C0050008C6
:10A18000024A136823EA000010607047C497002059
:10A19000F8B51A4D2B789F2B2ED16B78BE2B2BD177
:10A1A00005221749A81C32F0B3FA28BB072229461A
:10A1B0004FF6FF70FEF70CFA124FEC1D22884AB1E1
:10A1C000A618BE4218D2052A16D92146FEF700FA73
:10A1D0003446F3E721460222FEF7FAF90222A118DB
:10A1E000FEF7F6F90634084B641B1C8041F60F534A
:10A1F000C31A58425841F8BD0020F8BD004000087D
:10A200002CF7030800800008DC3300202DE9F04F14
:10A21000DFF85891504F8DB00326A7EB090718229D
:10A220000DEB0200002132F028FA4C4BCDF81890CB
:10A2300007971A69002A04DA494A5A6002F18832FB
:10A240005A6001228DF82C20F322DA60454B464CEF
:10A2500018689A8804909B79ADF8142004A9072205
:10A2600006A88DF81630FEF711FF072204A94FF655
:10A27000FF70FEF7ADF9DFF8F8B080464FF0000A46
:10A280005C4539D30CAC002524F82C5D0222214614
:10A2900006A8FEF7FBFE022221464046FEF798F98B
:10A2A00040BAC043ADF80800022202A906A8FEF792
:10A2B000EDFE099878B108ABC0F1040229461844B4
:10A2C00032F0DBF90A9818B9089906A8FEF740FEA3
:10A2D00000230A9009939DF82C300A9A23B11F4954
:10A2E0000B6943F000430B61013E2DD0002A96D14B
:10A2F000FFF74EFF50B32CE065888DF80DA0C5F335
:10A300000B05AA1DADF808202288C2F30B01120B21
:10A31000ADF80A108DF80C2002A9062206A8FEF757
:10A32000B5FE062202A94046FEF752F96168804652
:10A330002A4606A8FEF7AAFE616840462A46FEF7AE
:10A3400047F9143480469BE7002AD1D0052002F05B
:10A350005FFF0DB0BDE8F08F00800008003C0240B8
:10A3600023016745F8C7030888010008004000087A
:10A37000C00500080378202B024600F10100F9D047
:10A38000092BF7D02D2B2CD02B2B03BF5378B7EEF6
:10A39000000A0246B7EE000AA3F13001C8B209284C
:10A3A0009FED467A10D8F2EE046A07EE901AF8EEA6
:10A3B000E77A12F8013FE7EE267AA3F13001C8B23E
:10A3C0000928B0EE677AF0D92E2B4CD003F0DF03CA
:10A3D000452B0BD0F7EE007A67EE276A20EE260AAF
:10A3E00070475378BFEE000A0246D5E710B45178A3
:10A3F0002D2959D02B290ABF9178501C901C00247C
:10A40000A1F13003092B53D8002303EB830301EBA5
:10A41000430310F8011FA1F13002092AA3F1300310
:10A42000F3D9B3F59A7F28BF4FF49A73072B42D91B
:10A43000DFED236A1A46F7EE007A083A072A67EE3C
:10A44000A67AFAD803F007032BB1F2EE046A013BB7
:10A4500067EEA67AFBD124B3C7EE276A5DF8044BFA
:10A4600020EE260A70475378A3F13001C8B20928BC
:10A4700002F10102AAD8F2EE046AF0EE665A07EE83
:10A48000901AF8EEE77A12F8013F87EEA66AA3F178
:10A490003001C8B2092866EEA56A37EE067AEED911
:10A4A00094E767EE276AD9E7901C91780124A7E723
:10A4B000F7EE007ACFE7F7EE007AC5E7000000007C
:10A4C00020BCBE4CB5EEC00ADFED317AF1EE10FAD9
:10A4D000CCBF30EE270A30EE670ADFED2E7A20EE91
:10A4E000270A30B5FDEEC07A87B017EE904A0546D0
:10A4F00084EAE470002303A9A0EBE47001930093C5
:10A50000029326F093FF002CACBF20232D2303A839
:10A510008DF800302FF0AEF8012803A924D00228CE
:10A520002DD0032805BF3023684668468DF80130DA
:10A5300032F0C9F868462FF09DF80338C4B22246BD
:10A540006946284632F01DF900232B5528462FF086
:10A5500091F82E22431C2A540DEB0401E81832F026
:10A56000CFF8284607B030BD302368468DF801305B
:10A570008DF802308DF8033032F0A5F8DAE7302399
:10A5800068468DF801308DF8023032F09CF8D1E742
:10A590006F12033A00007A442DE9F0410646154651
:10A5A0000846B6FBF2F43CB905FB1464124B1B5D84
:10A5B00000F8013BBDE8F081B4FBF2F767B90E4B40
:10A5C00005FB174705FB1464DA5D00F8012B1B5DE2
:10A5D00000F8013BBDE8F081B7FBF2F8B8F1000FDD
:10A5E00002D04046FFF7D8FF05FB1878024B13F85E
:10A5F000082000F8012BE3E734F7030830B40268C1
:10A600001146531C036011F8024B0160D31C5178B2
:10A6100003609378151D05601B0443EA0123D0787D
:10A62000234343EA006030BC704700BF0368591CF5
:10A630001A46016012F8021B0260587841EA0020B5
:10A64000704700BF38B50446006815462FF094FDEA
:10A6500022682A44226038BD036810B40A0E5C1CCC
:10A6600004601A7003680A0C5C1C04601A700368AA
:10A670000A0A5C1C04601A7003685A1C0260197094
:10A680005DF8044B704700BF036810B40A0A5C1CF5
:10A6900004601A7003685A1C026019705DF8044B5C
:10A6A000704700BF03685A1C026010B41970036839
:10A6B0000A0A5C1C04601A7003680A0C5C1C0460C3
:10A6C0001A700368090E5A1C026019705DF8044B79
:10A6D000704700BF03685A1C026019700368090ABA
:10A6E0005A1C0260197070472DE9F047002488B0A9
:10A6F00080460F461E46A14605AD531C03931178B4
:10A7000039B3252933D1931CCDF810900393507899
:10A7100030284ED04FF0000AA0F13003DBB2092BF5
:10A7200042D96C2819D0642800F0938024D82528B9
:10A730001CD063D9582876D063281BD13178404685
:10A74000B847039A531C0393117804360134002947
:10A75000D7D1204608B0BDE8F087039B5A1C03926E
:10A760001B78642B7CD02AD8252B54D12521404638
:10A770000134B847039AC0E7732833D044D9752809
:10A780004FD106F1040E30682B4600220A2176468E
:10A79000FDF7A2FE049A0095534639464046FDF760
:10A7A000D9FE039A0444A8E704AA03A926F01AFED6
:10A7B000B7E7D31C039390784FF0010AACE7732BF3
:10A7C00010D05BD9752B3AD0782B96D1A3F15802D3
:10A7D000B2FA82F2306852092B4610210436FDF796
:10A7E0007BFED7E73368049A00933946002340463E
:10A7F000FDF7B0FE04360444039A7EE70028B9D181
:10A80000204608B0BDE8F0876E28B3D1039A3368BC
:10A8100004361C6071E72AD9582BD7D0632B8DD012
:10A820006BE77828A6D1A0F15802B2FA82F230681C
:10A8300052092B461021FDF74FFE0436AAE706F118
:10A84000040E30682B4600220A217646FDF744FEAE
:10A85000A0E7331D306829461E46FDF70FFE99E735
:10A86000331D306829461E46FDF708FE92E7002B8F
:10A870007FF443AF204608B0BDE8F0876E2BC6D00A
:10A880003BE700BF0EB400B584B005AB019053F8B0
:10A89000042B0649039301A8FFF726FF019B002222
:10A8A0001A7004B05DF804EB03B0704749850008E6
:10A8B0000FB430B583B006AB0A490B4853F8042BEC
:10A8C000096800680193FFF70FFF084C05462068F0
:10A8D000FEF75AFD0028FAD0284603B0BDE8304004
:10A8E00004B070471433002018330020B0A80020B3
:10A8F000DFED2B7AB4EEE70AF1EE10FA4ADDDFED78
:10A90000296A9FED297A01E0B0EE670AB4EEC70A22
:10A91000F1EE10FA70EE667AF6DC9FED247AF4EE32
:10A92000C77AF1EE10FA38D5DFED1E6A9FED207A76
:10A9300001E0F0EE407AF4EEC77AF1EE10FA37EE6D
:10A94000A60AF6D4DFED1B7AB4EEE70AF1EE10FAB0
:10A9500014DDDFED137A37EEC00A60EE006A9FED7A
:10A96000166A9FED167ADFED167AA6EE867A20EE4D
:10A97000266AE6EE877AA6EE270A7047DFED117A9F
:10A98000B4EEE70AF1EE10FA44BFDFED087A37EED5
:10A99000C00AE2E7F0EE407ABFE7B0EE670AD1E71F
:10A9A000DB0F4940DB0FC940E4CB1641DB0F49C048
:10A9B000E4CB16C1DB0FC93F92E741B99730083CA1
:10A9C00015A82ABEDB0FC9BF41404A0011F0800F15
:10A9D00082F0D503D2B2DBB208BF1346590013F0A0
:10A9E000800F81F0D502C9B2D2B208BF0A46510029
:10A9F00012F0800F81F0D503C9B2DBB208BF0B465D
:10AA0000590013F0800F81F0D502C9B2D2B208BF4D
:10AA10000A46510012F0800F81F0D503C9B2DBB2B3
:10AA200008BF0B46590013F0800F81F0D502C9B260
:10AA3000D2B208BF0A46510012F0800F81F0D50350
:10AA4000C9B2DBB208BF0B465A0082F0D50013F042
:10AA5000800FD2B2C0B208BF1046704780EAE073E0
:10AA6000A3EBE0738B4205DB002801DD401A704741
:10AA700002D17047002070470844704709B909E0C7
:10AA8000194690FBF1F301FB13030846002BF7D1A5
:10AA9000084670470146FBE7F0EEC07AB0EEE07A78
:10AAA000B4EEE77AF1EE10FAB4BFB0EE676AB0EE3A
:10AAB000476AB5EE406AF1EE10FA46D0B4EEE77A96
:10AAC000F1EE10FA8CBFF0EE675AF0EE475AC5EE81
:10AAD000866A9FED1F3A9FED1F6A9FED1F4A9FED0B
:10AAE0001F5ADFED1F3ADFED1F4ADFED1F5AA6EEBA
:10AAF000C36AE6EEA34AA6EE864AB7EE006AA6EE61
:10AB0000845AA6EEA46AE6EE855AC5EE866AB4EECD
:10AB1000E77AF1EE10FA48BFDFED147AF5EEC00ADD
:10AB200048BF77EEE66AF1EE10FA48BFDFED107A23
:10AB3000B5EEC00A48BF77EEE66AF1EE10FA48BFFC
:10AB4000F1EE666AB0EE660A7047DFED076ADEE78F
:10AB500039094E3DE3B59E3E88FA163E45FE7F3FDD
:10AB600099FB243F69A2163EA7DFA834DB0FC93F3B
:10AB7000DB0F4940DFED317A30EE277AFDEEC76A10
:10AB800016EE903A2033402B02D99FED2D0A7047E4
:10AB9000B4EEE70AF1EE10FA4DDD9FED2A6ADFED23
:10ABA0002A6A01E0B0EE677AB4EEE67AF1EE10FAC6
:10ABB00077EE467AF6DC9FED257AF4EEC77AF1EE71
:10ABC00010FA35D5DFED1F6A9FED217A01E0F0EE36
:10ABD000407AF4EEC77AF1EE10FA37EEA60AF6D410
:10ABE000DFED167AB4EEE70AF1EE10FA1BDCDFEDCA
:10ABF000197AB4EEE70AF1EE10FA44BFDFED137AEA
:10AC000037EEC00A60EE006A9FED136A9FED137A7B
:10AC1000DFED137AA6EE867A20EE266AE6EE877AD4
:10AC2000A6EE270A7047DFED0F7A37EEC00AE9E794
:10AC3000B0EE670AD4E7F0EE477ABCE7DB0FC93F16
:10AC400000000000DB0FC940E4CB1641DB0F49C018
:10AC5000E4CB16C1DB0FC9BF92E741B99730083C7E
:10AC600015A82ABEDB0F4940FDEEC07A17EE903AD8
:10AC70002033402B51D8DFED2D7AB4EEE70AF1EE08
:10AC800010FA50DDDFED2A6A9FED2A7A01E0B0EE7E
:10AC9000670AB4EEC70AF1EE10FA70EE667AF6DCD7
:10ACA0009FED257AF4EEC77AF1EE10FA38D5DFED94
:10ACB000206A9FED227A01E0F0EE407AF4EEC77A46
:10ACC000F1EE10FA37EEA60AF6D4DFED1D7AB4EEF7
:10ACD000E70AF1EE10FA1BDCDFED1A7AB4EEE70AB0
:10ACE000F1EE10FA44BFDFED147A37EEC00A60EEE1
:10ACF000006A9FED156A9FED157ADFED157AA6EED5
:10AD0000867A20EE266AE6EE877AA6EE270A704754
:10AD1000DFED067A37EEC00AE9E79FED0E0A7047CD
:10AD2000B0EE670AD1E7F0EE407AB9E7DB0F4940B1
:10AD3000DB0FC940E4CB1641DB0F49C0E4CB16C1A1
:10AD4000DB0FC93FDB0FC9BF92E741B99730083C21
:10AD500015A82ABE0000000010B507EE901A2DEDD0
:10AD6000028BB8EE678ADFED227A28EE008A04466D
:10AD700028EE278AB0EE480A2FF0BEFBF0EE408A9C
:10AD8000B0EE480A2FF01AFBF7EE007A9FED197A21
:10AD9000F0EE675AE8EE875A0023A361B0EE676AC7
:10ADA000C7EEA56A63612362E361A3626362A8EEF2
:10ADB000C76ABDEC028B77EEC07AB6EE007AF8EE89
:10ADC000005A27EE877A20EE250A27EE267A26EE0D
:10ADD000266A67EEA67A20EE260A84ED046AC4EDA0
:10ADE000017A84ED007A84ED027A84ED030A10BDC5
:10ADF00027D4D236F304353F10B44C09012250F861
:10AE0000243001F01F0102FA01F10B4340F8243015
:10AE10005DF8044B704700BF4B0901F01F0150F86B
:10AE20002320012303FA01F1114214BF1846002028
:10AE3000704700BFF0B40E4E0E4F0F4C0F4A104B30
:10AE4000104D11480A2131700226267279602D2496
:10AE500040F22E414FF4FA6701269182D78240F2E8
:10AE6000A46140221C72EE7059810282F0BC7047CE
:10AE70009039002050330020B0720020D46D0020A3
:10AE8000AC550020FC390020685E0020074A084BC2
:10AE900010781B78074A834296BFC31AC3F1800318
:10AEA0000020126818441044704700BF4C950020E1
:10AEB000C99400208C390020064A074B10781B7873
:10AEC00083428ABFC3F18003C01AC018C0F17F005B
:10AED000704700BF4C950020C994002010B582B087
:10AEE00000249F2332208DF804308DF805408DF822
:10AEF00006408DF8074003F011FD8DF8014000BFBA
:10AF0000334C2068FEF746FE01A9042268462CF067
:10AF1000A3FC2068FEF744FE00BF9DF802309DF8B8
:10AF200001009DF803102B4A1B0243EA00430B4328
:10AF3000934246D01ADD284A93423AD02FDD274A61
:10AF400093422FD00132934222D1254B4FF480728D
:10AF50001A805A809A881988224C120202FB01F149
:10AF600001209A60D960207302B010BD1E4A93423E
:10AF700018D001329342E8D0A2F51A42033A934224
:10AF800006D1174B20214FF4807219805A80E1E7D7
:10AF9000134B0020188058809860D860E4E7023A8C
:10AFA0009342F5D10E4B80214FF4807219805A8064
:10AFB000D0E70B4B4FF400714FF4807219805A8028
:10AFC000C8E7074B40214FF4807219805A80C1E7CF
:10AFD0008C3300201620C2001920C2001740EF0059
:10AFE0006C1C0020581E002017BA200030B5124CEF
:10AFF000237B83B01BB90120237303B030BD05222E
:10B0000000238DF800208DF8013000BF0B4D28681B
:10B01000FEF7C0FD6946022201A82CF01DFC28683D
:10B02000FEF7BEFD00BF9DF8053003F0010383F07D
:10B030000100237303B030BD581E00208C33002064
:10B0400070B5064C0646256803E023685B1BB342D7
:10B0500003D8FFF7CBFF0028F7D070BD80A80020F1
:10B060002DE9F04F89B0B2F10008019003910293ED
:10B0700040F39F800B46002201EB880153F8040B3C
:10B080008B420244FAD1029B0592002B00F089808A
:10B09000059B002B5ED04B4BDDF814B01B685FFAAC
:10B0A00083FA0AEB0B02B2F5807F474AD2688CBF65
:10B0B000CAF5807ADA469A425ED9190C1A0A4FF01C
:10B0C000020406208DF81F308DF81E208DF81D100B
:10B0D0008DF81C40FFF7B4FF0620FEF767FD3B4AE2
:10B0E0000123137300BF3A4B1868FEF753FD07A9FD
:10B0F000042200202CF0B0FB0024039D019E574643
:10B10000A1462968A30000200A46013459B1B9427A
:10B1100024D231682CF0A0FB2A68336813443360D2
:10B12000BF1AC5F80090A04505F1040506F1040614
:10B13000E7D1274B1868FEF733FD00BF214B214AAA
:10B140001B6853441360029AABEB0A0B0AB3BBF1C2
:10B15000000FA4D1059809B0BDE8F08F019C0493BD
:10B160003A46E1582CF078FB049B2A68E1583944B0
:10B17000D71BE1502F60DCE705981649164AA0EB73
:10B180000B000590059800230B70137009B0BDE803
:10B19000F08F059BA3EB0B030593059809B0BDE861
:10B1A000F08FFFF723FF00287FF472AF029B059317
:10B1B000D0E7029C1CB9FFF719FF0594CAE70023EA
:10B1C0000593C7E78C3900206C1C0020581E002016
:10B1D0008C3300204C950020C994002070B5104D90
:10B1E000104E2B7831788B4284B016D00E4A0392E1
:10B1F0001A4402928CBF0C46CA1A04A98CBFC3F130
:10B2000080020024012341F8102D02A8022201949B
:10B21000FFF726FF002333702B7004B070BD00BF12
:10B22000C99400204C950020CC94002070B5194C96
:10B23000194D23782978994284B027D0174A039270
:10B240001A44029234BF0E46CA1A04A934BFC3F18D
:10B2500080020026002341F8102D02A80222019648
:10B26000FFF7FEFE23781844C0B203062B7848BFD0
:10B2700080F080008342207002D0002004B070BDB6
:10B28000002301202B70237004B070BD012004B096
:10B2900070BD00BFC99400204C950020CC940020C4
:10B2A00008B545F20820FFF7CBFE0620FEF77EFC2E
:10B2B000064B0122C7201A73FEF778FC04480549A3
:10B2C000054A002303700B70136008BD581E002050
:10B2D0004C950020C99400208C3900202DE9F041C4
:10B2E00082B00346060C050A032406208DF80730B9
:10B2F000884617468DF805608DF806508DF8044095
:10B30000FFF79EFE98B100BF0A4C2068FEF742FC92
:10B3100001A9042200202CF09FFA3A460021404661
:10B320002CF09AFA2068FEF73BFC00BF384602B0CA
:10B33000BDE8F0818C330020F0B5124BDD6885B09C
:10B340000DB905B0F0BDED0A14D0002704AE7C198C
:10B350006410E00210226946FFF7C0FF0F2809DDE4
:10B360006B4653F8042B01320AD1B342F9D125467A
:10B37000AF42ECDBFFF732FF034BED021D60E0E76D
:10B38000671CF5E76C1C00208C3900200C4B9842A0
:10B3900013D0A3F5806398420FD003F58043984201
:10B3A0000BD003F58063984207D003F58063984281
:10B3B00003D0044B186840087047024B1868704768
:10B3C00000040140D06D0020F0B5774B774A87B07C
:10B3D0001968914200AF00F0DB800023744A3B60A3
:10B3E0007B60136843F48033136003E03B68B3F57C
:10B3F000A04F09D0136803F400337B603B6801332E
:10B400003B607B68002BF1D0694B1B6813F4003361
:10B4100018BF01237B607B68012B7BD0654D644B9B
:10B42000654AEA606549586F654A0860AA605E6BC4
:10B43000644C654A654826F080065E635E6F46F0A0
:10B4400080765E67196B0C431C63596B5963996B6B
:10B450009963196C41F05B5141F47B1141F41F6118
:10B4600041F00F011964596C07F118040A4348F2BE
:10B47000FF715A6444F8101D002621460123FB7316
:10B480003E737E73BE731FF0C7FE21464FF6FF73F7
:10B490004F48BB601FF0C0FE4FF6FF7321464D487A
:10B4A000BB601FF0B9FE21464B481FF0B5FE214698
:10B4B0004A481FF0B1FE214649481FF0ADFE214623
:10B4C00048481FF0A9FE214647481FF0A5FE214627
:10B4D00046481FF0A1FE20461FF0A8FF444B454CF4
:10B4E0001B68BA6844484549A4FB03439B09A0FB79
:10B4F0000202013B920CB3F1807F0A6007D2404AFE
:10B50000F0200721536085F82300966011601C37F6
:10B51000BD46F0BD264B3B4C1A6C3B4942F0805275
:10B520001A6420680A69CD68496940F44040206087
:10B53000986898609868120640F40040986042EA63
:10B540008512986842F48002490842F010020139DD
:10B5500042EA014240F4A05098605A601A6842F0F2
:10B5600080721A601A689201FCD52849104A40F28C
:10B5700005700860996821F003019960996841F0AD
:10B5800002019960936803F00C03082BFAD145E798
:10B5900000221A6062B61E4B1B6883F308881D4B9D
:10B5A0001B689847FEE700BFFCFF0120EFBEADDE41
:10B5B0000038024000ED00E00005FA056C83002031
:10B5C00000000008FF916700335F070000000240A1
:10B5D0000004024000080240000C0240001002403B
:10B5E0000014024000180240001C024000200240EB
:10B5F000D06D0020D34D621083DE1B4384A8002051
:10B6000010E000E00070004000000020003C02401C
:10B610000000FF1F0400FF1F08B5054B1B6803B1A6
:10B620009847044B044A1A6072B6FDF7C9F900BF87
:10B6300050670020FCFF0120EFBEADDE08B5034BD4
:10B640001B6803B1984772B6FDF7BAF9506700203E
:10B65000084B10B507281B68C8BF143818440C469F
:10B66000007EFDF785FF20B12146BDE81040FEF7C2
:10B67000B1BA10BDE056002030B50446806D61714E
:10B680008389A26823F400531B041B0C838185B0BB
:10B69000A379009213F0040230D04FF4805213F0DB
:10B6A0000203ADF8042056D1ADF806304FF48063A4
:10B6B0000022ADF8083011F00103ADF80C2028D1BC
:10B6C000ADF80A3008238D07694648BFADF80A3047
:10B6D0001FF0EEFEA279A36DD10724D412F0080F5B
:10B6E0009A8A1BD122F008021204120C9A829A89BB
:10B6F00092B242F400529A8105B030BD13F00203B9
:10B70000ADF8042024D04FF400551346ADF8065090
:10B71000CEE70423ADF80A300C23D4E792B242F00E
:10B7200008029A82E3E70D498B420FD0A1F54C4104
:10B730008B4209D00A498B42D0D102200121FFF768
:10B7400087FFA279A36DC9E70120F7E70020F5E79D
:10B75000ADF80630ACE74FF40053A5E70010014008
:10B760000048004010B50446806DA160838923F431
:10B7700000531B041B0C8381A37984B013F00402D3
:10B78000009135D04FF4805213F00203ADF804203D
:10B7900056D1ADF806304FF480636279ADF80830C9
:10B7A000D1074FF00003ADF80A30ADF80C3045BFBB
:10B7B0000423ADF80A3008230C236946920748BFDA
:10B7C000ADF80A301FF074FEA279A36DD1071FD423
:10B7D00012F0080F9A8A16D122F008021204120CF5
:10B7E0009A829A8992B242F400529A8104B010BDB2
:10B7F00013F00203ADF804201FD04FF4005113469C
:10B80000ADF80610C9E792B242F008029A82E8E762
:10B810000D498B420FD0A1F54C418B4209D00B4909
:10B820008B42D5D102200121FFF712FFA279A36D2F
:10B83000CEE70120F7E70020F5E7ADF80630ACE7EA
:10B840004FF40053A5E700BF00100140004800403E
:10B8500038B50C4B07281B68CCBFA0F11404044674
:10B8600023440546187EFDF783FE50B1013427229C
:10B87000C47182712BF042FF28460021BDE8384098
:10B88000E6E638BDE056002070B50F4C0F4DC0EB1A
:10B89000C00004EB8004286B26693043286382B023
:10B8A0009209667BA1600025012101A863618DF8E2
:10B8B00004608DF805208DF806508DF807102BF0E8
:10B8C00079FE02B070BD00BF840100200038024044
:10B8D0002DE9F04F6A4C54F8205083B0002D00F051
:10B8E000CA80EE6D002E00F0C8803769D6F804C01B
:10B8F000644CA96005F162012C60696105F2622463
:10B900004FF400719B46AC61E9602961C5F858C0ED
:10B91000AA4647B35C4C4FF0000E21464B689F424D
:10B9200001F11C0106D00EF1010EBEF1100FF5D190
:10B930004FF0000ECEEBCE0E04EB8E04DFF85081FC
:10B940002369D8F830104FF00C0941EA030E411C6E
:10B95000C8F830E084F818906176B168A9630CF1FA
:10B9600004046C652F630746F068D946904640B3DF
:10B97000454C002123465A68904203F11C0365D0D0
:10B9800001311029F7D100210846C1EBC10104EBB8
:10B990008104DFF8FCE02369DEF830203B491343E3
:10B9A000CEF830300B227B1C63762276F27F2B465A
:10B9B000FFF76AFFAB6DB168F2686A630433E9634D
:10B9C0002B6595F86100FDF7D3FD044695F86000FE
:10B9D000FDF7CEFD8346307F002849D119F0080FCE
:10B9E00036D118F0020F09D044B10B227B1CA27192
:10B9F000E3712046727F2221FDF780FE18F0010FCF
:10BA000015D1AB6B7BB996F82020B17F8DF806304D
:10BA100001A8930901228DF805308DF804108DF8E6
:10BA200007202BF0C7FD504603B0BDE8F08FBBF1F7
:10BA3000000FE6D001370C238BF807708BF8063027
:10BA40005846727F2221FDF759FEDAE7C8B29CE71B
:10BA50000137FFB214B10B23E771A37119F0100F76
:10BA600020460CBF12210221727FFDF747FEC8E776
:10BA70002BF0C2FDB2E7AA46D5E7B246D3E700BF36
:10BA80002033002000C8030884010020E589000855
:10BA9000003802400348D0F8AC3113B100F5D27041
:10BAA00018477047840100200348D0F8903113B143
:10BAB00000F5C47018477047840100200348D0F88F
:10BAC000743113B100F5B670184770478401002037
:10BAD0000348D0F8583113B100F5A87018477047E3
:10BAE000840100200348D0F83C3113B100F59A706E
:10BAF00018477047840100200348D0F8203113B163
:10BB000000F58C7018477047840100200348D0F876
:10BB100004310BB1FC301847704700BF840100208E
:10BB20000348D0F8E8300BB1E0301847704700BF49
:10BB3000840100200348D0F8CC300BB1C430184742
:10BB4000704700BF840100200348D0F8B0300BB12B
:10BB5000A8301847704700BF840100200348D0F880
:10BB600094300BB18C301847704700BF840100201F
:10BB70000248836F0BB17030184770478401002072
:10BB80000248C36D0BB15430184770478401002040
:10BB90000248036C0BB1383018477047840100200D
:10BBA0000248436A0BB11C301847704784010020DB
:10BBB0000248836803B11847704700BF8401002022
:10BBC000431C00F01D812DE9F04F4FEAC00808EB3F
:10BBD00000039B00DFF814A35AF803B087B00AEB08
:10BBE0000304BBF1000F00F0088114330AEB0301DA
:10BBF0000022DBF804704AF803204A608A60CA60B9
:10BC00000346A56801900133D4F80C90DBB2002DF7
:10BC100000F0FD801522EB71AA71B9F1000F00F060
:10BC20000F81162289F8062089F807309BF80E004C
:10BC30002BF0E2FCBB8823F440731B041B0CBB807D
:10BC40002846FDF7ADFF4846FDF7AAFF112128461B
:10BC5000FDF7D8FB11214846FDF7D4FB08266424E4
:10BC600004E00A203CB102F0FFFD013C2846FDF74C
:10BC7000D3FF0028F5D02846FDF78CFF0A2002F0FC
:10BC8000F3FD2846FDF78CFF0A2002F0EDFD013E92
:10BC9000ECD14846FDF77EFF0A2002F0E5FD28467C
:10BCA000FDF778FF0A2002F0DFFD2846FDF778FF58
:10BCB0000A2002F0D9FD4846FDF772FF019B08EB10
:10BCC00003040AEB84042846637C002B0CBF12217A
:10BCD00032210422FDF712FD637C002B0CBF1221E0
:10BCE000322148460422FDF709FD774B9F4200F0C0
:10BCF000C680764B9F4200F0CC80754B9F4200F08F
:10BD0000B480BB880199734A734C23F440731B04BD
:10BD10001B0CBB803B8888440AEB880A9BB243F02B
:10BD200001039AF810103B80BD8802A8002918BFB3
:10BD300014461FF07BFB049A6848B2FBF4F325F02D
:10BD40003F05A0FB02122D04900C2D0C0543BD8075
:10BD5000634C39884FF4967202FB00F284FB024078
:10BD60009BB2D217002BC2EBA01221F0010108BF39
:10BD700001230904013243F40043090C92B23980D3
:10BD80003A84BB833B889BB243F001033B803B88F2
:10BD900023F4816323F002031B041B0C4FF4804245
:10BDA00043F480633B803A813B8823F080031B048B
:10BDB0001B0C3B809BF810308DF80830002402A843
:10BDC00001258DF809408DF80A408DF80B502BF0B5
:10BDD000F1FB9DF80B209BF80F308DF808308DF8A3
:10BDE00009408DF80A4062B95A09203203F01F0356
:10BDF0003C4905FA03F341F8223007B0BDE8F08F63
:10BE0000704702A82BF0D6FB07B0BDE8F08FB9F160
:10BE1000000F48D0162289F8073089F806209BF8D1
:10BE20000E002BF0E9FBBB8823F440731B041B0CB2
:10BE30002846BB80FDF7B4FE4846FDF7B1FE09E792
:10BE40009BF80E002BF0D8FBBB8823F440731B0437
:10BE50001B0CBB802846FDF7A3FE4846FDF7A0FE5D
:10BE600011212846FDF7CEFAF8E61F4A136A43F47B
:10BE7000000313624FF400001FF022FA41E71A4A50
:10BE8000136A43F4001313624FF400101FF018FA02
:10BE900037E7154A136A43F4800313624FF48000B6
:10BEA0001FF00EFA2DE79BF80E002BF0A5FBBB88C8
:10BEB00023F440731B041B0C4846BB80FDF770FE47
:10BEC0004846FDF76DFEC9E60054004000580040AA
:10BED000005C0040009F2400804F120083DE1B4363
:10BEE000D34D621000E100E000380240A8A5002018
:10BEF000F0B5C60033189B00254DEA585468A28A55
:10BF000083B092B20192019A2B4412F4706F1CBF5D
:10BF100001221A75019B13F4E06F07460CD1A38A26
:10BF20003E4423F4706305EB86051B041B0C0022C2
:10BF3000A3826A7503B0F0BD238BA38823F48063CA
:10BF40001B041B0CA380019B9B05E8D42388980548
:10BF5000E5D42388D9050ED52388DA05FCD42388B7
:10BF60009BB243F40073238023889B05FCD438469E
:10BF7000FFF726FED3E723889BB243F400732380A8
:10BF8000A38823F440731B041B0CA380C7E700BFE6
:10BF9000A8A50020F0B583B0441C8DF8073001D06F
:10BFA000032802DD002003B0F0BDC700244E3B187B
:10BFB00006EB83035D68002DF4D04900C9B2997582
:10BFC00001240021DA755C7699761C765C7519750A
:10BFD000A9880DF107028905DA611A6214D42B8849
:10BFE000DA050CD44FF4805401E0013C1ED02B88BC
:10BFF0009B05FAD42B889BB243F480732B80AB88CB
:10C000009BB243F44073AB80074406EB87024FF4C6
:10C01000805401E0013C09D0537D002BFAD106EB9E
:10C0200087073C7D84F0010003B0F0BD054A13880A
:10C0300001339BB21380FFF7C3FD2046B3E700BF77
:10C04000A8A5002014A600202DE9F043322083B0DB
:10C0500002F064FC112300221E210220FFF79AFF48
:10C06000602301221E210220FFF794FF642002F0CA
:10C0700055FC6846FDF726F80024DFF88C8125463C
:10C0800026460A270222104601231E21FFF782FFBF
:10C09000322002F043FC6846FDF714F8BDF900E0D9
:10C0A000BDF90210BDF904208E457346A8BF0B46AA
:10C0B0009342A8BF134643454FF0010076440D4418
:10C0C0001444C0F29180FDF78DF9013FDAD14FF0B1
:10C0D0000109122300221E210220FFF75BFFDFF877
:10C0E00028810A270222104601231E21FFF752FF52
:10C0F000322002F013FC6846FCF7E4FFBDF900E0D3
:10C10000BDF90210BDF904208E457346A8BF0B4649
:10C110009342A8BF134643454FF00100A6EB0E061D
:10C12000A5EB0105A4EB02045BDBFDF75BF9013F26
:10C13000D8D107EE906AF8EEE76A07EE905AB8EEAB
:10C14000E77A07EE904ADFED2A5A9FED2A5A2A4EE7
:10C15000F8EEE77A85EEA66A702300221E210220FF
:10C16000C5EE876A85EE277AB0EEC66AF0EEE66A1B
:10C17000F0EEC77A86ED006AC6ED016AC6ED027A76
:10C18000FFF708FF202301221E210220FFF702FFF4
:10C190000222104600231E21FFF7FCFE642002F05D
:10C1A000BDFBB9F1000F04D14FF07E5333607360D3
:10C1B000B360124C206810B1FDF72EFD18B90120B4
:10C1C00003B0BDE8F0830E490E4B41F8103F2068E4
:10C1D00021F0E8FF206821F0D3FF012003B0BDE883
:10C1E000F0834FF00009A4E74FF0000971E700BFAA
:10C1F00000406F4601C05E4600000020083A002063
:10C20000581E00209987000801F0FFFF01234822F3
:10C2100077210220BEE600BF0123582277210220A9
:10C22000B8E600BF134602200A466821B2E600BF06
:10C230000220FCF7C5BC00BF022059E60120FCF734
:10C24000BFBC00BF012053E60020FCF7B9BC00BF13
:10C2500000204DE61549164B1648CA6810B44C69C3
:10C260001549B2FBF4F203FB02F30360D1F8882016
:10C27000124B134C42F47002C1F888201A68002057
:10C2800042F001021A6098601A6822F0847222F467
:10C2900080321A605C601A684FF0006422F48022D9
:10C2A0001A60D8608C605DF8044B70470000002075
:10C2B00040420F00D06D002000ED00E00038024049
:10C2C00010300024044B4FF4F07002210A22D86091
:10C2D00059611A61FFF7BEBF0000002003680A7AA7
:10C2E000591C01601A70704738B50B4C23688BB12C
:10C2F0005A68821A002A054604DA0CE05A68AA1A1B
:10C30000002A07DB9A68226018461A68904723685B
:10C31000002BF3D138BD38BD4C3D00200B4B002223
:10C3200010B4027203F5C074032102E0072A09DC8D
:10C330009979890702D51979815401329C4203F118
:10C340001803F3D15DF8044B704700BF34E90308CC
:10C350001A230370704700BF70B54E68054630461B
:10C360002DF088F931460446024628682DF004FF76
:10C370002A68131901333B212B60115570BD00BF92
:10C3800008B51DF06BFAFFF759F900BF024A034BDD
:10C390001278197821F008BB8C1E00208D1E002019
:10C3A00038B5384B5A899989914224BF00225A8165
:10C3B000198ADA89914224BF0022DA81DA788AB1B7
:10C3C000072A0FD0304C3148A27801210025062AD7
:10C3D00001709970DD714CD92379DFED2D6A002B46
:10C3E00036D138BDDA799B78284807EE103A002A12
:10C3F00044D0DFED276A0178234CB8EEC77A07EE08
:10C40000901AA278F8EEE77A27EE267A062A67EEE7
:10C41000877A2BD81F4B03EB8203D3ED006AF4EE2F
:10C42000E76AF1EE10FA10DDC6EE877AFDEEE77AE4
:10C4300017EE903A102BA8BF1023012BB8BF012391
:10C44000DBB28B4228BF0B4603702379002BC8D088
:10C45000013A032AC5D8B7EE000A80EE260A2DF06D
:10C46000FFFF2388984238BF208038BDDFED086A7F
:10C47000D5E7DFED097AB0EE677ACBE7DFED076A43
:10C48000B9E700BF9C5E0020D46D0020284F00203B
:10C490006F12033828C803086F12833A6F120339EA
:10C4A000038A2DE9F0478589ADB21D4029D00F469A
:10C4B00006464FF000484FF00009B5FA85F328FA18
:10C4C00003F2D24391B21B3B15403182042B16D8A4
:10C4D000DFE803F03129211903007B6A002B32D0F9
:10C4E00003F1FF3A1FFA8AFAC7F824903C6A34B184
:10C4F00023682046514698476468002CF8D1002DE7
:10C50000DBD1BDE8F0873868716B036889B2984762
:10C51000002DD2D1F5E77868B16B036889B29847EE
:10C52000002DCAD1EDE7B868F16B036889B298476E
:10C53000002DC2D1E5E7F868316C036889B29847ED
:10C54000002DBAD1DDE7F36A1FFA83FACEE700BF08
:10C55000F0B54B4B4B491A68096883B00123570269
:10C5600000935CBF03F180530093D6005CBF43F09F
:10C57000100300938C0744BF43F0C60300934807A1
:10C5800044BF43F0080300930F0748BF43F0200364
:10C590003D4948BF0093160648BF43F440630978FD
:10C5A00048BF0093D40548BF43F0006301F0EF009B
:10C5B00048BF009308286D4655D00E2953D0D003AC
:10C5C0003248009B00784CBF43F4204343F40053AF
:10C5D000D7044CBF43F0644343F0444300280CBFEE
:10C5E00007200F20960648BF43F48073540748BFC6
:10C5F00043F4003343F400245205009402D5244A46
:10C600001279A2BB182936D001900027012639469D
:10C610002846FCB2FEF700FC60B11E4B002203F579
:10C62000D87103E08B420FD013F80C2C944203F125
:10C630000C03F7D10137242FE9D195E80300164BFD
:10C6400083E8030003B0F0BD7A0904F01F0455F835
:10C65000223006FA04F4013723EA0404242F45F8B3
:10C660002240D4D1E9E743F480530093A7E743F491
:10C67000C0130093C6E7009B43F060730093C3E7C9
:10C68000708300205467002090390020FC6D00204A
:10C69000705200201CC90308841E00202DE9F84FA9
:10C6A0004E014FF0000B174D8146904606F12007D2
:10C6B0005C46594628465FFA8BFAFEF7ADFBC0B1DF
:10C6C000A64215D8A74213D900200F4A014604E01C
:10C6D0000131242914D012F80C0C504502F10C023F
:10C6E000F6D10A4B01EB410103EB81014846C047FB
:10C6F00001340BF1010BBBF1240FDAD1BDE8F88F47
:10C700000021F3E7841E00201CC9030810C9030898
:10C7100000210A4A0B4604E00133242B0BD012F807
:10C720000C1C884202F10C02F6D1054803EB4303CE
:10C7300000EB830070470020704700BF24C9030846
:10C7400010C9030800210A4A0B4604E00133242BD8
:10C750000BD012F80C1C884202F10C02F6D10548ED
:10C7600003EB430300EB830070470020704700BFDA
:10C770001CC9030810C9030808B501210220FDF7F0
:10C7800031FA094B1B7803F00503052B08D0002173
:10C790000120FDF727FA00210846FDF723FAFEE7FE
:10C7A0001DF00CF9F3E700BF1C330020022828BF5E
:10C7B000022010B4084C094B207000EBC00200EBC3
:10C7C000820207495DF8044B013003EB4203C0B21B
:10C7D0000B601BF0C5BC00BF95550020B49600202F
:10C7E000E454002008B517F0E1FFFDF70FFDBDE8A8
:10C7F000084017F0C3BF00BF38B50E4C0E4DAC4219
:10C8000006D2616820461434FDF783FCAC42F8D3AD
:10C81000FEF710FB094C0A4B0A48186000252570EA
:10C820001CF0A0FE084B094A65701A60BDE838404C
:10C830001AF034B988010008C00500089555002099
:10C84000E4540020B4960020E8540020AC550020A9
:10C8500008B5FFF7D1FF17F0A9FFFDF7D7FCBDE83A
:10C86000084017F08BBF00BFF0B50C2934D8DFE8C3
:10C8700001F0893333335E333333343333330700DA
:10C88000048C9689B2F802E01788734D24F4805422
:10C890002404240C0484038C8488818B23F40053A7
:10C8A00021F4E6411B0409041B0C46EA0E06090CA0
:10C8B00043EA063341EA0721A8429BB2A4B289B2F7
:10C8C00000F09E8005F58065A84200F0998092688E
:10C8D0008480818302640384F0BD048C9589B2F85E
:10C8E00002C0B2F800E05C4F24F480742404240CED
:10C8F0000484038C8688818B23F400731B0421F04D
:10C9000073011B0C45EA0C04090443EA0423090CD7
:10C91000B8429BB2B6B241EA0E015CD04F4CA04285
:10C9200059D0926886808183C2630384F0BD048CF1
:10C930009589B2F802C0B2F800E0474E24F0100426
:10C940002404240C0484038C8788018B23F02003A7
:10C9500021F4E6411B0409041B0C45EA0C04090CF4
:10C9600043EA041341EA0E21B0429BB2BFB289B23E
:10C970005DD03A4CA0425AD092688780018382638E
:10C980000384F0BD048C9789B2F802E01688324D1A
:10C9900024F001042404240C0484038C8488018B77
:10C9A00023F002031B0421F073011B0C47EA0E075E
:10C9B00009043B43090CA8429BB2A4B241EA060118
:10C9C00025D005F58065A84221D092688480018336
:10C9D00042630384F0BDD589148A578A23F4006327
:10C9E00043EA05254FF6FF332B40958826F4405641
:10C9F0003C4343EA052346EA04169BB2B6B290E7ED
:10CA0000158A24F4804444EA8514A4B25FE7D689E9
:10CA1000158A578A23F00803334324F44074968818
:10CA20003D4323F004032C433343A4B2CDE7D48920
:10CA3000158A568A23F0800343EA04134FF6BF7425
:10CA40001C40938827F44067354344EA031347EAC0
:10CA500085079BB2BFB28FE7000001400004014090
:10CA60002DE9F84F4FF4B47200218D488D4C8E4D56
:10CA70008E4E8F4FDFF85482DFF854922FF0FDFD79
:10CA80008C488D49DFF84CE2DFF84CC20022135885
:10CA90008B4200F0D280B3F1804F00F0D580AB42E2
:10CAA00000F0D980B34200F0D980BB4200F0D980B9
:10CAB000734500F0D980634500F0D980434500F00C
:10CAC000D9804B4500F0D980DFF810A2534500F023
:10CAD000D7800AF5806A534500F0D580AAF5983AC8
:10CAE000534500F0D3800AF5806A534500F0D180A9
:10CAF0000AF5806A534500F0CF801832B2F5CC7F3A
:10CB0000C5D1DFF8B0816D4E08F5CC774FF0030A40
:10CB10004FF0020998F804301C09013C032C03F083
:10CB20000F0377D8664A32F8140040FA03F2D207AE
:10CB300070D5012505FA03F3013B18402DF044FAA6
:10CB4000604B1B5D184416EBC00263D056F83030C2
:10CB50005D4C98F8081003F13F4000F57E00800A14
:10CB6000205C00F01F044009032805FA04F55ED09C
:10CB7000042856D0022804D14A48406C054349484D
:10CB80004564B2F804E0BEFA8EF2C2F11F0292B21E
:10CB9000D00803EB800002F00702046A92000F2520
:10CBA000954024EA05040462046A01FA02F2224371
:10CBB000002502624FF0010C2A4603E0102A05F11D
:10CBC000020527D00CFA02F030EA0E0102F1010250
:10CBD000F4D11C680AFA05F1C9430C401C60D3F873
:10CBE00000B009FA05F444EA0B041C609C680C4090
:10CBF0009C609C689C605C6824EA000058605868EF
:10CC00005860D8680140D960D968D960102A05F108
:10CC10000205D7D108F11808B8457FF47BAFBDE80D
:10CC2000F88F2048006B05431E480563A9E71D489F
:10CC3000006C05431B480564A3E74FF0010A636CD1
:10CC400043EA0A03636458E74FF0010A236C43EA9E
:10CC50000A03236451E74FF0020AF7E74FF0040A92
:10CC6000F4E74FF0080AF1E74FF0100AEEE74FF053
:10CC7000200AEBE74FF0020AE1E74FF4803ADEE7E3
:10CC80004FF4003ADBE74FF4802AD8E74FF0400A30
:10CC9000DCE74FF0800AD9E74FF4807AD6E700BF8F
:10CCA00008570020003802400004004000080040FF
:10CCB000000C004034E903080000014048A60020B1
:10CCC00014F7030810F7030808F7030800040140ED
:10CCD00000400140001000400014004000440140AA
:10CCE00001490248FFF7DCBB48580020001800400B
:10CCF00001490248FFF7D4BB2058002000480140FA
:10CD000001490248FFF7CCBBD05700200004014086
:10CD100001490248FFF7C4BBD0570020000401407E
:10CD200001490248FFF7BCBBA8570020000C004097
:10CD300001490248FFF7B4BB8057002000080040BB
:10CD400001490248FFF7ACBB5857002000040040DF
:10CD500002494FF08040FFF7A3BB00BF30570020CF
:10CD600010B5064C06482146FFF79AFB04F1F00186
:10CD70000448BDE81040FFF793BB00BF08570020F0
:10CD8000000001400044014001490248FFF788BB10
:10CD90000857002000000140F0B50468A30AA3F57D
:10CDA0008013522B2BD8DFE803F02B7B978F2A2A96
:10CDB000932A2A2A2A2A2A2A2A2A2A2A2A2A2A2A6A
:10CDC0002A2A2A2A2A2A2A2A2A2A2A2A2A2A2A2AC3
:10CDD0002A2A2A2A2A2A2A2A2A2A2A2A2A2A2A2AB3
:10CDE0002A2A2A2A2A2A2A2A2A2A7F832A2A2A2AF5
:10CDF0002A2A2A2A2A2A2A2A2A2A2A878B00F0BDA6
:10CE00004FF0480E01264779B0004FEA970C0029F1
:10CE10006FD063460227A5899F4083190CEB43031B
:10CE20002F4303F1040C3D4DBFB245F8231045F8E4
:10CE30002C20A781EFF31181502282F312888219EE
:10CE400005EBC2021369002B4AD013620433821926
:10CE500005EBC202576917B11F6053690433821989
:10CE600005EBC202976917B11F60936904338219F9
:10CE700005EBC202D76917B11F60D36904330027DD
:10CE8000CAB21F6082F31188304405EBC000036A08
:10CE90004BBBA38923F001031B041B0CA381F0BD32
:10CEA0004FF0700E0226AEE74FF0200E0026AAE7E4
:10CEB0004FF0E80E0526A6E74FF4887E0626A2E787
:10CEC0004FF49C7E07269EE74FF0C00E04269AE79B
:10CED0004FF4B07E082696E74FF0980E032692E7AF
:10CEE00005EB0E03B3E7A3899BB243F00103A381D3
:10CEF000F0BD0223BF0803FA07F7A389074D9BB2D1
:10CF000023EA070387190CEB470CA3810CF10403F8
:10CF100045F82C1045F823208CE700BF0857002067
:10CF200010B5036883480139834282B089B200F0AA
:10CF3000CB80A0F58060834200F0C68000F5804081
:10CF4000834200F0B88000F58060834200F0B38037
:10CF500000F58060834200F0AE80774C188824682A
:10CF60006408B4FBF2F4013CA4B282B2B3F1804F86
:10CF70000AD07248834207D000F58060834203D014
:10CF800000F58060834202D122F0700292B26C48B8
:10CF9000834200F0A28000F58060834200F0A78009
:10CFA00022F4407200F56C4092B283421A80D9623A
:10CFB0001C854FD05F4A93424CD001229A821A8836
:10CFC00092B242F001021A80B3F1804F00F09980D2
:10CFD0005A4A934200F0978002F58062934200F033
:10CFE000948002F58062934200F0918002F58062A5
:10CFF000934200F08E8002F58062934200F08B80B5
:10D0000002F57042934200F0888002F5705293421C
:10D0100000F0858002F58062934200F0828002F584
:10D02000806293427FD0A2F5983293427DD002F580
:10D03000806293427BD002F58062934208BF0D224A
:10D0400015D002A84FF0012340F8043D2AF0B2FAAF
:10D0500002B010BD0122002119869A821A8839482F
:10D0600092B242F0010283421A80ADD10A46364B99
:10D0700003EBC20301A893F821408DF8044001237B
:10D0800000228DF805308DF807308DF806202AF043
:10D0900091FA1B2C08D02E2CDAD12C4B019301A82D
:10D0A0002AF088FA02B010BD294B019301A82AF09A
:10D0B00081FA02B010BD204C18882468B4FBF2F449
:10D0C000013CA4B282B251E71B4C18882468B4FB1F
:10D0D000F2F4013CA4B282B256E701201A80D96270
:10D0E0001C8598821A8892B202431A8070E7012048
:10D0F0001A80D9621C8598821A8892B202431A80DB
:10D1000062E70122B3E70222B1E70322AFE704227C
:10D11000ADE70522ABE70622A9E70722A7E7082229
:10D12000A5E70922A3E70A22A1E70B229FE70C2229
:10D130009DE700BF00040140D06D002000040040C6
:10D14000001000400000014028C803082C01000125
:10D15000190100012C4B98423DD0B0F1804F3CD0DA
:10D16000A3F57C4398423AD003F58063984238D0C7
:10D1700003F58063984236D003F58063984234D03B
:10D1800003F58063984232D003F57043984230D063
:10D1900003F5705398422ED003F5806398422CD04B
:10D1A00003F5806398422AD0A3F59833984228D09B
:10D1B00003F58063984207D003F58063984208BF67
:10D1C0000D2202D0002070470C22104B03EBC2034B
:10D1D00093F8200070470022F7E70122F5E70222CA
:10D1E000F3E70322F1E70422EFE70522EDE7062249
:10D1F000EBE70722E9E70822E7E70922E5E70A2249
:10D20000E3E70B22E1E700BF0000014028C8030864
:10D210002DE98048013085B0C3B203938A4D8B4F0E
:10D220008B4C8C4E0A230293DFF82C9220F014FED4
:10D230004FF4FA7A4FF0100C4FF47A70D9F80430AA
:10D24000C3F30803002B40F0C180EFF31183002BE0
:10D2500040F0BC802968A26800BF2B689942F9D1D0
:10D26000D7F800E000FB0EF39B1AB3FBFEF300FBC4
:10D2700001314FF0010E0191D9F80430C3F30803D6
:10D28000002B40F08780EFF31183002B40F0828069
:10D290002B68A16800BF2A689342F9D1D7F800B083
:10D2A00000FB0BF2521AB2FBFBF200FB0323019AC4
:10D2B0009B1AB3F57A7FDFD3BAF1010ABED1039B83
:10D2C000002B40F0BD804FF47A7ADFF88C91504605
:10D2D0004FF0100CD9F80430C3F30803002B40F0D2
:10D2E0009280EFF31183002B40F08D802968A268B3
:10D2F00000BF2B689942F9D1D7F800E000FB0EF38C
:10D300009B1AB3FBFEF300FB01314FF0010E0191BC
:10D31000D9F80430C3F3080303BBEFF31183EBB96F
:10D320002B68A16800BF2A689342F9D1D7F800B0F2
:10D3300000FB0BF2521AB2FBFBF200FB0323019A33
:10D340009B1AB3F57A7FE3D3BAF1010AC2D1029BEB
:10D35000013B02937FF468AFFEF770F9EFF3118899
:10D360008CF31288A1682368DB0344BFC6F800E091
:10D37000A1682B6832685FFA88F888F31188D7F8BB
:10D3800000801A4400FB08F35B1AB3FBF8F300FBC0
:10D390000233D4E7EFF311888CF31288A168236875
:10D3A000DB0344BFC6F800E0A1682B6832685FFA6F
:10D3B00088F888F31188D7F800801A4400FB08F336
:10D3C0005B1AB3FBF8F300FB023370E7EFF3118253
:10D3D0008CF31288D4F808E02368D90303D501231D
:10D3E0003360D4F808E02B683168D2B282F3118838
:10D3F0003A68194400FB02F3A3EB0E03B3FBF2F30C
:10D4000000FB013135E7EFF311828CF31288D4F879
:10D4100008E02368D90303D501233360D4F808E07A
:10D420002B683168D2B282F311883A68194400FB44
:10D4300002F3A3EB0E03B3FBF2F300FB013164E74D
:10D4400018462AF075FA3EE780A8002084A800203C
:10D4500010E000E07CA8002000ED00E02DE9F0479E
:10D46000AD4FAE4E17F0A2F9BE421ED2DFF83883A0
:10D47000DFF838934446258862197DB14A450DD2BC
:10D48000052D0BD933886188C3F30B03994200F053
:10D49000D880144625886219002DEFD17168304676
:10D4A0001436FCF736FEBE42E4D39D4B5A78022A6E
:10D4B00040F2EC8000225A701A789A489A4901602A
:10D4C000022A00F2DD8002EBC201984B02EB8102DE
:10D4D00003EB4202964C104622601CF043F8954A3A
:10D4E0001378A3F1170102290FD9934911F83300DA
:10D4F000002840F00381D8000144497829B18F49C0
:10D5000011F833300BB9182313708D4B9A78042A15
:10D5100000F0EB8032B91A88B2F5F07F84BF4FF487
:10D52000F0721A80874D884A2B681A40002A00F052
:10D53000EE80DE0700F1B580580400F1B9801907CC
:10D5400000F1BD809A0100F1C1809B0400F1C6800A
:10D5500023689A8CD98C914224BF00229A84FEF7CA
:10D560001FFF23F0DFF910B9784819F0D5FB2AF036
:10D57000A9FD0021302276482FF07FF8754B2568F1
:10D5800003F1500102E0043399427DD01A78002A59
:10D59000F9D19C78D8788442F5D26F496F4B0A70E4
:10D5A00028461D6020F038F96D4B6E4A1E786E4992
:10D5B0006E486F4B1160C825642212FB06526D4CF9
:10D5C000006B31F8041C5A60002221809A60DA60F6
:10D5D0001A615A619A61DA6183F8202083F8212068
:10D5E00008B115F083FB644B9FED645A1B88644AB5
:10D5F0009FED646A5579644C64496548086006EE9D
:10D60000903AF8EEE66A1388C5EE265A07EE103A0D
:10D6100053881279C4ED005A07EE903AB8EEC77AF3
:10D620005C4BF8EEE77A1D725A7227EE067A67EEC7
:10D63000867ABDE8F04783ED017AC3ED007A17F0F2
:10D640009DB863799B077FF424AF716894F804A0B8
:10D650003046FCF75EFD3388BAEB133F0BD173887D
:10D660007068AA1FC3F30B039A4204F10601A8BF16
:10D670001A462CF081FD1436BE42FFF4FBAE14E7CF
:10D6800000221A70294A25E7012286E72649254803
:10D6900002EB420201EB82011A780160022AEFD804
:10D6A00011E73D48FCF76CFD2B6858047FF547AF48
:10D6B0003A48FCF765FD2B6819077FF543AF3848FA
:10D6C000FCF75EFD2B689A017FF53FAF46F209003B
:10D6D000FCF756FD2B689B047FF53AAF3148FCF709
:10D6E0004FFD4020FCF74CFD32E71A8BB2F57A7FF4
:10D6F000BFF418AF4FF47A721A8313E7D8000D18ED
:10D700006D68002D7FF4F8AE17251570F4E643F030
:10D7100008032B600DE700BFC00500088801000862
:10D7200095550020E8540020AC550020B496002008
:10D73000E45400209039002028EC03080CD9030899
:10D74000D46D0020C497002009600002685E0020AC
:10D75000E0210020943900207C1C002014220020AD
:10D760004C50002000A90020FC36002098540020D6
:10D77000489200200637002020240020C0C9FB4822
:10D78000741E002017B7D1382424002078470020C9
:10D790003661023D54470020086000020920000263
:10D7A00001600002094000020740000800800008F4
:10D7B0002DE9F0430B684A680B388BB00C46D51A3C
:10D7C000EF2800F27881DFE810F07C017601760125
:10D7D0007601760176017601760176017601760191
:10D7E0007601760176017601760176017601760181
:10D7F00076017601760176017601A902760186022C
:10D800007601770276017601760170027601C40115
:10D810007601AC0176019B0176019401760112023A
:10D820007601520176017601760176014D0176018D
:10D830007F04760176017304760176017601760124
:10D84000760176016F047601760176015104760146
:10D85000A004760176018B047601760176017601CB
:10D86000760176017601F00076011B047601C8038B
:10D8700076019A037601E603760176017601760158
:10D8800076017601760176017601760176017601E0
:10D8900076017601760176017601760176017601D0
:10D8A00076017601760176017601760176017601C0
:10D8B00076017601760176017601760176017601B0
:10D8C00076017601760176017601760176017601A0
:10D8D0007601760176017601760176017601760190
:10D8E0007601760176017601760176017601760180
:10D8F0007601760176017601760176017601760170
:10D90000760176017601760176017601760176015F
:10D91000760176017601760176017601760176014F
:10D92000760176017601760176017601760176013F
:10D93000760176017601760176017601760176012F
:10D94000760176016E0347032E037601F102E602AB
:10D95000660576015A052B0519051205E8047601BE
:10D96000D50476017601C604CB05C205AF05730563
:10D97000F605E10506067601760176017601760167
:10D9800076017601760176017601760176017601DF
:10D990007601DB0276017601450276017601760199
:10D9A00076017601760176013A020846FCF73EFEE2
:10D9B00005461FF0DDFFFF2854D0B5F57A7F80F0D3
:10D9C0003A850AAF002307F8243DEE0839460DF1E9
:10D9D00003008DF8033001361FF0AAFF9DF80330D5
:10D9E000F6B205F00705B34205F1010503D19DF834
:10D9F0000430AB4203D0294630461FF0A5FF94E81F
:10DA00000C009B1A012B2DDD531C0AA82360002358
:10DA1000157800F8253D1FF07FFF9DF80330AB42DD
:10DA20000AD0B24B1B683BB19A79AA4204D31B6857
:10DA30001B690BB12846984723685A1C2260384658
:10DA400000221C788DF804201FF05AFF9DF8043046
:10DA5000A34207D0A54B1B6823B11B685B690BB1C0
:10DA600020469847012318460BB0BDE8F083A04933
:10DA7000A1FB05216A1A01EB52018908C1EBC10221
:10DA8000B5EB020817D1C9B24E1EF6B20029E9D093
:10DA9000DFF8609201365A1C226093F90010954B12
:10DAA000002593F902208A4203F1080300F09E84C6
:10DAB0000135062DF5D14FF0FF3318460BB0BDE808
:10DAC000F0838D49102D4FF0000328BF10250B6007
:10DAD0004B608B60CB600B74002DC3D023685A1948
:10DAE0000133236013F8010C01F8010B9A42F7D1BE
:10DAF000B8E75A1C0A60814A1B7853750123B2E7C4
:10DB00005A1C0A601E781F2ED5D8052DD3D1084681
:10DB1000FCF774FD7A4B43F8260018F0BFFF012391
:10DB2000A1E7774D05F140062046FCF77FFD23680D
:10DB3000A5F88000591C1A46216012F8021B85F8CE
:10DB4000821022605B7885F883300435AE42EBD1D9
:10DB500088E75A1C0A60694E1B7833720846FCF746
:10DB600065FDB0832046FCF761FD30832046FCF75D
:10DB70005DFD236870835A1C22601B78F374082DA6
:10DB80007FF670AF2046FCF751FDF0842046FCF78D
:10DB90004DFD0C2D30857FF665AF23681A46591C64
:10DBA000216012F8021BB17722605B7886F8203082
:10DBB0002046FCF73BFD102DB0847FF653AF236861
:10DBC0005A1C22601B78F3722046FCF717FD23686D
:10DBD000F0605A1C22601A783274162D7FF642AF1C
:10DBE0009A1C22605B7886F8213001233BE75A1C9F
:10DBF0000A601A780E2A3FF65EAF991C21605878A9
:10DC000003283FF658AF3F4D02EB42025200A918DD
:10DC1000DE1C487126609878A8541A1D2260DA78B4
:10DC20004A705A1D22601A798A709A1D22605A79A8
:10DC3000CA70DA1D22609B790B71012313E7324B06
:10DC40001B78DB073FF537AFFEF7CCFDFFF706FC8F
:10DC5000012308E75A1C0A601A780F2A3FF62BAFF7
:10DC6000991C2160C2EBC202284958788854D81CFC
:10DC700020600A4499785170191D2160D9789170FB
:10DC8000591D21601979D170991D2160597911713F
:10DC9000D91D21609979517103F108012160DB7967
:10DCA00093711BF0F1F80123DDE65A1C0A60184A53
:10DCB0001B7813700123D6E60846FCF7B7FC154D18
:10DCC00028602046FCF7B2FC68602046FCF7AEFCFA
:10DCD0000123A860C7E6104D00232B600846FCF71F
:10DCE0008DFC2B68184328600123BCE6E455002016
:10DCF00025499224685E00209A550020B0720020C9
:10DD00000C910020F0340020C4510020F048002085
:10DD10009039002050330020C49700205A1C0A601C
:10DD20001E78132E3FF6C7AE9A1C0A6000205D785D
:10DD3000A249024605E00132242A3FF4BCAE11F8A4
:10DD40000C0C854201F10C01F5D19D489D4902EB77
:10DD5000420210F8222001F82620D81C206001EB96
:10DD6000860299785170191D2160D8789070581DDD
:10DD7000206095491B790868D3702AF031F971E663
:10DD80000846FCF753FC914DA8812046FCF74EFC59
:10DD90000123688167E68E4B1B78D9073FF562AE99
:10DDA0008C4B4FF4C8721A8001235CE6092D7FF674
:10DDB00082AE894F1A46591C3E68216012F8021B38
:10DDC000317022605A78B270DA1C22609A78642A24
:10DDD00003F10401A8BF642272712160DA78642A19
:10DDE00003F10501A8BF6422B27121601A79F271B2
:10DDF0009A1D22605A79642A28BF6422D91D327282
:10DE000021609A79F27003F108022260DB793371A4
:10DE10002046FCF70BFC0A2D708140F079832AF034
:10DE200051F901231FE6684A1068DA1C01462133C4
:10DE3000951E256012F8035C0D70551E256012F8C2
:10DE4000025C4D70226012F8015C8D7003329A42C0
:10DE500001F10301ECD17CE05A1C0A601A785F4999
:10DE6000002A00F0E4820A7842F00202981C0A704C
:10DE70005B4D20605B782B702046FCF7BFFB686031
:10DE80002046FCF7BBFBA8602046FCF7CFFBA8812F
:10DE90002046FCF7CBFB534A6882137843F0020319
:10DEA00013700123DFE5C5F34705122D3FF603AEDE
:10DEB000BDB10AAB0DF1020703EB45083E46A8F1E0
:10DEC00026082046FCF7B2FB26F8020FB045F8D131
:10DED000454B37F8022F23F8022FBE42F9D1112DFE
:10DEE00009D8424A6B00023B13440021223223F836
:10DEF000021F9342FBD13E4A01231370B3E508464B
:10DF0000FCF794FB2046FCF791FB2046FCF78EFBC8
:10DF100023682D4F9A1C3E6822605A7886F82F207D
:10DF2000DA1C22609A7886F83A201A1D2260DA7884
:10DF300086F83B20073323602046FCF777FBF08709
:10DF400020463E68FCF772FB112DB08700F28A82F2
:10DF500038681BF02DF8012385E55A1C0A601A4F1A
:10DF6000DFF898801B783E6888F805300846FCF793
:10DF70005DFB308420463E68FCF758FB052D70841D
:10DF800000F27E82FEF70CFA20F0A0FF38681BF04A
:10DF900023F9012367E51A46591C21600B4912F841
:10DFA000020BC870226013495A780A70DA1C22608A
:10DFB000114A9B78D370012355E500BF24C903089B
:10DFC00010C9030894390020E4540020F8360020DA
:10DFD000C4510020A2A80020E85400206154002071
:10DFE00064540020CC3E00208E3C0020903C002059
:10DFF000B43C0020103A0020FC3900209C5E002038
:10E000001A46591C2160B34E12F8021BB1702260EF
:10E01000B1495A780A70DA1C2260B04D9A782A7198
:10E020001A1D2260DB78092BA8BF09232046AB709C
:10E03000FCF7FCFA236862682880D11A012905DD03
:10E040002046FCF7F3FA626823686882934240F046
:10E050004D82FEF7A5F9236862689A423FF402AD4B
:10E060005A1C22601B78EB700123FCE41A46591CF1
:10E0700021609B4D12F8021B297022605B786B7047
:10E080002046FCF7D3FA236868805A1C22601B786C
:10E090002B712046FCF7CAFA2368E8805A1C2260DC
:10E0A0001B782B720123DEE4FDF7FAF80123DAE492
:10E0B0008C4A03F108000133236013F8011C02F8B5
:10E0C000011F9842F7D1CDE4591C1A4621608649B8
:10E0D00012F8020B887022605B784B700123C2E457
:10E0E000824A1278012A3FF6BDAC19465A1C2260BA
:10E0F0007F4A11F8020B9070216059781170D91C79
:10E1000021609B7853700123ADE45A1C0A601E788D
:10E11000112E3FF6D0AC9A1C0A60764D5B7805F85C
:10E1200016300846FCF782FA40F6CA039842A8BFA8
:10E13000184640F2EE239842B8BF18466E4BA0F244
:10E14000EE2083FB002305EB4605C017C0EBE3037D
:10E150006B70012387E40846FCF768FA674D288056
:10E160002046FCF763FA68802046FCF75FFA01233B
:10E17000A88078E4624F3B78002B3FF473AC614E8B
:10E1800000252046FCF752FA1BF032FB3B78A6EC48
:10E19000010A0135AB42F4DC64E40F2D7FF48BAC53
:10E1A0005A1C0A601D78072D3FF685AC0846564F6D
:10E1B00005EB4505FCF73AFAAD007E19B080204624
:10E1C000FCF734FAF0802046FCF730FA23683081FF
:10E1D0001A46591C216012F8021BB17222605B784A
:10E1E000F3722046FCF70AFA012378513BE4084613
:10E1F000FCF71CFA454A0123108034E45A1C0A60DB
:10E200001878050600F17A81414B1B78DC073FF551
:10E2100029AC032828BF0020FEF7C8FA012322E416
:10E220005A1C0A6008461D78FCF7E8F9804620462B
:10E23000FCF7E4F907462046FCF7E0F906462046DD
:10E24000FCF7F4F92046FCF7F1F923680133236069
:10E25000002D00F03781102D7FF404AC2D4BC3F856
:10E2600000805F600EB12C4B1E602C492C4B0222AB
:10E27000081F1A701FF06EFA0123FFF7F4BB244B3E
:10E280001B78D8073FF5EEABFEF7E2FAFFF7E6F8AA
:10E290000123FFF7E8BB1E4B1B78DA073FF5E2AB23
:10E2A000204A137843F0040313700123FFF7DBBB0C
:10E2B0001A46591C216012F8020B2260DA1C5978A8
:10E2C00022609A7824F04CFF00287FF4CBABFFF754
:10E2D000F2BB00BF9C5E0020284F0020D46D0020C0
:10E2E0004C500020AF7200208C240020C8970020E2
:10E2F000C9970020803E00201F85EB51345000203C
:10E30000C9510020384F0020D0500020E43F0020A9
:10E31000C451002018220020142400201C220020B8
:10E32000CE3E0020615400201A46591C21607F49CE
:10E3300012F8020B087022607D495A788A70DA1C44
:10E3400022607C4A9B7893700123FFF78CBB7A4B49
:10E350007A4918684A222BF00FFF0123FFF783BB8D
:10E3600019465A1C2260764A11F8020B107021607F
:10E3700059785170D91C21609B7893702046FCF726
:10E3800055F9704A0123D080FFF76DBB19465A1C1E
:10E3900022606D4A11F8020B10702160597851709B
:10E3A000D91C216099789170191D2160DB78D37098
:10E3B0000123FFF758BB0846FCF738F9634DA882E4
:10E3C0002046FCF733F9E8822046FCF72FF90123B9
:10E3D0002883FFF748BB0846FCF728F9554B00EBAC
:10E3E0008000400018800123FFF73DBB09EBC50703
:10E3F0002046B970FCF71AF9216829F835000B4658
:10E400004A1C226013F8022BFA7023604B783B7190
:10E41000CB1C23608B78BB710B1D236008F10108B6
:10E42000CA787A7146457FF436ABFFF71BBB0A7892
:10E4300002F0FD021AE501AF38461FF055FABDF8AB
:10E440000430AB423FF4DBAA414B1B68002B3FF486
:10E45000D6AA1B689B69002B3FF4D1AA284698478F
:10E46000FFF7CDBA23683868591C1A46216012F8A4
:10E47000021B80F8311022605B7880F8323068E54A
:10E480002046FCF7D3F8A8F80A002046FCF7CEF89F
:10E49000A8F80C0020463E68FCF7C8F8B084204677
:10E4A0003E68FCF7C3F80D2DF0847FF66BAD204677
:10E4B000FCF7BCF8A8F80E002046FCF7B7F8A8F85F
:10E4C00010005FE5234B1020C3F800805F6019F057
:10E4D0005FFE214A137843F001031370002E3FF4CE
:10E4E000C1AA1E4A01231660FFF7BDBA5A1C22605A
:10E4F0001B78003318BF0123F371AAE500F07F00F9
:10E50000032828BF00200FF031F90123FFF7ABBA31
:10E5100023683A68591C2160197851720B2D3FF419
:10E520007EAC991C21605B78537078E49C5E00207F
:10E53000F8360020FC390020E454002040D60308BF
:10E54000F823002034500020E83F0020D46D002044
:10E55000E4550020103F00206154002014240020C6
:10E5600008B516F023F9FBF751FE16F007F9FEF790
:10E5700075FF0120BDE8084019F0F2BD2DE9F04F0C
:10E58000013085B0C3B203930B4602918B4C8C4E85
:10E59000002B00F099808B4D8B4FDFF830921FF0ED
:10E5A0005BFC4FF4FA7A4FF0100C4FF47A70D9F804
:10E5B0000430C3F30803002B40F0DE80EFF3118337
:10E5C000002B40F0D9802968A26800BF2B689942CF
:10E5D000F9D1D7F800E000FB0EF39B1AB3FBFEF372
:10E5E00000FB01314FF0010E0191D9F80430C3F363
:10E5F0000803002B40F08780EFF31183002B40F0DD
:10E6000082802B68A16800BF2A689342F9D1D7F8AD
:10E6100000B000FB0BF2521AB2FBFBF200FB03232B
:10E62000019A9B1AB3F57A7FDFD3BAF1010ABED102
:10E63000039B002B40F0BD804FF47A7ADFF88C9179
:10E6400050464FF0100CD9F80430C3F30803002BE8
:10E6500075D1EFF31183002B71D12968A26800BF37
:10E660002B689942F9D1D7F800E000FB0EF39B1A12
:10E67000B3FBFEF300FB01314FF0010E0191D9F81D
:10E680000430C3F3080313BBEFF31183FBB92B680A
:10E69000A16800BF2A689342F9D1D7F800B000FB07
:10E6A0000BF2521AB2FBFBF200FB0323019A9B1AF6
:10E6B000B3F57A7FE3D3BAF1010AC4D1029B013BDF
:10E6C0000293002B7FF467AF05B0BDE8F08FEFF346
:10E6D00011888CF31288A1682368DB0344BFC6F855
:10E6E00000E0A1682B6832685FFA88F888F3118827
:10E6F000D7F800801A4400FB08F35B1AB3FBF8F369
:10E7000000FB0233D2E7EFF311888CF31288A16883
:10E710002368DB0344BFC6F800E0A1682B683268B9
:10E720005FFA88F888F31188D7F800801A4400FB54
:10E7300008F35B1AB3FBF8F300FB023370E7EFF367
:10E7400011828CF31288D4F808E02368D90303D52A
:10E7500001233360D4F808E02B683168D2B282F329
:10E7600011883A68194400FB02F3A3EB0E03B3FBD4
:10E77000F2F300FB01317FE7EFF311828CF3128893
:10E78000D4F808E02368D90303D501233360D4F813
:10E7900008E02B683168D2B282F311883A681944D4
:10E7A00000FB02F3A3EB0E03B3FBF2F300FB01311A
:10E7B00018E7184629F0BCF83EE700BF10E000E07B
:10E7C0007CA8002080A8002084A8002000ED00E0A4
:10E7D000204B5B68C3F3080330B4BBB9EFF311837C
:10E7E000A3B91D4B1D4C1868A16800BF1A68904260
:10E7F000F9D11B4B1C684FF47A7202FB04F3591ACF
:10E80000B1FBF4F130BC02FB00107047EFF3118252
:10E81000102383F3128811498C680B6813F4803F2E
:10E82000104B02D0012018608C680B49D2B20D68E1
:10E83000186882F311880A4B19684FF47A722844D9
:10E8400002FB01F31B1B30BCB3FBF1F302FB0030F6
:10E85000704700BF00ED00E080A8002010E000E05D
:10E8600084A800207CA800202DE9F84F8046FFF7FF
:10E87000AFFF254E2549DFF8A0E0254A254D844607
:10E8800010274FF47A740120DEF80430C3F3080334
:10E89000D3B9EFF31183BBB90B68D2F808A000BF5E
:10E8A000D1F800904B45F7D1D6F800B004FB0BF936
:10E8B000A9EB0A09B9FBFBF904FB0393A3EB0C03D7
:10E8C0004345E1D3BDE8F88FEFF3118A87F312884F
:10E8D000D2F808B01368DB0344BF2860D2F808B050
:10E8E0000B68D5F800905FFA8AFA8AF31188D6F897
:10E8F00000A0994404FB0AF3A3EB0B03B3FBFAF368
:10E9000004FB0933DAE700BF84A8002080A80020B8
:10E9100010E000E07CA8002000ED00E02DE9F04FC1
:10E92000DFF830C1474A4849484E494D80461027D4
:10E9300018F1FF38C0F08480DCF80430C3F308031A
:10E94000002B5CD1EFF31183002B58D10B68946836
:10E9500000BF08688342F9D1D6F800904FF47A706E
:10E9600000FB09FEAEEB040EBEFBF9FE00FB03EE5E
:10E97000DCF80430C3F308034FF47A740120FBB9C8
:10E98000EFF31183E3B90B68D2F808A000BFD1F808
:10E9900000904B45F7D1D6F800B004FB0BF9A9EB7A
:10E9A0000A09B9FBFBF904FB0393A3EB0E03B3F5D0
:10E9B0007A7FBDD2DCF80430C3F30803002BDFD02C
:10E9C000EFF3118A87F31288D2F808B01368DB03DB
:10E9D00044BF2860D2F808B00B68D5F800905FFA01
:10E9E0008AFA8AF31188D6F800A0994404FB0AF346
:10E9F000A3EB0B03B3FBFAF304FB0933D5E7EFF307
:10EA0000118487F31288D2F808901368D80303D5CD
:10EA100001232B60D2F808900B682868E4B284F3D5
:10EA20001188D6F800A04FF47A7400EB030E04FBB3
:10EA30000AF3A3EB0903B3FBFAF304FB0E3E97E7DB
:10EA4000BDE8F08F10E000E080A8002084A800203E
:10EA50007CA8002000ED00E030B4EFF31183102219
:10EA600082F312880649074C0A68074801320025DC
:10EA70000A602560DBB2026883F3118830BC7047FE
:10EA800080A800207CA8002010E000E00F4B1B882D
:10EA9000014643B90E4B0F4A1B7810680BB981F041
:10EAA0000101FBF797B80C4B5A691AB118B91A68EB
:10EAB000106058747047094A18681188084A92FB18
:10EAC000F1F2012102605974704700BF58A800207C
:10EAD0005AA800205CA8002060A8002078A8002088
:10EAE00020A1070038B5254B9C68236B73B1A36D3B
:10EAF000626BCAB1998A1A88C90592B201D5D20748
:10EB000000D438BD4FF6F7721A8038BDA36D9989CD
:10EB10001A88890692B2EBD59206E9D5E26ACAB1A3
:10EB2000988880B29047E2E799891A880D0692B2D8
:10EB3000E0D51006DED5A26A616A8A4219D0A169C1
:10EB40002569885C98800132B2FBF5F105FB112242
:10EB5000A262CFE79B88E2696169DBB28B54E2690C
:10EB6000E068A36D0132B2FBF0F100FB1122E2611B
:10EB7000BEE7DA6822F08002DA60BBE720330020CB
:10EB80002DE9F04FB0F908502DED048B0D81EDB259
:10EB9000382D87B00C4600F096828046914634D9D5
:10EBA000802D00F0E48078D8522D00F0948040F25F
:10EBB0006A82542D00F0AD826E2D40F01F81814B92
:10EBC0000A681B88804DFF2BA8BFFF23511C2160C2
:10EBD0001370A96881F3100189B22046FBF77AFD12
:10EBE0007A4B20461988FBF775FD296801F30F0160
:10EBF00089B22046FBF76EFD01252B46284663812E
:10EC000007B0BDEC048BBDE8F08F042D5AD040F264
:10EC10000582202D00F08F8040F24082242D00F0EC
:10EC20008482282D40F0EA800B68DFF8C481684EAA
:10EC3000591C022221601A70236806275A1C226080
:10EC40001F7023680A22591C21601A70236801254D
:10EC50005A1922601D70B8F800102046FBF73AFDE3
:10EC6000B8F802102046FBF735FD23685A192260D8
:10EC70001F7023685022591921601A7023680022DE
:10EC8000591921601A7031882046FBF723FD7188DD
:10EC90002046FBF71FFD2B46B0E7822D23D0C0F0A6
:10ECA0005682A02D00F04782FE2D40F0A780494DEE
:10ECB00005F1080635F8021B2046FBF70BFDB542AF
:10ECC000F8D199E72A4644492046FBF7BBFC0021CE
:10ECD0002046FBF7FFFC22680021531C012523601E
:10ECE0002B4611708AE70B683C4A374D11783C4A35
:10ECF000581C20601970D1882046FBF7EBFC314B83
:10ED000022681B88FF2B02F10101A8BFFF232160AD
:10ED10001370A96881F3100189B22046FBF7DAFC71
:10ED2000296801F30F0189B22046FBF7D3FC2D4B74
:10ED300022681978D1E70B68294D591C6A7821603F
:10ED40001A7023682A78591C21601A702368AA78DF
:10ED5000591C21601A70E9882046FBF7BBFC236828
:10ED60002A79591C21601A7022686979B5E71E4E0C
:10ED70001E4FDFF880A0DFF8809006F10D080A250D
:10ED800017E0322D00F06281A5F13C00C0B21328DB
:10ED900040F2638100232268511C216015702268B3
:10EDA000464502F10101216013703FF425AF16F8CA
:10EDB000015B0A2DE5D1B9F80030FF2BA8BFFF2376
:10EDC000DBB2E8E780520020845200203C92002011
:10EDD000F4240020DC51002064F70308C75200200F
:10EDE0007C54002042920020F5C8030867666666DE
:10EDF000882400200C2500203C250020A5F10A03D2
:10EE0000E72B00F2EA80DFE813F08805E800E8006D
:10EE1000E800E800E800E800E800E800E800E800B2
:10EE2000E800E800E800E800E800E800E800E800A2
:10EE3000E800E800E800E800E8005705E800E8001E
:10EE4000E8004605E800E800E8004105E8000005A4
:10EE5000E800E704E800DB04E800D604E800630407
:10EE6000E8005004E800E800E80047024704E80032
:10EE7000CC04E800E800C304E800E800E800E8008B
:10EE8000E800A504E800E800E800E8008904E800DC
:10EE9000F207E8003602DA07E800E800E800E800D8
:10EEA000E800E800E8009607E8006B07E8000807BC
:10EEB000E800BE06E800AD06E800E800E800E8006B
:10EEC000870654064B0623061106EB05D5059A0561
:10EED000C003E80086036903E800E800E800E800F2
:10EEE0005D03E800E800DF03E800E800E800CE0387
:10EEF00001044D030F03E800E800E800FE02EB0206
:10EF0000E102E800E800E800E800E800E800E800C6
:10EF1000E800E800E800E800E800E800E800E800B1
:10EF2000E8008706E800E800E800E800E800E800FC
:10EF3000E800E800E800E800E800E800E800A902CE
:10EF4000E800E800E800E800E800E800E800E80081
:10EF5000E800E800E800E800E800E800E800E80071
:10EF6000E800E800E800E800E800E800E800E80061
:10EF7000E800E800E800E800E800E800E800E80051
:10EF8000E800E800E800E800E800E800E800E80041
:10EF9000E800E800E800E800E800E800E800E80031
:10EFA000E800E800E800E800E800E800E800E80021
:10EFB000E800E800E800E800E800E800E800E80011
:10EFC000E800E800E800E800E800E800E800E80001
:10EFD000E800E800E80078024E02742D00F0278176
:10EFE000772D00F03581F52D00F04987762D00F062
:10EFF0002087472D01F02380292DD8F8003001F01B
:10F000000780392D00F0BA87212D00F0C3872846EC
:10F010004146FEF7CDFB054603B2EFE5022D00F0B9
:10F02000FE8000F2EB80012D7FF4E8AE0B68002239
:10F03000591C21601A7023685A1C22601D702268B6
:10F040002421531C23602B461170D7E5BAF80030F9
:10F05000FF2BA8BFFF23DBB29DE61CF065FE002856
:10F060003FF498AE03780A2B00F20381B0F9023026
:10F0700087FB0312DB17C3EBA2039BB2FF2BA8BFD6
:10F08000FF23DBB287E6442D7FF4B8AE002A3FF4BD
:10F09000B3ADA04B136001252B46AFE5052D7FF4E2
:10F0A000ADAE0B229C492046FBF7CCFA08229B49C7
:10F0B0002046FBF7C7FA0125072299492046FBF7AE
:10F0C000C1FA2B469AE50A68964B0125511C21602E
:10F0D00015702268052150192060117022680A21DC
:10F0E00050192060117022680021501920601170A1
:10F0F00022681978501920601170226859785019C7
:10F100002060117022689978531923602B46117082
:10F1100074E50B6800215A1C2260197022680125D1
:10F12000531923602B46117068E57F4B1968204600
:10F13000FBF7B8FA60E57D4B08461968FBF7B2FAB1
:10F140007B4B20461968FBF7ADFA7A4BEEE7DFF808
:10F150000892794F09F10E064FF00A081DE0B8F148
:10F16000500F32D0B8F1320F31D0A8F13C00C0B20C
:10F1700013282FD90025294623685A1C22602046CF
:10F1800083F80080FBF7A6FA29462046FBF7A2FA8F
:10F19000B1453FF431AD19F8018BB8F10A0FDED15A
:10F1A000664B9D68196805EB85054FF6FF736D008A
:10F1B0009D42A8BF1D469942A8BF194625EAE5759C
:10F1C00021EAE171ADB289B2D6E75D4BE9E797E894
:10F1D0002200E8E71CF0A8FD0028CBD003780A2B1A
:10F1E000C8D8B0F90430B0F9061003EB830383F3F9
:10F1F000500521EAE171ADB289B2BDE70B68022288
:10F20000591C21601A70236801255A1922601D704B
:10F2100022680021531923602B461170EEE404226A
:10F22000484920460125FBF70DFA2B46E6E4D8F8BD
:10F230000030D8F804209A421EBF5A1CC8F800209B
:10F240001978414A08BF00212046FDF727FAD3E488
:10F25000D8F80030D8F804209A421EBF5A1CC8F8CB
:10F2600000201978394A08BF00212046FDF716FA18
:10F27000C2E4002305E7236800255A1C22601D70A4
:10F2800023685A1C22601D7023685A1C226029467C
:10F290001D702046FBF706FA002120460125FBF7EA
:10F2A00001FA2B46AAE42A4B03F17005226819786B
:10F2B000501C2060117022685978501C2060117019
:10F2C00022689978501C206011702268D978501CEF
:10F2D0002060117022681979501C2060117022681A
:10F2E0005979501C20601170226899790733501C9D
:10F2F000AB4220601170D9D17EE4164D2046A98919
:10F30000FBF7E8F9698920460125FBF7E3F92B466D
:10F3100074E400BF81C300086CF7030878F70308A2
:10F3200084F70308A3960020C4970020107AFF1FDB
:10F33000147AFF1F187AFF1F04250020B82400202C
:10F34000F82400205CF7030859C30008DDC2000858
:10F35000F0480020F8360020E5C803082368DFF8ED
:10F3600030C3591C9CF8002021601A709CF80030B2
:10F37000002B3FF441ACB24EB24DB348B349002329
:10F38000226816F8017F02F1010EC4F800E0177040
:10F39000226815F8017F02F1010EC4F800E0177031
:10F3A000226810F8017F02F1010EC4F800E0177026
:10F3B000226811F8017F02F1010EC4F800E0177015
:10F3C0009CF8002001339342DADB15E4A04BA149FD
:10F3D000B3F9003081FB0321DB17C3EBA10107E484
:10F3E00022689D4B501C1978206011702268597852
:10F3F000501C2060117022689978501C2060117098
:10F400002268D97869E4954D2046A98AFBF762F90C
:10F41000E98A2046FBF75EF9298B20460125FBF798
:10F4200059F92B46FFF7EABBDFF868E20027FEB286
:10F43000714600232268501C206016702268501C00
:10F4400020601370226811F8010F0133551C062B40
:10F4500025601070EED10137062F0EF1060EE6D1B1
:10F460007F4900232268501C206017702268501CBE
:10F4700020601370226811F8010F0133551C0B2B0B
:10F4800025601070EED123687649581C0722206051
:10F490001A7023680022581C20601A70226891F8A4
:10F4A000F0101AE42368704A694910786F4A5D1CAD
:10F4B0002560187023689278581C20601A702268A2
:10F4C00089780AE46A4952232268501C206013702C
:10F4D00011F8013F002BF7D1FFF78EBB65480023E1
:10F4E0002268056803EB4301561C6D5C26601570AD
:10F4F000026825680A446E1C527826602A700268E9
:10F5000025680A4401339278691C0A2B21602A700D
:10F51000E6D1FFF771BB584D23682A68591C127851
:10F5200021601A702B6822689978531C236000238D
:10F5300011702A6821681A4401335279481C032B40
:10F5400020600A70F5D123682A68591C127A21605C
:10F550001A7023682A68591CD27821601A702368AF
:10F560002A68591C127921601A702B682046598923
:10F57000FBF7B0F823682A68591C527A21601A7088
:10F580002B6822685978FFF7A8BB3C4B20461968C6
:10F59000FBF788F83A4B204619880125FBF79AF8C3
:10F5A0002B46FFF72BBB374D20462988FBF792F8F7
:10F5B00069882046FBF78EF8A98820460125FBF7CD
:10F5C00089F82B46FFF71ABB2F4D05F16006A98875
:10F5D0002046FBF77FF8E9882046FBF77BF829896E
:10F5E0002046FBF777F82368AA7A591C21601A7025
:10F5F0002368EA7A591C21601A7055F80C1B2046C2
:10F60000FBF750F8AE42E2D1FFF7F6BA22681F4B83
:10F610001C491878551C2560107022685878551CB4
:10F620002560107022689B78501C20601370C98878
:10F6300020460125FBF74EF82B46FFF7DFBA00BF47
:10F6400003400020134000203340002023400020CE
:10F65000FC39002067666666E83F0020D46D002014
:10F66000EF9100200C9100209C5E0020F8360020D5
:10F67000B4C80308E4540020E85400208854002053
:10F680008C54002034500020D0500020F82300205B
:10F6900001400020CB9100202268012153182360F3
:10F6A0000D460B461170FFF7A9BAB14DB14E05F1E9
:10F6B000300795F902100023F2568A4200F0408488
:10F6C0000C33482BF8D10835AF42F2D1FFF794BA8A
:10F6D000A94B03F15A0522685979501C206011701A
:10F6E00022681978501C2060117022685978501CCB
:10F6F0002060117022689978501C20601170226877
:10F70000D978501C20601170226819790633501C7A
:10F710009D4220601170DED1FFF76EBA2368974DCD
:10F72000591C2A7821601A7023686A78591C216054
:10F730001A7069882046FAF7CDFF23682A79591C88
:10F7400021601A70E9882046FAF7C4FF2268297AF6
:10F75000FFF7C3BAFBF74AFC2368894D002803F181
:10F7600001010CBF0222032221601A702988204661
:10F77000FAF798FFE9682046FAF794FFFBF786FB53
:10F78000012501462046FAF78DFF2B46FFF736BAD2
:10F7900008227C4920460125FAF754FF2B46FFF743
:10F7A0002DBA2268784B501C99782060117022681D
:10F7B0005978FFF792BA734B2268597DFFF78DBADB
:10F7C000724D05F1800655F8041F2046FAF76AFFCE
:10F7D000AE42F8D1FFF710BA6D4D05F14006B5F80D
:10F7E00080102046FAF776FF236895F88220591C8E
:10F7F00021601A70236895F883200435591CAE42A5
:10F8000021601A70EBD1FFF7F7B95E4D23682A7AB1
:10F81000591C21601A70A98B2046FAF75BFF298BCF
:10F820002046FAF757FF698B2046FAF753FF236803
:10F83000EA7C591C21601A70E98C2046FAF74AFFCD
:10F84000298D2046FAF746FF2368AA7F591C2160BC
:10F850001A70236895F82020591C21601A70A98C11
:10F860002046FAF737FF2368EA7A591C21601A709C
:10F87000E9682046FAF716FF23682A7C591C2160A4
:10F880001A70226895F82110FFF727BA414B2268B9
:10F890001978FFF722BA404D20462988FAF71AFF57
:10F8A000A9882046FAF716FF298920460125FAF78C
:10F8B00011FF2B46FFF7A2B9384D394F05F150061D
:10F8C00000212878374A0B4607E00133242B02F148
:10F8D0000C0200F0328312F80C1C8842F5D103EBC5
:10F8E0004303226807EB8303511C93F864302160C3
:10F8F000137023686A78591C21601A702368AA78EB
:10F90000591C21601A702368EA780435591CAE42EC
:10F9100021601A70D4D1FFF76FB9234829F0AAFEED
:10F9200000287FF769A9204B1D18226813F8011BD6
:10F93000501C9D4220601170F7D1FFF75DB91B4D3F
:10F9400020462988FAF7C6FE69882046FAF7C2FEE3
:10F95000B5F904301649DA1781FB0313C2EBA30390
:10F9600099B220460125FAF7B5FE2B46FFF746B9B6
:10F97000685E002068720020F03400204C500020A7
:10F980006C1C0020B07200208C2400200891002004
:10F990000C91002090390020503300209439002031
:10F9A000B4C803081CC903089A55002090540020CD
:10F9B00067666666B04B20461988FAF78BFEAF4B38
:10F9C00020461988FAF786FEAD4B21681A78012582
:10F9D0004B1C02F0010223602B460A70FFF70EB9A0
:10F9E000A84B22681B78A84D511C03F0020321602C
:10F9F000137023682A78591C21601A7069682046A0
:10FA0000FAF750FEA9682046FAF74CFEA98920466D
:10FA1000FAF760FE698A2046FAF75CFEA98A20465A
:10FA20000125FAF757FE2B46FFF7E8B8974E3378D3
:10FA3000002B3FF4E1A8964F002537F8021F20461F
:10FA4000FAF748FE337801359D42F6DBFFF7D4B86C
:10FA5000904D914EDFF87882DFF87892DFED8F8A53
:10FA6000DFED8F9A9FED8F9A05F1200708E0204681
:10FA70000435FAF72FFEAF4206F118063FF4BCA892
:10FA8000717C0029F3D095ED008AB0EE480A2AF087
:10FA9000E7FC98F80030002B40F0C08381B2E6E725
:10FAA0001022814920460125FAF7CCFD2B46FFF7AD
:10FAB000A5B87E4E338AB3F5007F06F1340594BFB6
:10FAC00001270427403655F8041B91FBF7F1204627
:10FAD00089B2FAF7FFFDAE42F5D1754D754F05F1CC
:10FAE0000C06B5EC010AD7ED087A80EE270A2AF059
:10FAF000B7FC81B22046FAF7EDFDAE42F1D16E4D72
:10FB000005F10C0655F8041B204689B2FAF7E2FD10
:10FB1000AE42F7D1FFF770B80023DFF8BC91DFF8F1
:10FB2000BCB10393029304930593984601214FF6C9
:10FB3000FF7A07E008F10108B8F10B0F00F0C78267
:10FB400019F9011F4E1CF5D04AFA08F3D807F1D570
:10FB5000BBF8003043FA08F3DA07EBD504A8FBF74B
:10FB60004BF9E7E72368554A5549D078554A5D1C5B
:10FB70002560187023681278581C20601A7022685B
:10FB8000C978FFF7AAB800212046FAF7A3FD0021A3
:10FB90002046FAF79FFD00212046FAF79BFD2268D8
:10FBA000494D0023511C2160137022682968501CA4
:10FBB00091F82F102060117022682968501C91F86C
:10FBC0003A102060117022682968501C91F83B108F
:10FBD000206011702268511C216013702268511C32
:10FBE000216013702268511C216013702B6820461D
:10FBF000D98FFAF76FFD2B682046998FFAF76AFDC7
:10FC000023682A68591C92F8312021601A702B68E9
:10FC1000226893F83210FFF760B82C4D23686A7998
:10FC2000294E591C21601A7033682046198CFAF746
:10FC300051FD33682046598CFAF74CFD69892046FE
:10FC4000FAF748FDA9892046FAF744FD33682046B3
:10FC5000998CFAF73FFD33682046D98CFAF73AFDC4
:10FC6000E9892046FAF736FD298A20460125FAF768
:10FC700031FD2B46FEF7C2BF183F00201A3F00207F
:10FC8000CC3E00206154002064540020D855002050
:10FC9000AE8F0020C8360020E06B002000004042FC
:10FCA0000040744400E08244B8360020985400209C
:10FCB000D8660020B05E002080550020F836002075
:10FCC000FC390020103A0020E45400209C5E002003
:10FCD000FC6D00207083002004C90308E05400205C
:10FCE000BE4EF378002B00F08D8223680822591C49
:10FCF00021601A7023680122991821601A70236804
:10FD0000B74D591C2A7921601A702368AA78591CAA
:10FD100021601A7029882046FAF7DCFC698A20469F
:10FD2000FAF7D8FC2368F279591C21601A7022680E
:10FD3000E978FEF7D2BF1DF01BFEFF28064600F053
:10FD4000A18206A9002501F8125D0DF105008DF8CC
:10FD500005501DF0EDFD06A800F8115D1DF0DCFD5D
:10FD600006A800F8105D1DF0CBFD06A820F8085D80
:10FD70001DF0BAFD23685A1C22601E7023689DF88E
:10FD80000520591C21601A7023689DF80620591C13
:10FD900021601A7023689DF80720591C21601A7091
:10FDA00023689DF80820591C21601A70BDF81010B6
:10FDB00020460125FAF78EFC2B46FEF71FBF22686E
:10FDC000884B0125511C21601570226899785019C3
:10FDD0002060117022681978501920601170226813
:10FDE0005978531923602B461170FEF707BF7E4EDA
:10FDF0003378002B3EF400AF7C4F0025B8462368D3
:10FE000017F81520591C21601A7098F8011001EBA1
:10FE1000810101EB810101F2EE2189B22046FAF75E
:10FE200059FC337801359D4208F10208E7DBFEF703
:10FE3000E3BED8F800305A1CC8F800201B78002B0D
:10FE400000F05782102B07BF694A92E82200002574
:10FE500029462268501C206013702046FAF722FCC5
:10FE600029462046FAF71EFC624B20461968FAF72D
:10FE700019FC00212046FAF72DFCFEF728BFD8F820
:10FE80000030D8F804209A4240F057825A4BFF22A3
:10FE90001A724FF00008594D0DF028FC41463022EF
:10FEA000574885F800802CF0E8FB8DF810809DF80D
:10FEB00010300B2B00F2A082524F514E42469DF85B
:10FEC000103003EB430307EBC3035B7CE3B19DF806
:10FED000103003EB430307EBC3035B69A3B19DF849
:10FEE000103003EB430307EBC3032021586946F8A6
:10FEF0002200F9F7CFFC2B7856F82300F9F750FED3
:10FF00002A780132D2B22A709DF810300133DBB268
:10FF10008DF810309DF810300B2BD0D92368591C68
:10FF200021601A70B9F1000F3EF466AE364BC9F885
:10FF3000003001252B46FEF761BE00231B7AFFDE51
:10FF400023685A1C2260197029882046FAF7C2FBE0
:10FF50002368EA78591C21601A7023682A79591C91
:10FF600021601A702368AA79591C21601A702368CD
:10FF70006A79591C21601A70FFF7A5BB5A1CC8F892
:10FF800000201A780A2A00F022824FF0FF352B4613
:10FF9000FEF734BE1A46591CC8F800101B4D12F863
:10FFA000021B6970C8F800205A782A70DA1CC8F859
:10FFB00000209B78AB704046FAF738FBD8F8003049
:10FFC000E880591C1A46C8F8001012F8021B297163
:10FFD000C8F800205B786B71D7E700BF9C5E0020FB
:10FFE000D46D0020C9970020D8550020803E002005
:10FFF0001822002014240020841E00209B9600203C
:020000040801F1
:100000004C960020E06B0020396303087C540020EC
:100010005A1CC8F800201B780A2B00F02E81502BA8
:10002000B3D14046FAF702FBCD4E30804046FAF796
:10003000FDFA4FF0FF3570802B46FEF7DFBDD8F894
:100040000430D8F8005040465D1BFAF7D7FA052D6A
:10005000064600F20A8180252F464FF0010894E8F9
:100060000C009B1A103BDFF82C939D42C8BF9FB237
:10007000D9F80C309B1B9F423146204688BF9FB267
:10008000FAF710FBB8F1000F00F00481D9F80C303A
:10009000D4F80080F219934200D29F1BFBF79EF820
:1000A00041463A463046FBF719F92368A842034413
:1000B0002360B8BF002102DBFEF79EBD236801303C
:1000C0005A1C854222601970F8D1FEF795BDDFF801
:1000D000C8A24FF000084FF0080908F10108B8F174
:1000E000240F1BD0C8F1200209FA02F22AFA08F6FE
:1000F000A8F12003164329FA03F31E4306F0010278
:1001000000231343E9D05FFA88F027F063FF00284B
:10011000E3D0414604A8FAF76FFEDEE7914B1B7867
:10012000DB0700F1D68000268F4FB04602E0013693
:10013000242E0ED031463846FAF76EFE0028F6D04F
:10014000314604A8FAF768FE002856D108F10108E4
:10015000EDE7864B864EB3F850102046FAF7BAFA10
:10016000844B1988204689B2FAF7B4FA824B1A6890
:10017000530103F02001C2F340030B43C2F380019B
:1001800043EA4103C2F3C00143EA8103C2F34011D1
:1001900043EAC10102F0100211432046FAF79AFA2D
:1001A00002A904222046FAF74DFA23683178734AEF
:1001B000581C2060197011886429A8BF642120464A
:1001C000FAF788FA962D00F0898000212046FAF788
:1001D00081FA2168B8F1190348BFA8F11203A3F30B
:1001E000C4034A1C226020460B701A4603A901254D
:1001F000FAF728FA2B46FEF701BD414602A8FAF7A6
:10020000FBFDA3E72368B1785D4A581C2060197094
:1002100023681278591C21601A7070E5D9F80030F3
:1002200013F48053B4EEE88A67D0F1EE10FA11DBD4
:10023000B4EEC98AF1EE10FA62D8DFED527A9FED82
:10024000527A77EEC87AB4EEC78AF1EE10FAB0EEC1
:10025000678A55D94FF47A71B5EE408AF1EE10FAFB
:1002600040F2DC5308BF194601E44046FAF7DEF9D4
:100270004FF0000807460546F1E64046FAF7D6F982
:10028000424ED2E622680125531923602B46107096
:10029000FEF7B4BC39462046FAF71CFA23685A1C0C
:1002A000226083F80080D9F80C50D4F80080F2194D
:1002B000AA4200F2A380FAF791FF3A46414630463F
:1002C000FBF70CF823680125034423602B46FEF757
:1002D00095BC049B43F00103049324E723680322A5
:1002E000591C21601A7023687278591C21601A7099
:1002F0006FE7274A92E82200ABE5F1EE10FA77DBD0
:10030000F7EE007A78EE677AB6EE007AF0EE696A78
:10031000E7EE876A40F2E932FDEEE67A17EE901AD0
:10032000B1F5FA6FA8BF4FF4FA619142B8BF114618
:1003300089B2002B3FF49BAB8EE75A1C1946C8F8D4
:100340000020094811F8022B0272C8F800105B78EF
:100350004372042A22D9FF2A7EF4BDAC99E500BF7E
:10036000F4240020C4510020841E00204C030020EF
:100370009555002014A6002054670020DE3300208D
:10038000284F002000C0884400C0824488240020F8
:10039000103F00206C1C002090E33FF41E490978B8
:1003A000994205D8022A7EF496ACFF2B7EF493ACDA
:1003B000236801255A1922601D70B9F1000F3EF41F
:1003C0001BAC164BC9F800302B46FEF717BC9A1C25
:1003D000C8F80020124A59781170D91CC8F80010CA
:1003E00099785170191DC8F80010DB789370CCE52E
:1003F0004FF47A71FFF73BBB42468FE5AD1BFAF72E
:10040000EDFE2A4641463046FAF768FF236803446A
:100410002360FEF7F1BB00BFC95100208DC3000867
:10042000A39600202DE9F04F2DED028B91B00546EB
:1004300022F058FB814B1F7827B111B0BDEC028B25
:10044000BDE8F08F7E4B1A685205F6D57D4A1278CA
:10045000002A40F098817C4B1B78002B6DD07B4CA0
:100460007B4AD4F81C31EB1A934201F26C8494F865
:100470002471A7BBDFF80C82D8F80000F8F794FFCE
:10048000C0B201280ED9022841F09686714B1A7825
:10049000002A42F07580D4F82821AA1AB2F57A6FA2
:1004A00082F02A81D4F82C31002B46D094F82431E4
:1004B000C3B9694B1B689B7801211E3B00228B420C
:1004C00084F8241184F8382142F2BF80D8F8000063
:1004D000022104301CF098F994F8303110E0D4F87F
:1004E0002C3153B3D4F8343140F6B732EB1A93427F
:1004F00023D994F83031002B01F08085DFF8848116
:10050000013BDBB284F83031002B01F05485D4F884
:100510002C7194F8382117F8011B94F83931D8F868
:100520000000C4F82C710A44013384F8382184F89F
:100530003931F8F73DFFC4F834511BF05BFD474BF0
:100540001B786BB1DFF84091D9F8003043B1444BD0
:100550003E4C1B68D4F83C219A1A632A00F2F681BB
:10056000404C2378022B01F03685DFF8208198F883
:100570000030032B01F00B853B4B1B7873B13B4FD5
:100580003B685BB1314CFEF723F9D4F8443101905C
:1005900044F61F62C31A934200F2BA82344B1B78AE
:1005A000002B75D1334B1B7843B1284CD4F89432CF
:1005B00003F5C333A0339D4281F086832E4B1B7815
:1005C000002B3FF43AAF214E2C4C2D4D06F2B527AF
:1005D0002068F8F7E9FE00283FF42FAF2068F8F70D
:1005E000DBFE2B7880465A1E33B120682A70F8F75C
:1005F000DBFE0028F2D120E703223946781E2CF0DA
:1006000022F896F8B43296F8B52286F8B78283F4C9
:100610007F4383F0FF039B1A1FFA88F89BB2B8EB65
:10062000132FD5D196F8B622DBB29A42D0D1781EDC
:100630001BF0F0FB2B7818442870C9E7D841002044
:10064000708300207C92002086920020901E002063
:100650003F0D030028000020F0540020909200205D
:1006600080A80020D23D0020989200209C9200207B
:10067000309300203E930020A2920020A8920020F8
:10068000AC920020EC540020D8520020F50000204D
:100690009D4C2278002A41F00E839C4CD4F88C3279
:1006A00003F5C333A0339D42FFF47CAF984A94F81E
:1006B0009032C4F88C52D75CFA0701F1E585BB078C
:1006C00001F1A085780701F12C863A074FD5914BAF
:1006D000DFF86C82099310AA1146A3F1210241F8B8
:1006E000202D0020A3F124020E4603F8240C0291D1
:1006F00002231121517093703046D8F80410F9F795
:10070000ABFF3046D8F80810F9F7A6FFB8F812305A
:10071000814903EBC3039B00053381FB0321DB17F6
:10072000C3EBA101304689B2F9F7AEFFB8F8143037
:1007300003EB8303590089B23046F9F7A5FF774BE5
:10074000029E1B789B0743BFB8F80C1001F57A7125
:1007500089B24FF47A713046F9F796FF089B98F802
:100760000020591C089130461A701CF02FF96C4A71
:1007700094F890321178013393FBF1F201FB1233BC
:1007800084F890320EE7614C664BD4F8102119685A
:100790008A1A7C2A7FF65FAE94F81421DFF8A491C0
:1007A0009FED618AC4F81011013284F81421A9F177
:1007B000340A4FF0240840461CF09EF8BAF8103076
:1007C000F9EC016A07EE103AF8EEE66AB8EEC77A7D
:1007D00008F10108C6EE877A5FFA88F867EE887A32
:1007E000FDEEE77ACDED017ABDF904B05FFA8BF04A
:1007F0001CF058F8CBF307201CF054F8B8F1270F81
:10080000D9D130201CF078F8484ADFF83C91D2F872
:1008100000805FFA88F01CF045F8C8F307201CF050
:1008200041F8D9F800005E21F8F7C2FD94F81421D0
:1008300093072DD1D4F8101141F28832914201F280
:100840002C8714201CF058F8394A3349B2F9042097
:1008500081FB02314FEAE278C8EBA1080FFA88F871
:100860005FFA88F01CF01EF8C8F307201CF01AF895
:100870001C201CF041F800201CF014F800201CF093
:1008800011F85E21D9F80000F8F792FD94F81421D0
:1008900012F0070801F0A685282A7FF4DCAD214B71
:1008A0004FF0000817201F6884F814811CF024F80A
:1008B00040461BF0F7FF1F4B1F4CA3FB07239B0B6E
:1008C000A4FB03125209C2EB0212A3EB8203D8B2BB
:1008D0001BF0E8FF18201CF00FF8184BA3FB0723B0
:1008E0009B09A4FB03125209C2EB0212A3EB820381
:1008F000D8B21BF0D7FF40461BF0D4FFD9F8000058
:100900005E21F8F755FDA6E540550020901E002019
:10091000389300201C5500206766666661540020ED
:100920003D93002080A8002000007A448C540020D1
:100930009054002073B2E74589888888D34D6210AF
:1009400064540020CC540020F4540020DFF8B0811F
:10095000019341201BF034FB644FB8F90220DFF80B
:10096000A4B187FB0230D217C2EBA00080B21BF00B
:100970000BFBB8F9002087FB0230D217C2EBA000B6
:1009800080B21BF001FBB8F9042087FB0230D217BC
:10099000C2EBA00080B21BF0F7FA9BF80010D9F868
:1009A0000000F8F705FD94F84071019B17F001086D
:1009B00001F07D83DFF844A1DAF80020910640F1D0
:1009C00085804B4ADFF840811278920741F13A86E0
:1009D00098F80020042A8CBF03270227472002939F
:1009E0001BF0EEFAD8F804001BF09AFAD8F80800C9
:1009F0001BF096FAB8F812203E49D9F80000A1FB86
:100A00000232C2F3471211460192F8F7D1FC9BF86B
:100A10000000DAF80010019A029B424011F0140F16
:100A20008BF8002041F0A885B8F80C20642000FB6A
:100A300002F001931BF074FA98F80020D9F8000036
:100A400047EA8207FFB23946F8F7B2FC9BF800206C
:100A5000D9F80000574039468BF80070F8F7A8FC29
:100A600094F84071019B8FBBDFF8A08001934F2069
:100A70001BF0A6FAD8F800001BF052FAD8F80400D0
:100A80001BF04EFA38461BF04BFA0121D9F8000052
:100A9000F8F78EFC16499BF800200F78D9F8000073
:100AA00007F00107394682F001028BF80020F8F7C1
:100AB0007FFC9BF80020D9F80000574039468BF89E
:100AC0000070F8F775FC94F84071019B0A4AC4F86D
:100AD0003C317B1CDBB2A2FB0312D20802EB820288
:100AE000A3EB420384F840313AE500BF67666666CF
:100AF000615400201F85EB51CDCCCCCC5467002035
:100B000090540020DC52002064540020103F00204C
:100B100094F84A31002B41F03383E84B1B6803F013
:100B20000802002A48F603414AF60B404BF60F42F2
:100B300049F6074804BF0246884613F0040F4FF0F9
:100B4000190118BF90469B0684F84A1103D548F452
:100B5000804848F02008DA4B1A79C8F3090B002ABC
:100B600041F0FE855B79002B41F08C87994664202B
:100B70004FF0FF334FF0000ACDF82080CDF82480ED
:100B8000CDF828B0ADF82E90ADF830308DF83E009D
:100B9000ADF82CA0CDF832A0CDF836A0CDF83AA013
:100BA0000DF1200EBEE80F00DFF824C384F805A085
:100BB000ACE80F009EE80F00ACE807002CF8023B01
:100BC00061464FF001081B0C4FF0FE0E1F20C8229B
:100BD00001F81E3984F802E0A27184F80780E07001
:100BE00094F85A01207180F0F10383EA0313DAB21A
:100BF000130983F0E70343EA022383EAC2031BB22B
:100C000083EA0312D2B2C3F3072383EA121343EA3F
:100C1000022383EAC2031BB283F0C80282EA0212F3
:100C2000D2B2C3F3072383EA121343EA022383EA0F
:100C3000C2031BB283EA080E8EEA0E1E5FFA8EFE16
:100C4000C3F3072282EA1E1242EA0E2200EB0803D7
:100C500082EACE0E0CEB080084F85A31A4F800E0CA
:100C600011F8013B83EA0E0383EA0313DBB21A098E
:100C700082EA1E2242EA032282EAC3031BB21FFA5F
:100C800083FE8142A4F800E0EAD183F07C0383EA8A
:100C90000313DBB24FEA131C8CEA1E2C8CEA032CE4
:100CA0008CEAC30C0FFA8CFC1FFA8CFADFF8249242
:100CB000A4F800A05FFA8CFC4FEA1A2A84F828A056
:100CC00084F827C009F5C17B04F12208D9F8000097
:100CD000D9F80410D9F80820D9F80C30DE46AEE86F
:100CE0000F0009F11009C145F346EFD1D9F8000012
:100CF000CEF80000DFF8E08199F804308EF8043077
:100D000008F1270984F8A9C184F8AAA118F8011FDD
:100D10003868F8F74DFBC145F8D194F84B21002A0B
:100D200041F078816749684B08781B680A2184F88C
:100D30004B11002801F05182DFF8A0C10128BCF856
:100D40000010039141F296860228BCF8029001F04F
:100D50004B85BCF804100291032801F0A3860428F7
:100D6000BCF806B001F099860528BCF808E001F04F
:100D700090860628BCF80A8001F066860728BCF831
:100D80000C1001D0BCF80E2094F85A0108930646C6
:100D900086F0300383EA0313DBB24FEA131C4B489F
:100DA00004968CF07A0C4CEA032C008826718CEAAD
:100DB000C303DFF82CC1C0EB00208CFB00AC8444E3
:100DC000C0171BB2C0EB6C200646C3F3072C83EAA6
:100DD0000310039B8DF83560C0B24FF0000A63F337
:100DE0000F0A8CEA101303934FF0000C029B69F377
:100DF0001F4A6EF30F0C4FF000094FF0000E63F323
:100E00000F0961F30F0E039BCDF824A068F31F4C6C
:100E100062F31F4E4FF000086BF31F49CDF8289086
:100E2000CDF82CC0CDF830E08DF8348043EA0023B3
:100E30000DF1200983EAC00EB9E80F000FFA8EFE0B
:100E40008EF0C80A8AEA0A1ADFF884C084F805809E
:100E50005FFA8AFACEF3072EACE80F008EEA1A1E6C
:100E60004EEA0A2399E8030083EACA031BB283F01F
:100E7000230E4CF8040B8EEA0E1E5FFA8EFEC3F3AF
:100E8000072282EA1E12049B604642EA0E2203F108
:100E9000010882EACE0E20F814194FF02309FE2132
:100EA0001622C82384F85A81A4F800E084F8079039
:100EB0000CF1020CA170E27014E000BF5467002036
:100EC0007C540020D855002080A800203C920020AF
:100ED000981E0020921E002013200020B08F0020BA
:100EE00003082080A37110F8013B83EA0E0383EA14
:100EF0000313DBB21A0982EA1E2242EA032282EAC3
:100F0000C3031BB21FFA83FE6045A4F800E0EAD1D8
:100F100083F0F40383EA0313DBB21A0982EA1E2288
:100F200082EA032282EAC3031BB21FFA83FEDFF8C0
:100F30000C84A4F800E05FFA83FC4FEA1E2A84F8D0
:100F40001EC084F81FA0D8F80410D8F80820D8F8DC
:100F50000000D8F80C3008F5C17EAEE80F00D8F8D4
:100F60001000D8F81410D8F8182004F2A119AEE82F
:100F7000070004F2831884F8A1A184F8A0C118F82E
:100F8000011F3868F8F714FAC145F8D194F84E31CA
:100F9000002B41F0FA80DFF8B0A3DAF80030192214
:100FA000980684F84E2140F12083E34BDFF89C83C0
:100FB0001B78990741F1D08398F80030042B8CBF3F
:100FC0004FF003094FF00209FDF702FCB8F81430A6
:100FD000B8F80C20089003EB83035B00ADF83A30BF
:100FE0004FF47A70D8F804300A93B8F8121098F8D1
:100FF00000E0D8F808308DF83C9000FB02F24FF08A
:10100000000C4FF0FF3008AE8DF83DE0CDF824C065
:101010000C920B93ADF838100D90B146B9E80F0063
:10102000DFF82CE30296AEE80F0099E80F00AEE877
:1010300007007246182122F81C39E17194F85A1100
:1010400084F805C081F0780383EA0313D8B203095A
:1010500083F0F60343EA002383EAC0031BB283EA6A
:101060000310C0B2C3F3072383EA101343EA00233B
:1010700083EAC0031BB283F0C80080EA001C5FFA59
:101080008CFCC3F3072080EA1C1040EA0C2080EAA5
:10109000CC0000B280F0180383EA0313DBB2C0F384
:1010A000072080EA131040EA032080EAC30301F11D
:1010B00001091E204FF0FE0C4FF0C80BE0700EF13E
:1010C000020E217184F85A91238084F802C084F8BA
:1010D00006B0184612F8011B414081EA0111C9B25D
:1010E0000B0983EA102343EA012383EAC10109B211
:1010F00088B272452080EDD181F0180181EA01119A
:10110000C9B20A0982EA102383EA012383EAC103F0
:101110001BB29AB289492280DBB2120A039104926F
:101120001E4684F8272084F826308E4601F5C17BC0
:1011300004F12209DEF80000DEF80410DEF80820D1
:10114000DEF80C30DC46ACE80F000EF1100ECE4598
:10115000E346EFD1DEF80000CCF80000DFF8F491B0
:101160009DF8103084F8A86184F8A931CB461BF8AB
:10117000011F3868F8F71CF9714B5B45F7D1FDF793
:1011800027FBDAF80030B8F80C20D8F804A0D8F81B
:1011900008804FF47A7113F0140F01FB02F141F053
:1011A0005D828E4694F85AB108908BF06A00654BC8
:1011B000DFF8A4C1B3F90420CDF824A080EA001020
:1011C000C0B2030983F0D50343EA002383EAC003D6
:1011D0001BB283EA0310C0B2C3F3072383EA1013E0
:1011E00043EA002383EAC0031BB28CFB020CD21734
:1011F0004FF0000ACDF82880C2EBAC02DDF8088081
:10120000CDF830E083F0C80C0B91ADF83A20ADF882
:1012100034A0ADF836A0ADF838A08CEA0C1C5FFA0B
:101220008CFCC3F3072EB8E80F008EEA1C1E4EEAB2
:101230000C2E8EEACC0CDFF818E184F804B00FFA1B
:101240008CFCAEE80F008CF0210398E8070083EADD
:101250000313DBB2CCF3072C8CEA131C4CEA0328F3
:101260000BF1010C8EE8070088EAC30384F85AC129
:101270004FF0210B4FF0FE084FF01C0CC8220EF16E
:101280000C0E84F805A084F807B084F8028084F876
:1012900003C0AEF11C01A2711846238011F8012B86
:1012A000424082EA0212D2B2130983EA102343EACF
:1012B000022383EAC20212B290B271452080EDD1BE
:1012C00082F0680282EA0212D2B24FEA121B8BEA63
:1012D000102B8BEA022B8BEAC20B0FFA8BFB1FFA47
:1012E0008BF3DFF858E023805FFA8BFB1B0A1E4666
:1012F00084F8253084F824B00EF5C17A04F1220870
:10130000DEF80000DEF80410DEF80820DEF80C300D
:10131000D446ACE80F000EF1100EC645E246EFD100
:10132000BEF80030DFF83480ACF80030CA4684F8EC
:10133000A6B184F8A76113E061540020921E00203A
:10134000392000209054002054670020645400206D
:10135000981E002013200020676666663720002054
:101360001AF8011F3868F8F723F8D045F8D194F837
:101370005AA1E14AE14E84F804A08AF0EB0383EA23
:101380000313D9B20B0983F0C50343EA012383EAAF
:10139000C1031BB283EA0310C0B2C3F3072181EA81
:1013A000101141EA002181EAC0010CCA09B281F0A2
:1013B000C80E8EEA0E1E5FFA8EFE4FF0000C0892E9
:1013C000C1F30721029A0993CDF828C081EA1E13C0
:1013D00043EA0E2307CA83EACE031BB283F0310E21
:1013E00086E807008EEA0E1E5FFA8EFEC3F307231F
:1013F00083EA1E1343EA0E2383EACE0394F808E03F
:10140000607AA27AE17A84F805C01BB28EEA030EF4
:101410008EEA0E1E5FFA8EFEC3F3072383EA1E13C5
:1014200043EA0E2383EACE031BB2584080EA001041
:10143000C0B2C3F3072383EA101343EA002383EA0D
:10144000C0031BB25A4082EA0210C0B2C3F30722A3
:1014500082EA101242EA002282EAC00212B251402D
:1014600081EA0111C9B2C2F3072383EA111343EAE7
:10147000012383EAC10394F80CC094F80DE0A07B2B
:10148000E17B227C94F811801BB28CEA030C8CEA7D
:101490000C1C5FFA8CFCC3F3072383EA1C1343EA9A
:1014A0000C2383EACC031BB28EEA030E8EEA0E1ED7
:1014B0005FFA8EFEC3F3072383EA1E1343EA0E236B
:1014C00083EACE031BB2584080EA0010C0B2C3F3D7
:1014D000072383EA101343EA002383EAC0031BB205
:1014E000594081EA0111C9B2C3F3072383EA1113FA
:1014F00043EA012383EAC1031BB25A4082EA021283
:10150000D2B2C3F3072383EA121343EA022383EA26
:10151000C2031BB288EA030888EA08185FFA88F851
:10152000C3F3072383EA181343EA082383EAC803B3
:10153000A17CE27C1BB2594081EA0111C9B2C3F31C
:10154000072383EA111343EA012383EAC1031BB291
:101550005A4082EA0212D2B2C3F3072383EA12137B
:1015600043EA022383EAC2031BB283F0270E8EEA0A
:101570000E12D2B2C3F3072E8EEA121E4EEA022ECC
:101580008EEAC20E0AF101030FFA8EFE1FFA8EF2E6
:101590004FF0310AFE200C2184F85A31C8234FEA5B
:1015A000122C06F5BE785FFA8EFE228084F807A022
:1015B000A070E170A371039E84F814E084F815C054
:1015C0007168B268F3683068B6F810A0A8E80F0038
:1015D00028F803AB84F897C184F896E119F8011F45
:1015E0003868F7F7E5FEC845F8D194F852C1BCF168
:1015F000000F40F05685424B94F85A91B3F9001011
:10160000B3F90220B3F904309FED3E6A84F805C0B7
:1016100007EE103A3C4B1B68089389F06A0383EA93
:10162000031306EE901AD9B20B0983F0D50343EAEF
:10163000012383EAC1031BB283EA03115242C9B2F8
:1016400007EE902AC3F3072383EA111343EA012329
:10165000F8EEE77AF8EEE66AB8EEC77A83EAC103F5
:101660001BB267EE867A66EE866A27EE067A00205F
:1016700083F0C808CDED0A7ACDED096A8DED0B7ABD
:101680000C900D900E9088EA081E0DF1200A5FFA6A
:101690008EFEC3F30728BAE80F0088EA1E1848EA4E
:1016A0000E2888EACE08DFF854E00FFA88F8AEE892
:1016B0000F0088F01E0C9AE807008CEA0C1C5FFAF9
:1016C0008CFCC8F3072383EA1C1343EA0C238EE83F
:1016D000070083EACC0CC8214FF0050A4FF01E0822
:1016E000FE231C2009F10102A17184F852A184F8A3
:1016F0000780A370E07009E0103F0020981E0020D2
:101700009054002088C3E43A80A80020AEF1100174
:1017100084F804900EF10C0EA4F800C084F85A214D
:1017200011F8013B83EA0C0383EA0313DBB21A09C5
:1017300082EA1C2242EA032282EAC3031BB21FFA96
:1017400083FC7145A4F800C0EAD183F0270383EA43
:101750000313DBB21A0982EA1C2C8CEA032C8CEAF4
:10176000C30C0FFA8CFC1FFA8CFADFF81094A4F863
:1017700000A05FFA8CFC4FEA1A2A84F825A084F8AE
:1017800024C009F5C17B04F12208D9F80000D9F87A
:101790000410D9F80820D9F80C30DE46AEE80F0066
:1017A00009F11009C145F346EFD1DFF8E483B9F838
:1017B0000030AEF8003008F1240984F8A6C184F89E
:1017C000A7A118F8011F3868F7F7F2FDC145F8D155
:1017D00094F853A1BAF1000F40F05E84E04B1B680F
:1017E000052284F853219A0640F10185DD4ADFED98
:1017F000DE7A518A07EE101AB8EEC77A13F0140F8A
:1018000027EE277A01F0E380D84BDFEDD76AD3EDDE
:10181000007AF8EEE77A67EEA67A94F85A91D44BFC
:10182000D44AB3F90410B2F90620DFF868E3D248CD
:101830008DED097A89F0220383EA03135FFA83FCB2
:101840004FEA1C1383F0590343EA0C2383EACC03C9
:10185000B2F5FA6F1BB2A8BF4FF4FA6283EA031C19
:101860005FFA8CFCB2F57A7FC3F3072383EA1C137B
:10187000B8BF4FF47A724FF0640843EA0C23A2F524
:101880007A7208FB02F283EACC0C8EFB026E80FBBC
:1018900001600FFA8CFCC917D217C2EBAE12C1EB74
:1018A000A0034FF0000B08A98CF0C80ECDED0A7A0A
:1018B000ADF83220ADF83030CDF820B0CDF82CB0F6
:1018C00088468EEA0E1E5FFA8EFE0291CCF3072C3C
:1018D000B8E80F008CEA1E1C4CEA0E2C8CEACE0EE7
:1018E000DFF8B4C2D8F8008084F80490ACE80F00A8
:1018F0000FFA8EFE8EF04A0383EA0313DBB2CEF3B7
:10190000072181EA1311624641EA032109F1010925
:1019100081EAC303142042F810894FF0FE0E4FF005
:101920004A08002184F85A914FF0C809E0702380DA
:101930000CF1040C84F8078084F802E0617184F8EB
:101940000690184612F8011B414081EA0111C9B204
:101950000B0983EA102343EA012383EAC10109B298
:1019600088B262452080EDD181F0140181EA011135
:10197000C9B24FEA111E8EEA102E8EEA012E8EEAAF
:10198000C10E7E4B0FFA8EFE1FFA8EFC1E464FEAEA
:101990001C2B5FFA8EFE84F81DB084F81CE0596899
:1019A0009A683068DB68A4F800C006F5C17CACE832
:1019B0000F0030697169B6F818900396ACE803001F
:1019C00004F28318ACF8009084F89FB1C14684F803
:1019D0009EE104F29F1B19F8011F3868F7F7E8FC35
:1019E000CB45F8D1664B674A1B781278013B12F061
:1019F0000100DBB214BFC0214021172B03D8624A7B
:101A0000134493F808A0614B1A8896071ABF002365
:101A100041F01001012312F4027F18BF022312F0DB
:101A2000100F18BF062312F0200F18BF1023002834
:101A300040F029864FF0030994F85AE108938EF09C
:101A4000460383EA0313DAB2130983F0920343EAED
:101A5000022383EAC2031BB283EA0310C0B2C3F3BA
:101A6000072282EA101242EA002282EAC00212B27F
:101A700082F0C80C8CEA0C1C5FFA8CFCC2F30722C3
:101A800082EA1C1200238DF82790032042EA0C29D9
:101A9000029A8DF824A08DF825308DF826108DF847
:101AA000280007CA89EACC0C0FFA8CFCDFF8E89012
:101AB000E3718CEA0C1AA9E803005FFA8AFACCF306
:101AC000072C8CEA1A1C4CEA0A2181EACA0A94F80B
:101AD00008C089F800200FFA8AFA8CEA0A0C8CEA0E
:101AE0000C1C5FFA8CFCCAF3072282EA1C1242EA41
:101AF0000C22607AA17A94F80BA0637182EACC027E
:101B000012B2504080EA001C5FFA8CFCC2F307203E
:101B100080EA1C1040EA0C2080EACC0000B2414070
:101B200081EA0111C9B2C0F3072282EA111242EA26
:101B3000012282EAC10212B28AEA020A8AEA0A1A77
:101B40005FFA8AFAC2F3072282EA1A1242EA0A22EA
:101B500094F80CC0607BA17B84F804E01EE000BF19
:101B600054670020645400200AD7233C8854002086
:101B700090540020B08F002067666666921E002099
:101B800090390020C4510020C0CA0308E05400204E
:101B900013200020D34D6210981E002082EACA0252
:101BA00012B28CEA020C8CEA0C1C5FFA8CFCC2F3B9
:101BB000072282EA1C1242EA0C2282EACC0212B20A
:101BC000504080EA0010C0B2C2F3072282EA10122D
:101BD00042EA002282EAC00212B2514081EA0111B7
:101BE000C9B2C2F3072282EA111242EA012282EA52
:101BF000C102E17B94F810A013B281EA030282EAE9
:101C00000212D2B2C3F3072383EA121343EA022378
:101C100083EAC2031BB28AEA030282EA0212D2B248
:101C2000C3F3072383EA121343EA022383EAC203BE
:101C30001BB283F0320282EA0212D2B2C3F307234C
:101C400083EA121343EA022383EAC2031BB29AB265
:101C50004FF0FE0C0920C8210EF1010EDBB284F812
:101C600002C04FEA122CE070A17184F85AE1228080
:101C700084F812C06374039E30687168B268B6F865
:101C80000CB009F5BA7EAEE8070009F5C2798EF806
:101C900002A0AEF800B084F894C184F8933118F82B
:101CA000011F3868F7F784FBC145F8D1019BC4F8E0
:101CB0004431FEF773BCDA4BDA491868F7F740FB9A
:101CC00000232370FEF7E9BC94F89832D64AC4F892
:101CD000945202EB8302126A42B310AD04F29F23C6
:101CE000D24E45F8203D002104F2B1233180099302
:101CF00080211523A52784F89E32284684F89D125A
:101D000084F89C72904728463188F8F7E3FC089DD8
:101D1000C74804F527716D1A152DA8BF15252A4649
:101D200028F02AFAC34A94F898321570C24A01334F
:101D300082FB0312A2EBE37202EB42029B1A84F8CD
:101D40009832FEF73BBCDFF828E3BC4ABC4BD4F822
:101D50002011DEF800001B8892F80BC0B94A401A27
:101D60004FF47A71DFB201FB0CF11B0A97771775FC
:101D700088424FF00007D37753759770177180F042
:101D80000C82B14BB14E1B68B149DFF8E89208688C
:101D90008968DFF8E4E2DFF8E482DEF800E086FB41
:101DA000036CDB17C3EB6C1303F5FA739BB29376EA
:101DB0001B0AD37689FB003AC01789FB0139CB1780
:101DC000C0EBAA0111770912DFF8B4C251779F491D
:101DD0009CF800C0C3EBA9030EF5EA4081FB0E1985
:101DE00082F820304FEAEE711B12C1EB69113030DE
:101DF00082F82130974B98F8009083F81A900012DF
:101E000078310EF1300E1CF0020F82F8230082F8B8
:101E1000241082F822E000F0BD81D8F804C08E4979
:101E2000D8F808A0DFF85CB28C4A81FB0C604FEA5E
:101E3000EC7E81FB0A61CEEBA05E4FEAEA70C0EB5C
:101E4000A1510BFB0EC00BFB01AB0BEB4B0B4FEA95
:101E50004B0600EB40000196400082FB007B01EB4B
:101E6000810182FB0672019E92140EEB8E0E01EB35
:101E700081014FEAAB4B04920EEB8E07B8F81220AB
:101E800005914FEAE67EC117B8F80C80744E0397AF
:101E90004FEADC7C83F809C0ABEB010C06FB1C01AC
:101EA00008F5FA78049E03981FFA88F70297A6EBC4
:101EB0000E086B4F019EDFF8D0E1B9F1050F4FFA24
:101EC0008CF909EB8009404607FB1868059EDFF88E
:101ED000BCC140B200EB860002EBC2025B4E4FEA8F
:101EE00082024FEADA7A8CFB02BC83F80EA086FBF2
:101EF000017A86FB08B74FEAE27B9DF808205A7505
:101F0000CBEBAC120192029ABEF80060DFF880E1E0
:101F10004FEAE8784FEAE1711FFA89F980B2C8EB1D
:101F20006717C1EB6A114FEA1228019A83F80A90E9
:101F30004FEA102B4FEA192C4FEA212A4FEA2729A2
:101F400083F810B0BEF800E083F80BC0D873C2F37A
:101F5000072C4FEA162034BF4FF0320B4FF0330BF3
:101F6000197383F80DA05F7483F8129083F81680BC
:101F70009DF80420DA7183F808C0DE74187583F8C0
:101F80001BB083F81CE0C4F81C51FEF770BA354F43
:101F9000386803685B69984700283EF4EDAA386802
:101FA000036801219B6998470222002388F80020DA
:101FB0002370FEF7E1BA94F8381194F83931D8F863
:101FC00000004A1C013384F8382184F83931F7F7CE
:101FD000EFF9FEF7B0BAFCF7FBFB234B1A6840F6AB
:101FE000B833801A984200F2EE80204F3B793A2BAA
:101FF00000F0CB8200232370FEF7BEBAC4F82C3168
:1020000084F82431DFF88C801AF032FC94F83031F7
:10201000FEF776BA013A84F84B21FEF7B7BF00BF4E
:10202000349300201C550020C0CA03087E520020B3
:102030004C3B0020613B0020565555557052002006
:1020400080520020B0920020885400201F85EB5160
:1020500084520020DC9200206BCA5F6B83DE1B433E
:1020600040420F00343E0020D83D0020C03D0020FB
:1020700080A80020676666668C54002064540020A7
:1020800061540020806967FF183F0020D34D621023
:102090001A3F0020EC5400200AF1FF3A84F853A1C3
:1020A00004E60CF1FF3C84F852C1FFF791BBB94A3A
:1020B0001288D70515D4D00600F1D882910600F118
:1020C0009A83570600F18A84100700F18B84D107A8
:1020D00000F1AE8412F0020F0CBF4FF004084FF075
:1020E0000C08AD49AD4A0F78D27807F001070AB164
:1020F00047F002075320019319F062FFA84A1288A3
:1021000002EB820202EB8202900080B219F03CFFE7
:10211000002019F039FFA34AA3491288D9F800001A
:10212000C2EBC212520081FB02311144D217C2EB42
:1021300061225FFA82FA5146F7F73AF99BF80020DC
:10214000D9F800008AEA020248EA070700218BF862
:102150000020F7F72DF93946D9F80000F7F728F9EC
:102160009BF80020D9F800007A40D2B211468BF8D3
:102170000020F7F71DF994F84071019BFEF773BC3E
:10218000013B84F84A31FEF7C8BD013B84F84E316B
:10219000FFF72BBA2D22DA76F5E6844BDEF8001035
:1021A0001B78C4F82011013B012B3FF6EAAD10214A
:1021B000022391701371E4E51AF04AFB7C4B012273
:1021C0001A70FEF76FB97B4AB2F842310021013331
:1021D000A2F842312170FEF7CFB90146804686460B
:1021E00083460290814603900246FEF7CDBD9FEDE7
:1021F000727A13F0140F08BFF0EE477A7FF404AB45
:10220000FFF70BBB6D4B664909930DF14008A3F135
:10221000210048F8200D4FF0080E4FF000090A2069
:1022200003F822EC03F8230C03F8249C40460988A9
:10223000F8F72AFA624B63491B6881FB0321DB171D
:10224000C3EBA101404689B2F8F71EFA5E4BB3F822
:1022500006A00BF09FFA089B5A1C089283F8009086
:10226000089B4FEA1A22591C08911A70089B5A1CA5
:10227000089283F800A0089B5A1C089218704046E8
:102280001AF0A4FBFEF71EBADFF850919FED4F8ABB
:10229000B9F90230494A099207EE903AF8EEE77A26
:1022A0000DF1400867EE887AA2F12403FDEEE77A8B
:1022B000A2F12101002048F8201D02F8240C082278
:1022C000CDED017A5A701E229A70BDF80410404676
:1022D000F8F7DAF9B9F9003007EE903AF8EEE77A54
:1022E000404667EE887AFDEEE77ACDED017ABDF8DB
:1022F0000410F8F7C9F9B9F9043007EE903AF8EE8E
:10230000E77A404667EE887AFDEEE77ACDED017A0E
:10231000BDF80410F8F7B8F940461AF057FBFEF77D
:10232000CEB92B4A254B12680993A3F1240800214A
:1023300003F8241C2123D10088F8023040F10082E8
:1023400024490326134B1B885A0500F1F681D80750
:1023500000F1F58203F002031F4A002B1CBF032685
:102360001146DFF87C903246484627F005FF06EB21
:10237000090310A80133A9F1020140F8203D002211
:102380005B1A06F8092088F801301AF01FFBFEF7E7
:102390009CB900BFE0540020C451002048920020A6
:1023A000805200203C9200200308208042920020AE
:1023B00028000020901E0020000000001C55002076
:1023C00084520020676666667C54002058A08B41CA
:1023D000DC37002030F9030840F90308905400204E
:1023E000FB54002002201AF087FAFF2019F09CFC11
:1023F0000278FF2A00F0E98290F901004FEAE078C4
:102400005FFA88F8C0B21AF04DFA40461AF04AFA5C
:1024100003201AF071FAFF2019F086FC0278FF2AD7
:1024200000F0CF82B0F908805FFA88F0C8F307287F
:10243000DFF898A31AF036FA40461AF033FA9AF801
:102440000420002A40F0E781D14A1268900640F14A
:102450001081DFF87CA3DFF87C839AF800209107D5
:1024600000F170824FF0000B01201AF045FA384657
:102470001AF018FA58461AF015FA09201AF03CFA20
:1024800000201AF00FFA00201AF00CFAB8F8161013
:1024900098F80030B1F5967F0AD994F8142102F02B
:1024A0000F02072A04D842F20F738B4228BF0B4653
:1024B000DFF824B3019305201AF01EFA9BF80820D8
:1024C000019B002A00F0A482203B07EE903A9FED8A
:1024D000B17AF8EEE77AF6EE006A67EE877ABEEE3A
:1024E000007AF5EEC07AF1EE10FA58BFB0EE667AD7
:1024F00077EE877AFDEEE77ACDED017ABDF904300B
:102500000193D8B21AF0CEF9019BC3F307201AF059
:10251000C9F99AF80020002306930793930700F166
:102520006D8194F81831012B00F06881BBF90030FF
:10253000DFED996A07EE103ABBF9023007EE903AE8
:10254000B8EEC77AF8EEE77A27EE267A67EEA67A33
:10255000BDEEC77AFDEEE77A08A88DED087ACDEDDD
:10256000097A1AF0DBF95E21D9F80000F6F720FFAE
:1025700094F81421FEF790B9884A1068FEF759BA0A
:10258000C4F828511F70FDF78DBFBB78DBB103F194
:10259000FF3C5FFA8CFC0CF1010CBC44BE460022EF
:1025A0001EF8013B534083EA0313DBB2120AD90041
:1025B00042EA0322F44581EA131382EA0302EFD1CF
:1025C000002A7FF417AD764BDFF810E21968734BE1
:1025D000D1F830C01B68734ADFF8EC81CEF8383090
:1025E000714BB8F80080CEF86800B3F8423110683B
:1025F0009268CEF81880CEF82800CEF84820CEF8A1
:102600005830BCF1000F00F01782DCF80430886C01
:1026100083423BBFCA681B1A1B1A9B18002B7DF410
:10262000A4AF0B68DFF8B8819B6908460221984780
:102630000423F87888F8003012F05AFC0323237042
:10264000FDF795BF0127FEF7C9B90221D8F80000B0
:10265000F6F796FE94F83031FDF752BF4F4B1B68EA
:1026600003EB83034FEA430EFEF79CBD4FF03408A3
:1026700037E54E4B93E8030008AB83E803001846A8
:102680001AF04CF96FE74A4AD278002A0CBF4FF093
:1026900004094FF00509FFF7CFB9DFF800B1DFF803
:1026A00044A110201AF028F9DBF800208AFB023838
:1026B000D217C2EB68185FFA88F01AF0F3F8C8F383
:1026C00007201AF0EFF821201AF016F9DBF80010B5
:1026D0008AFB013ACA17C2EB6A12642000FB12128D
:1026E000002AD8BF524212B2D0B21AF0DBF8002052
:1026F0001AF0D8F8FEF7A5B80122D8F800001A7031
:10270000F6F74AFE0746D8F80000F6F745FE7F06C2
:102710007DF4C8AE8A2800F069818E287DF4C2AEAF
:1027200094F82431002B7DF4DAAE224BC4F82C311E
:102730002D2384F83031FDF7BCBE03261E4910E678
:102740001E4B1F4A1B681F4903F48003002B16BF52
:10275000114604260326F5E54FF00109FEF734BCC7
:1027600019495A790B8803EB830303EB83034FEA80
:1027700083091FFA89F9002A00F09A81094B1B6826
:102780001BB202930BF006F8029B40B2FEF7F2B9BF
:1027900054670020E4380E3F0050C347885400209F
:1027A000343E002084520020901E0020C0CA03083E
:1027B00048920020B092002034F903087083002072
:1027C00030F9030828F90308805200207C540020C7
:1027D00061540020645400207052002084000020C6
:1027E000F50000201F85EB51114690469646934612
:1027F0000292FEF7C9BA4FF0240872E40121D8F81A
:102800000420D8F8083084F8181106A80692079317
:102810001AF084F8A7E6DFF8C0B29BF80020002A7F
:102820003FF412AEA449B4F81681088802914FEA29
:1028300008184FF0640E1FFA88F80EFB00204FEACC
:10284000420EB0FBFEF048EA00281FFA88F8C0F3F9
:10285000032048EA0008062001921AF04DF85FFABA
:1028600088F01AF01FF84FEA18201AF01BF8B4F895
:102870001601019A914B0299013080B290FBF2FC53
:1028800002FB1C02587AB1F80080A4F81621012836
:1028900000F0E4805A7B6E2303FB08F8152198FBB7
:1028A000F1F8002A40F0D3803A201AF025F81FFAF8
:1028B00088F84FF0640BB8FBFBF291B2C8B20292F9
:1028C000019119F0EFFF0199080A19F0EBFF3B2085
:1028D0001AF012F8029A0BFB128080B20A2205301D
:1028E00090FBF2F0C0B219F0DDFF002019F0DAFF22
:1028F000DFF8E0B1282019F0FFFF4FF00A08DBF8FD
:10290000002092FBF8F85FFA88F019F0CBFFC8F3CB
:10291000072019F0C7FF042019F0EEFFBAF80620CF
:10292000002A7DD1DBF8082082F310085FFA88F0D6
:1029300019F0B8FFC8F3072019F0B4FF84E5604927
:1029400004260EE5112019F0D7FFB8F812205D49D2
:102950004FF4F36B0BFB02F281FB0231D217C2EB97
:102960006132D0B2019219F09DFF019AC2F30720A3
:1029700019F098FF192019F0BFFFB8F8122052493A
:102980000BFB02F281FB0230D217C2EB601281FB1B
:102990000230D117C1EB6011642000FB1120C0B2DE
:1029A00019F080FF002019F07DFF9AF80020B8F898
:1029B0000CB092077FF556AD5FFA8BF74FEA1B2BF1
:1029C00052E54FF00008404632E540461BE593894A
:1029D00007EE903AF8EE677AFEF71FBF4FF0100847
:1029E000FFF77FBB4FF02008FFF77BBB374B1B681F
:1029F00098067DF557AD94F82431002B7DF46FAD2A
:102A0000334BC4F82C312D2384F83031FDF751BD00
:102A1000D8B219F047FF019B180A19F043FF78E577
:102A20000AF0B8FE19F03EFF002019F03BFF0BE55D
:102A30004FF00808FFF755BBCA690B6A9A423CBFC2
:102A4000C8681218D31AE9E51146FEF79DB91FFAB6
:102A500088F89BF8002098FBF2F825E7392019F058
:102A60004BFF5FFA88F019F01DFF4FEA182019F0AC
:102A700019FF3DE7114690469646934602929146CD
:102A8000FEF782B9134B9146B3F900306420FEF78C
:102A900071B811469046FEF777B9114690469646B2
:102AA000FEF772B91146904696469346FEF76CB90A
:102AB0004FF0FF3364E600BF8052002070520020C8
:102AC00038F9030889B5F8141F85EB5154670020C5
:102AD000DC92002084520020C75200202DE9F04FE4
:102AE00099499A4C0A7897B000F59C4320330B9093
:102AF0002360002A00F0BC84954B1B689842954BDC
:102B0000079340F29280D3F80080934B934804934C
:102B1000013A08F48053DFF880B203900A700A93F8
:102B2000002B40F09080049B5B7D002B40F067837E
:102B300018F4807F0BD00B9A894BDFF860929A4291
:102B400099F8022000F2F687002A40F0F787854BBB
:102B5000854C069318F4805640F07284049BBBF9B0
:102B600006505B8B9D42B4BF002501257F4F3B681B
:102B700013F0805374D0069A127812F0010276D0C6
:102B800004987B49808C91ED037A07EE900AF8EE69
:102B9000E77AB4EEE77AF1EE10FA80F2CA86002DF9
:102BA0006BD1039991F88C10002966D17148724954
:102BB000006890F830004FF0000EC1F800E0C1F856
:102BC00004E0C1F808E06D49002857D10870002AD8
:102BD00058D018F0100F55D0694A1278D00651D449
:102BE000002E4FD1002B4DD118F4800F4AD194F80C
:102BF00000C0BCF1000F01F02286624B9B78002DD3
:102C000041F072863BB1604A604B12681B689B1AA8
:102C1000002BC1F25386102015F08EF9039A94F818
:102C200000C0012382F88D302EE0D3F800804A4B9B
:102C30004A4A049308F480530392DFF85CB10A9384
:102C4000002B3FF470AF00214848F8F7E5F8002862
:102C50007FF469AF07F048FC079BD3F8008062E778
:102C600018F4800F87D1069A127802F001020398B7
:102C7000002180F88C10002D98D040490120087068
:102C8000002AA6D194F800C0049ABBF900E0508B4A
:102C9000918BBBF902208645CCBF8026002646F0EA
:102CA00040038E45A8BF33469B0843F0800682420E
:102CB000C8BF334643F040068A42B4BF32461A4684
:102CC0009208BBF904E0BBF9066042F08003864538
:102CD000C8BF1A4642F040038E45A8BF13469B0862
:102CE00043F080028642D4BF18461046039B40F052
:102CF000400293F88E308E42ACBF014611468B42A3
:102D000000F08C840398002380F88E1080F88F30B8
:102D1000BCF1000F00F06A85079B1D4A1B680592F5
:102D200003F00403002B40F053840DF1500A194CBA
:102D30000023CAF8043004F15008149340F6330914
:102D4000192640F283352EE0E43D00208C3C002023
:102D5000E03D002070830020B07200204821002058
:102D6000404B4C00C45100207C1C0020DC3700206C
:102D7000C8520020E4540020803600209C2300200C
:102D8000615400208C24002080A80020F023002023
:102D90005467002094390020B08F00204892002012
:102DA0000434444520D0A278E3789A4216FB0251BD
:102DB000F6D26278043216FB03533BF912204A45DF
:102DC000A8BF4A46B2F5617FB8BF4FF46172914225
:102DD000E6DA9A42E4DC21782329E1D8504604342B
:102DE000F8F70AF84445DED1B14B9AE803001D78A4
:102DF00087E80300002D00F063820121AD48F8F759
:102E00000BF8002840F00981079B1B68DC0500F1E6
:102E1000FF80A94C23881DB225F00105AFB2BB424B
:102E2000278000F02484A54D02260F204FF01409BE
:102E30004FF0FF082E7085F8019085F8028015F09C
:102E40007BF831469B482788F7F7E6FF002800F01B
:102E5000FD8027F001039BB2BB42238008D00F20E6
:102E60002E7085F8019085F8028015F065F82788A6
:102E7000BA0740F17685924B04931978DFF85CA28B
:102E8000BB0708BF81F00201DAF80400C1F340017A
:102E9000F6F7A0FE059B1B6813F00A0F1DD0052155
:102EA0008448F7F7B9FF002800F08B8425886F0766
:102EB00040F111877F480621F7F7AEFF002800F0A8
:102EC0006D846E0640F1FF8607217A48F7F7A4FF6C
:102ED000002840F0B681059B1B689D0600F1C1816A
:102EE000258874480C21F7F797FF002800F0C1806F
:102EF00045F48073AB42238009D0704B0225142126
:102F0000FF220F201D7059709A7015F015F86D4B47
:102F10001B78082B00F0B9800E2B00F0B680079BC1
:102F20001B685E0542D5684B1B79002B58D01421D5
:102F30006048F7F771FF002856D11FF0D3FD01203C
:102F400014F04CFF90B3DFF8988100254FF0CC09C6
:102F500002E0DDB2022D29D809FB05F76B1C58F8F9
:102F60000760002EF5D1C378584A90F9020052F854
:102F700023300196032200920121324613F0F6FE1F
:102F8000034605EB450000EB0010039353B13146B7
:102F900008EB8000CC2229F070FB039B48F8073037
:102FA0000135EDB21BF038FF0028D3D1069B1B780A
:102FB000DD0740F197804649464A01230B701370A4
:102FC000049BDAF80000197801F00101F6F702FE1F
:102FD000059B1B685A0700F1F58017B0BDE8F08F1C
:102FE000069B1B78D807A8D53C201EF01DFC0028A6
:102FF000DCD00BF0DDFB3C201EF0B8FB0028D5D068
:103000000BF0D6FB3C201EF0B1FB0028F1D1CDE740
:10301000314BDB78002B3FF4FCAE059B1B68980717
:103020007FF5F7AE244C2788F9070FD447F001034A
:103030009F4223800AD0214B1421FF2202250F201A
:103040001D7059709A7014F077FF278827F00203DB
:103050009BB2BB4223803FF40EAF184B1421FF22DA
:1030600002250F201D7059709A7014F065FF278893
:1030700001E725F480739BB2AB4223807FF43DAF20
:10308000104B1B78082B7FF447AF228822F04003B7
:103090009BB29A4223803FF442AF084B0225142191
:1030A000FF220F201D7059709A7014F045FF36E70B
:1030B000D8410020DC370020E054002008360020F2
:1030C00048A800209039002070520020A4F2030884
:1030D000C551002028240020489200204CA8002040
:1030E000E88B0020B14B93F80090B9F1000F5FD14D
:1030F000DFF84083AE4F18F8030C3E784146A8F144
:10310000030524F03DFF002800F0BB82002E40F0B4
:103110000D8305F10801687924F032FF002841F0A1
:103120002982A449A87A24F02BFF002800F0BC8251
:10313000022E41F01782A049E87B24F021FF0028ED
:1031400041F014829D49287D24F01AFF002800F0E8
:10315000BC82042E41F0FA819949687E24F010FF68
:10316000002841F0F7819749A87F24F009FF002843
:1031700000F0BC82062E41F0F181934995F82300BE
:1031800024F0FEFE002840F02C87904995F8280096
:1031900024F0F6FE002800F0BC82082E40F00B87D9
:1031A0008B4995F82D0024F0EBFE002840F0BC82FE
:1031B000884B01221A7025F068F9059B1B685A0795
:1031C0007FF50BAF032024F005FF002800F0FC85FD
:1031D000238813F008047FF400AF082014F0F0FFF8
:1031E0007D487E4D7E497F4A7F4BBBF80660006874
:1031F0002E80086014601C6017B0BDE8F08F049A40
:10320000013BD27D3BF913301AB1C3F53B63083360
:103210001BB2A3F57A73B3F57A7FA8BF4FF47A7324
:1032200023EAE37307EE903A9FED707A704AF8EE66
:10323000E77A67EE877AFCEEE77A17EE903A13802A
:1032400076E46C4B6C4AB3F904306C4982FB0302A0
:10325000DB17C3EBA202059B0A801B689D067FF566
:103260003FAE674B1B78980704D5664E3378042B26
:1032700000F24A86258815F0300F3FF432AE102058
:1032800014F086FF202014F083FF5F4B2588002276
:103290001A705E495E485F4F5F4E00220A605F49C8
:1032A0003A60002332604260826103608360436160
:1032B000C3610B604A608B604B618A61CB6110E631
:1032C000DFF87481564EDDF80C9008F15A0401279E
:1032D000414618F8010C24F053FEF8B198F80400A8
:1032E00098F8023098F803E000EB400109EB810107
:1032F000013BD1F89C2003EB4303334493420DD0B0
:1033000099F8C82081F898E007FA00F022EA000056
:10331000C1F89C30C1F8A05089F8C80008F106082F
:103320004445D5D13F4A404BD2F8008093F80090F5
:103330003E493F4C0968DFF804A108914F46C14659
:10334000DDF80C80002563684BB31E783EB3A1689E
:10335000A9EB010100290ADB98F8C8100120A84058
:1033600021EA000109F5FA7088F8C810A060B7B129
:10337000217858780431C9B2002840F0E082049ADC
:103380003BF91110108B00F1C80E714540F37A859E
:1033900098F8C8109B782941C90740F1FC85013590
:1033A000042D04F10C04CED127E500BFC551002047
:1033B00029000020E3350020E8350020ED3500200D
:1033C000F2350020F7350020FC35002001360020C2
:1033D00006360020282400208854002008240020DD
:1033E000142400200C24002004240020AAF1823F91
:1033F0003C9200209054002067666666FE23002001
:103400006154002064540020CE3E0020C43F0020C0
:10341000743F002070230020842400209C3F002063
:10342000ECCA030880A8002009920020E85400207C
:10343000E0210020D9350020F1340020C997002078
:103440001D21BC48F7F7E8FC00287FF487ABBA4A97
:10345000049BD2881B8BBBF90650991A8D4240F30E
:103460003E8513449D42B4BF00250125FFF77EBB76
:10347000B24B03931E78B24B0493DFF8C8A2002E20
:1034800000F02B82C6B1DFF80483DFF804B3AD4F40
:10349000454600244FF47A79072C3846E1B2DAF831
:1034A000043041F35681984700B20134A6422BF80C
:1034B000020F05F10405EFD1A34B0793D3F8008069
:1034C000A24E0B9BA6FB033642F2010318EA03034C
:1034D0004FEA9616099300F0FC819D489D4A9E4B49
:1034E00000789E49069012781A70069B08702BB1DE
:1034F000994B93F8009089F001030693984A994BF1
:1035000012780C920C9A039804999AF800E00478C7
:103510000398CDF840E0A3FB02935B08B1F826E0E6
:10352000B1F828C091F82270098B139103EB430383
:1035300090F829101191D31ADBB204370F22CDF87D
:1035400038C00D93FFB208F48053CDF848A0864DE3
:10355000DFF840B2DFF840C2DDF844A0CDF814E057
:10356000A146DDF840E080F828200F920A93002160
:103570000897CDF8408034B9089B734599BF9946A8
:103580004C46F1467446A14280F25E82069B002BB7
:1035900000F02982754B059833F911201FFA82F843
:1035A00080454FEA410303D30E98804540F2EE81F7
:1035B0005CF82120964280F020823BF90320099894
:1035C000002840F0EB812BF8032001310635D2E7CB
:1035D000039B93F8933053B1069B1B78D80706D50D
:1035E000049BBBF906205B8B9A4200F3C584112132
:1035F0005048F7F711FC002800F05881039991F822
:1036000096302BB991F8913013B93223A1F8943048
:10361000039A012382F89630FFF787BB039890F84E
:103620008F80B8F1F90F00F27C8108F101085FFA90
:1036300088F880F88F8080F88E10BCF1000F00F0C1
:10364000D680B8F1140F7FF467AB5F2940F0618139
:10365000069D2B7813F0010300F0168706F044FF57
:103660002B7803F00103002B7FF456ABD0E002214E
:103670003048F7F7D1FB00283FF4E8AC2580FFF78E
:10368000F7BB08F10501687924F07AFC00283FF4C3
:1036900048AD012E40F06E8705F10D01A87A24F0A7
:1036A0006FFC002840F05E873149E87B24F068FC1D
:1036B00000283FF447AD032E40F058872D49287D60
:1036C00024F05EFC002840F041872B49687E24F0FE
:1036D00057FC00283FF447AD052E40F03B872749B3
:1036E000A87F24F04DFC002840F03887244995F845
:1036F000230024F045FC00283FF447AD072E40F09E
:103700007084204995F8280024F03AFC002840F005
:1037100052841D4995F82D0024F032FC00283FF416
:1037200047AD092E3FF444AD4FF009094B4600F078
:1037300045BC00BFDC370020345000204821002069
:10374000B0720020D855002070830020D34D621045
:10375000683C0020740000207500002009920020C1
:10376000E53D0020ABAAAAAA742100204C2100202C
:10377000E8350020ED350020F2350020F735002037
:10378000FC35002001360020063600204C3E00208B
:103790004A210020B08F0020E83D002025F04003A2
:1037A0009BB2AB4223803FF48FABA04B0225142188
:1037B000FF220F201D7059709A7014F0BDFBFFF7A7
:1037C00083BB238823F00405ADB2AB4225803FF4D0
:1037D00071AB964B02251421FF220F201D705970EA
:1037E0009A7014F0A9FB2588FFF764BBE04600211E
:1037F0008F48F7F711FB00287BD1069B8D4A1B7879
:103800001060D90700F19585B8F1140F7FF484AAF0
:10381000039B93F88E20572A00F0A985079B1B680D
:1038200013F0040302D05A2A00F0DF835D2A00F06F
:1038300010865B2A00F045865E2A00F0B183562A86
:1038400000F0A08623782BB16F2A00F09786794B81
:1038500000211960972A00F0A586A72A00F07F832F
:103860000021BB2A149100F05C87B72A00F038874A
:10387000BE2A00F05987BD2A00F05F87792A00F040
:10388000CB877A2A00F0C1879E2A00F0B6879D2A4E
:1038900000F0AA87AE2A00F05387AD2A7FF43CAA35
:1038A000FF21002017F066FEFFF736BA039890F864
:1038B0009130002B3FF439AA069B1B7813F00103CB
:1038C0007FF433AA012280F8913080F89220FFF72C
:1038D0002CBA594B1B78069309E693F822309AF8D4
:1038E00000600433DBB2B34240F27982039B1E7066
:1038F000C8E5039A002382F8903006F027F9039B6D
:1039000093F88F30142B7FF407AA2378002B40F014
:10391000B787069B1B7803F00103002B7FF4FCA9FB
:1039200076E780F88E30BCF1000F3FF460AFFFF710
:10393000F3B90398012180F88C10FFF79EB9012894
:1039400000F0348598F8C8100123AB4001350B43D3
:10395000042D88F8C83004F10C047FF4F4ACFFF7B0
:103960004CBA47F00203BB4223803FF484AA2F4B9A
:10397000022214211A700F20FF2259709A7014F03D
:10398000DBFA2788FFF777BA1A464B00099806F545
:1039900096784CF8218000283FF415AE0D9803EB83
:1039A00001088044039800EB4808A8F82C20BAF1DD
:1039B000000F03D10C9802287FF605AEB5F802A0DF
:1039C0002A88B5F80480524490441C4A0FFA88F8BB
:1039D00082FB08021A48A2EBE87220F8038012B2B8
:1039E0004FF0010AEFE5059B002BCDD05CF82120BC
:1039F00096424FEA4103FFF4E0AD124A1148D25C0F
:103A000000EB0308002A00F08381022A40F04C8179
:103A100098F8012002EB820202EB820202F2EE220F
:103A200092B203297DDD12B2C9E500BF083600203D
:103A3000DC370020F423002009920020565555550C
:103A4000BC210020803E00200F9D0398B74BDDF87D
:103A5000408080F8009056460F2D014632460CBF3C
:103A600001220022DDF848A081F8296081F8285061
:103A70001A7006D11B21AE48F7F7CEF9002800F0E6
:103A8000D384AC48AC4B826819684368AB4DC160C5
:103A90008A1A9A42049AAA4EB2F826E0178B4FF07F
:103AA000010188BF0023297092F8225088BF80F856
:103AB00021300A9B317004359AF80000EDB2002BDA
:103AC00000F0568185429F4A40F295819E4D1646F0
:103AD00000210CB981460446A14218DA12F81130CF
:103AE00083B1022B0CD1737803EB830303EB8303C5
:103AF00003F2EE239BB225F8023B01310236E8E7E0
:103B00002B88F8E7CBB2032BFAD83B46F3E7039BAD
:103B100083F800900C9B8D4A013313700A9BFEF7CB
:103B2000FFBF012000FA01F80F9820EA080012B246
:103B30000F9044E512B9012289F80220844B0693C4
:103B400093F800A099F821700AF001031B20059357
:103B500024F040FA012F089000F0C4810AF0020A14
:103B600099F820207B4CDFF804827B4D724E052AA9
:103B700000F29180DFE802F08176032E3D4F012FA5
:103B800004BF052389F82030059B002B00F09980A5
:103B9000049B3068B3F91810B8F80230002261F3C2
:103BA0000F0263F31F42002361F30F0361F31F430E
:103BB000D9F81410CBF804208842CBF8003040F23A
:103BC00013814FF0030A47F230520323C9F81C2037
:103BD00089F820302B8843F002032B8006F084FC08
:103BE0003268D9F81C3013440422C9F8183089F817
:103BF0002020012F40F026843368D9F818209A42FB
:103C000049D2207818B924F0E5F9002843D12B884F
:103C100023F002032B803268B8F80630642101FBE0
:103C200003234FF48060002289F8202089F80320C4
:103C3000C9F8103014F0ACFA99F8202097E724F076
:103C4000F5F9012800F06284089B002B40F04D81BB
:103C5000012F20D03368D9F810209A4227D30123AE
:103C600089F82030012FD6D098F80830012B1ED0CB
:103C700016F026FB99F8202079E7059B002BDED172
:103C8000089B4FF48060002B00F09B8014F098FAA2
:103C90000022C9F81020BAF1000F40F09C80079B69
:103CA000D3F80080FEF756BF3BF80320B9E616F0C4
:103CB00007FB032240F6B83389F82020C9F81C30EE
:103CC00088E733687FE745F04003AB4223807FF409
:103CD0006CADFFF7F9B845F004039D4223800AD08C
:103CE0001E4B02251421FF220F201D7059709A705F
:103CF00014F022F925881A4B1A4AB3F904301A49EC
:103D000082FB0302DB17C3EBA2030B80FFF7D2B8E1
:103D1000CAB2022A40F20A83032AC5D1139A0A982A
:103D2000059F002808BF3A467BE600BFFD41002002
:103D3000DC3700204892002080A800207500002079
:103D400074000020803E0020B08F0020E53D002060
:103D5000C45100207C1C0020DE54002008360020C6
:103D60009054002067666666E43F00204C500020B7
:103D700085421946B04A60D8B04816460CB9A946E3
:103D80002C468C427FF7C3AE12F8113083B1022B60
:103D90000CD1737803EB830303EB830303F2EE236D
:103DA0009BB220F8023B01310236E7E70388F8E7CF
:103DB000CBB2022B03D9032BF8D17346F1E73B4674
:103DC000EFE714F0E5F963E7082014F0E1F9FFF7F5
:103DD00004B94FF0030A504614F0AEF85FE7039AB7
:103DE0001E461370FFF74EBB012FF2D199F8202029
:103DF0004FF0030ABBE69148164600210CB9A946CC
:103E00002C468C427FF783AE12F8113083B1022B1F
:103E10000CD1737803EB830303EB830303F2EE23EC
:103E20009BB220F8023B01310236E7E70388F8E74E
:103E3000CBB2032BFAD83B46F3E7804D16460CB9BC
:103E400081460446A142BFF662AE12F8113083B13A
:103E5000022B0CD1737803EB830303EB830303F290
:103E6000EE239BB225F8023B01310236E7E72B88AF
:103E7000F8E7CBB2022B03D9032BF8D17346F1E755
:103E80003B46EFE7C83881425CDA98F8C8109B7867
:103E90002941CA073FF583AA5B420120099314F028
:103EA0005FF9711E099B162900F20281DFE811F00B
:103EB000F2010602DB0153011A022B02C801B5010F
:103EC000A0018B0176010001530163012B02C8019F
:103ED000B5013F012B011701F000DC0003010125B2
:103EE000FEF744BE4FF0000A3AE698F80430002B83
:103EF0003FF4AEAE16F0E4F903224FF47A7389F87A
:103F00002020C9F81C3065E60A2024F063F82588D3
:103F10000746002800F0A182E90640F16583039B73
:103F200093F8D870002F7EF4DCAF0E2014F004F864
:103F3000039A2588012382F8D830002F7FF4A9A99D
:103F4000FEF7CFBF98F8C8300121A94023EA01034A
:103F500009F5FA7188F8C830A160FFF720BA38492E
:103F6000079B0A781B6842F004020A7003F00403FE
:103F7000344A0592FEF7D6BE00213348F6F74CFFCF
:103F800000287FF434AB0399322381F89300A1F821
:103F90009430FFF72CBB002B0CBF012002207DE7E3
:103FA0002A4B022203202A4C2A4922700B6014F06B
:103FB000D7F8FEF7B1BE4FF008094B4603EB830379
:103FC0001D4487F80090A978687819F0BDFC069B1D
:103FD000214A1B7801211170D9077FF5ECA8FEF763
:103FE000EFBF4FF007094B46E8E7039A92F891209C
:103FF000002A40F0EE83039991F8932082F00102A9
:1040000081F89320002A40F0DF831449096811F4F5
:10401000003104D012490979002940F036840A465B
:104020001048845C0D2C02F10C0200F0B4830131C5
:104030001529F6D19CE700BF803E0020B08F0020FC
:104040006154002054670020DC370020489700208E
:1040500095550020E454002028240020C03300207F
:104060007C54002070D10308D8F8CC009AF8026084
:1040700090F83B101944FE29A8BFFE2121EAE17106
:1040800080F83B10002E40F0F58314F091FF59E4C6
:10409000089841781944B1F5967FA8BF4FF49671FE
:1040A00021EAE17141709AF80230002B40F0FF8361
:1040B000D8F8CC00E9E7D8F8CC009AF8026090F87C
:1040C0003A1019446429A8BF642121EAE17180F8FB
:1040D0003A10002ED9D0172023F0DAFFE8E7D8F8FD
:1040E000CC0081781944C829A8BFC82121EAE17110
:1040F00081709AF80230002BC7D0142023F0C8FF3B
:10410000D8F8CC00C1E7D8F8CC0041781944C829C8
:10411000A8BFC82121EAE17141709AF80230002B52
:10412000B3D0132023F0B4FFD8F8CC00ADE7D8F813
:10413000CC0001781944C829A8BFC82121EAE1713F
:1041400001709AF80230002B9FD0122023F0A0FFBC
:10415000D8F8CC0099E7089A9AF8020091791944A6
:104160006429A8BF642121EAE1719171002840F01F
:10417000B5830D2E9CD0089E9AF8020071791944DF
:104180006429A8BF642121EAE171717100288FD0F0
:104190000E2023F07DFFD8F8CC0076E7D8F8CC00CD
:1041A0009AF80260017A1944C829A8BFC82121EAF7
:1041B000E1710172002E3FF468AF0B2023F068FF1D
:1041C000D8F8CC0061E7D8F8CC009AF80260C17941
:1041D0001944C829A8BFC82121EAE171C171002E84
:1041E0003FF453AF0A2023F053FFD8F8CC004CE73C
:1041F000D8F8CC009AF8026081791944C829A8BF80
:10420000C82121EAE1718171002E3FF43EAF0920FF
:1042100023F03EFFD8F8CC0037E7D8F8CC009AF866
:10422000022041791944C829A8BFC82121EAE171B7
:104230004171002A40F04A83112E7FF452AF24E7E7
:10424000D8F8CC009AF8022001791944C829A8BFEF
:10425000C82121EAE1710171002A40F01D83102E6E
:104260007FF453AF11E708990E791E44642EA8BF5E
:10427000642626EAE6760E7123F024FF9AF80230CF
:10428000002B3FF415AF0320314623F001FFD8F88F
:10429000CC00FAE6089801781944FA29A8BFFA2157
:1042A00021EAE17101709AF80230002B3FF400AF6F
:1042B000012023F0EDFED8F8CC00E6E608988178DE
:1042C00019446429A8BF642121EAE17181709AF838
:1042D0000230002B3FF4ECAE022023F0D9FED8F8D8
:1042E000CC00D2E6089E9AF80200F179194481F3D5
:1042F0000801F17100283FF4DBAE052023F0C8FE71
:10430000D8F8CC00C1E6D8F8CC009AF80220C178E1
:104310001944C829A8BFC82121EAE171C170002A47
:1043200040F0A0820F2E7FF404AFAEE6139AFFF7A1
:1043300078BBB84B1B78002B3EF4EEACB64BDB7869
:10434000002B7EF4E9AC039A92F890300133DBB293
:10435000032B82F890307EF6DFACB04B5B7813B95C
:10436000002D7EF4D9AC06F0BFF8FFF7C8BAAC4B0D
:10437000AC491A684FF47A73B3FBF2F3C3EB431200
:1043800003EB8203079A1268DB001606A1F8A83037
:1043900000F1CF80A44B05931B685C0700F1C0803F
:1043A000079B1B6803F00403FEF7BCBC3BF911102C
:1043B0009878B1F5617F4FF4966393FBF0F3C0F208
:1043C0009D8040F633008142A8BF01460C2EA1F526
:1043D000617191FBF3F100F08181182E7FF4B2AA94
:1043E000C9B2C8290B46A8BFC823D8F8CC00C67DDF
:1043F0005FFA83FEB6453FF4A5AA9B1B48BF07336F
:10440000DB109AF8022080F817E05E1CF6B23AB989
:10441000002E3FF497AA304613F0A2FEFFF792BA9F
:10442000182023F035FEF3E77B49804BCA681B68F0
:104430008B609B1AC82B7FF66DAB012381F821306E
:10444000FFF768BB3168D9F81C200A44C9F8182066
:1044500021E4774B00220120A5E5EA0600F1368130
:104460000B2023F0B7FD002840F00081AB0600F1DF
:104470005D81039B93F8D830002B3FF456AD002F9D
:104480007EF407AFFEF72DBD6A4A1268920304D589
:10449000694A1279002A40F0C681684819461A46CE
:1044A000455C0B2D01F10C010FD00132152AF7D11B
:1044B0000399002281F88F20002B7EF42DACFFF7AA
:1044C000A7B95F4B012202206DE55E4DD5F800E0F3
:1044D0005100BEF1000F07D08E1800EB86069EF843
:1044E00001E076787645E3D20A44574E574900EB0F
:1044F000820200202A6030800860D9E70C2E5DD04F
:10450000182E7FF41FAA00210B466EE73268B8F818
:104510000630642101FB0323C9F81030FFF794BB78
:10452000079B4B4A1B680A21118003F00403FEF726
:10453000F9BB484B1B789D077FF52CAF464B1B788A
:10454000042B7FF627AF19F08FF823E74FF004090B
:104550004B4633E54FF005094B462FE54FF0060972
:104560004B462BE54FF002094B4627E54FF0030978
:104570004B4623E54FF001094B461FE505F0E6FAEF
:10458000FEF7CABB10F012F9F5F740FE10F0F6F88E
:10459000F8F764FF012013F0E3FD039B93F88E20EE
:1045A000FFF750B9079B2D4A1B684FF4C871118063
:1045B0001D4A059203F00403FEF7B4BB0026314602
:1045C000274B09915B78B3423FF4BCA9304609F010
:1045D000CDF89AF8023009991BB1C9B20C2023F02A
:1045E00057FD0136F6B213E7102013F0E9FD202045
:1045F00013F0CEFD1B49081F19F0ACF81A4B02222C
:104600001A70039B93F8D830002B00F04D81258859
:10461000FEF73FBE09920020489200208C24002023
:10462000D4660020B05E00205467002080A80020DF
:10463000B4960020C03300207C54002070D10308C1
:10464000FE96002048230020E2230020E4230020DF
:10465000A0A800206154002064540020A2A80020DB
:1046600095550020143F0020CE3E0020AD4AAE4BB1
:10467000528993ED007A07EE902AF8EEE77AB0EED1
:10468000C77AB4EEE77AF1EE10FA7FF5EFAE93ED6C
:10469000017AB0EEC77AF4EEC77AF1EE10FA7FF73E
:1046A000E5AEAB063FF5E5AE202013F089FD9F494E
:1046B000039D7268B368C5F8D020081FC5F8D430D0
:1046C00019F048F89A4B01221A709AE7102013F05B
:1046D0005FFD974B25881F700127C1E6CEB26FE7BB
:1046E0000B464FF6FE71934A934854890590908982
:1046F000234401445381918110F058F8F5F786FD69
:1047000010F03CF8F8F7AAFE012013F029FD079BF2
:1047100003991B68002203F0040381F88F20FEF741
:1047200001BB0B460221DEE70223DCE7202013F069
:104730002FFD7F4B00221A7063E74FF6FE73D2E71E
:104740000121002016F016FF039B93F88E20FFF73F
:10475000A4B8049A115D9847032C19DC40F2EE22AC
:1047600040F6CA0300283EF4A0AE38F824E0698879
:10477000A0EB0E0009FB00F0A1EB0E0190FBF1F0A5
:1047800000F57A709042B8BF10469842A8BF18460C
:1047900000B2FEF78ABE694D2E684A003EB1541839
:1047A00000EB840476786478B442BFF4E1AB0A4449
:1047B00000EB8202624E634C2A6000215E4A318027
:1047C00021600592FEF7AEBA0C2013F0B5FBFEF7A0
:1047D000A3BA039C0122002184F89220564A84F84F
:1047E00091100592FEF79EBA0021FF2016F0C2FE3E
:1047F000039B93F88E20FFF74DB8012016F0BAFE08
:10480000039B93F88E20FFF742B84F4A137A43F088
:1048100001031372FEF780BA4B4A137A23F00103A7
:104820001372FEF779BA494A1278002A7FF435AE3E
:1048300013F066FB069B1B7803F0010338E6002D9E
:104840003EF4E9A9039B93F88DC0BCF1000F3EF440
:104850001BAA13F055FB039B94F800C083F88D60EE
:10486000FEF712BA0F20099323F012FCD8F8CC00FF
:10487000099B57E5162023F00BFCD8F8CC0004E484
:10488000039B93F88E10FEF7E0BE304909780029AB
:1048900043D01146FFF7C4BB1020099323F0F8FB67
:1048A000D8F8CC00099BDAE40127FFF73EBB1520BE
:1048B00023F0EEFBD8F8CC00FFF7E7BB05F014FEC1
:1048C000039A002382F88D30FEF7DCB9112009939A
:1048D00023F0DEFBD8F8CC00099BADE40D20099352
:1048E00023F0D6FB099B44E43BB11949194A0968F6
:1048F0004FF47A7000FB03131360039B93F88D3021
:10490000002B3EF4C1A913F0FBFA039A94F800C0FF
:10491000002382F88D30FEF7B7B913F0F1FAFEF7F5
:10492000FBB900BF683F0020C85200201C220020B5
:10493000CE3E0020F8360020546700204823002097
:10494000E2230020E4230020E8410020C752002099
:1049500080A80020F0230020F8B55D4B1B78DB0712
:104960002DD55C4B5C4D1C785C4E012C49D079D325
:10497000022C1BD06B7A7BB1EB886BB1584B1B7848
:1049800053B108F007FF00287CD0AB7A83422CBFDC
:1049900001230023337000E0337852492A7A9C4285
:1049A00038BF1C460C70002A53D1F8BD4E494F4AFF
:1049B000098812889142DDD901241C70DAE74A4B3C
:1049C0004B48454D1988EC78B0F8DA30A142A1EB9C
:1049D000030303F1020223D32B788B4220D33D4BF8
:1049E0001C78032C51D03D4E424A1278022A04D141
:1049F0003B4F414A3F78D7809480012CA0F8DA10D1
:104A0000B5D13A4A38491288E87A0988121A91428F
:104A100035DD3A4A12888A42ACD200241C70A9E7DC
:104A2000B1EB440FDBDC2B4B1C78032CDBD0042ACE
:104A3000D9D82A4EDFF8A8C0DFF8C0E02B4F0022FB
:104A4000032434701C708CF80020AEF800203A80EB
:104A5000CAE7012C36D0022C10D10720BDE8F8405F
:104A600013F06ABA254A20491288E87A0988121A8E
:104A700091423FF77FAF01241C707BE7F8BD022411
:104A80001C7077E70223337087E7042AABD82A78B3
:104A900091FBF2F20132082ADFF844E06C78AE783C
:104AA000164FA8BF08228EF8002092B216FB02F61D
:104AB00014FB02F20D4C3E80084E2280002434701C
:104AC0001C7091E70820BDE8F84013F035BA00BF2C
:104AD000C45100206C2500207C5400207225002049
:104AE000C7520020429200208052002070250020F2
:104AF00048210020D9510020DC5100206E250020E3
:104B00002DE9F04FDFF808B12DED0C8B9BF800304C
:104B100099B0012B039001F03082DFF8F8A09AF8E9
:104B20000021002A41F03882072B01F03F824FF02C
:104B30000009344C63682046984700286ED0B4F8CA
:104B4000A860002284F84920002E40F09382B4F936
:104B50002450E16AB4F92600226BB4F92830691AAE
:104B6000A16329490091821A606BE2630D461B1A0A
:104B700094F84A10236404F138000EF039F82B68D9
:104B800013F0005302F0CA81D4ED0F5AD4ED0E7A1F
:104B90001E4A9AED416ADAED426A9AED437ADAF8F2
:104BA00010311268B8EEE58AD4ED105AF8EEE77AC3
:104BB000F8EEE58A013377EE867A38EE268A78EECB
:104BC000878A9342CAED417A8AED428ACAED438AC6
:104BD000CAF8103101F0A8869BF80060142E02F08C
:104BE000AE870023DAF818510193062D02F258829D
:104BF000DFE815F0DF14CB14F61126171E16B516D4
:104C0000A21500BFB05E002070830020586700200E
:104C1000D951002024220020DDF804909BF8008068
:104C2000B8F1070F00F0DD829AF828310593002BC8
:104C300040F0E382CD4B5B79002B40F016820123DC
:104C40009BF800208AF82831072A02F0838200238B
:104C50000793C74B9AED4CAA93ED007AC54AC64B11
:104C60001268C64F9AED4B9ADFF890939FEDC4BA45
:104C7000DFEDC49ADFEDC4BADFEDC4CADFEDC4AA2C
:104C80009FEDC4CADFF87883C34E0493F7EE007A31
:104C900077EECA8A002468EE878A0292F4EEE78AE9
:104CA000F1EE10FA88BFF0EE678A0193254600976F
:104CB000BA4B2344D3ED007AB94BF5EE407A234446
:104CC000F1EE10FA93ED008A17D0B64B234493ED22
:104CD000007A78EE476AB0EEE66AF4EEC67AF1EE54
:104CE00010FA08D5F5EEC06AF1EE10FACCBF37EE37
:104CF000878A37EE678A83ED008AAB4B1F88BB0734
:104D000000F08382022D04F02C850299A74B91F8C4
:104D1000322006EE902A33F91520234407EE102A9C
:104D200093ED016A91F83130B8EEC77AF8EEE66A91
:104D30005A4207EE902AA6EE867A6900F8EEE77AE4
:104D4000B4EEE77AF1EE10FA0AD407EE903AF8EEF4
:104D5000677AF4EEC77AF1EE10FA88BFF0EE477A80
:104D6000934B0693934A0B44515EB3F90A30C81A29
:104D700007EE100AB8EEC77AF807E7EE697A40F155
:104D8000B9828D4F97ED008A27EE888A9AF868716C
:104D9000E7B1894FDAF86C01D7ED007A874F5B1ADB
:104DA00007EE103A039B396867EEA97AB8EEC78A16
:104DB0001F1A8F4228EE278A01F3AE81F7EE007AA0
:104DC000B4EEE7AAF1EE10FA01F172817C4B2344B4
:104DD000D3ED007A019BD3ED01DA009B69EE277ACF
:104DE00038EE6DDA67EE8D7AC3ED007A754B99ED8A
:104DF000007AD3ED007A744BD6ED006A67EE277A1D
:104E0000234427EEA87AD3ED007A67EE277AB0EE36
:104E1000667AA7EE8D7AF0EE477A9AED4C6AB7EE95
:104E2000007AB4EEC76AF1EE10FAACBF012300239A
:104E300043B1F0EEE66AB0EEE77AB4EEE67AF1EE70
:104E400010FA01D5C6ED007A022D04F083845F4A82
:104E50005F4B52F825001B68B0EE6D0A98475D4A1B
:104E60005D4B52F825001B689847029B93F83A3037
:104E7000632B04D84C4B1B88002B01F05F81B0EEF4
:104E80006C8A564BD9ED007A38EE400A234493EDF4
:104E9000008A83ED000A029B30EE480A93F848200E
:104EA00080EE278ADAB1F7EE007AB4EEE7AAF1EEE7
:104EB00010FA14DB4A4BD3ED007AB0EEC87AB4EEA8
:104EC000E77AF1EE10FA0ADD464BD3ED007AB0EE48
:104ED000CDDAB4EEE7DAF1EE10FA01F38D81424B50
:104EE0009AF878212344D3ED007A69EE277A27EEE9
:104EF000888A88ED008A32B9009BC6ED00CAC3EDEE
:104F000000CAC8ED00CA009B04330093019B04341F
:104F100004330C2C05F1010508F1040806F1040620
:104F200001937FF4C5AE9BF80030072B02F0CC80D4
:104F3000012B02F0FF80002304932C4B00931A46B0
:104F40000C4B12681B680192114693F82F2011F444
:104F50008053069300F05082254B02931B7825481E
:104F6000079013F0010F244B03934BE09C5E00204D
:104F7000304A0020E4540020D4660020743600201B
:104F800000009642CDCCCC3DAE47813F00000000F2
:104F90000000C8420000344380360020244A00202C
:104FA0005823002064230020E054002070230020B8
:104FB000F836002090540020084A0020344A00208F
:104FC000DC4900202C000020E84900204C4A002049
:104FD000484A0020B04A0020AC4A00209423002018
:104FE000444A0020404A0020F449002070830020F9
:104FF000C4510020C8520020B0720020204A002076
:105000008C360020198BA94B90ED037ADB8808BF02
:10501000AAF88011C81A07EE900AF8EEE77AB4EE03
:10502000E77AF1EE10FA42F26980CC1806EE904A67
:10503000F8EEE66AB4EEE67AF1EE10FA81F23D841B
:10504000BAF88031984283F24881994B994993ED9F
:10505000004AD1ED004A984BCAED614A8AED624A96
:10506000D3ED006ADFED957AE2E1954B1B78013BC9
:10507000DBB2E5E59349944B4978049300911B68B2
:10508000924F9BF80080B7F906004FF47A71B1FB9C
:10509000F3F3C3EB431503EB8503DD00ADB2AE4282
:1050A00002F03186E16FB4F924E0236E4A1C07EE6A
:1050B00090EA7344012AE2672366F8EEE77A02F089
:1050C0002C86D4ED1B5AD4ED1D6A07EE102A37EE5C
:1050D000E56AB8EEC75A012E86EE057A37EE257AD4
:1050E00077EEC77A84ED1C7AE6EE276A84ED1B7AA8
:1050F000F0EE667AC4ED1E6AC4ED1D6A03F04C81C1
:10510000D4F89010B4F926E0636E4A1C07EE90EADA
:105110007344012AC4F890206366F8EEE77A02F03F
:105120001486D4ED205AD4ED226A07EE102A37EE09
:10513000E56AB8EEC75A012E86EE057A37EE257A73
:1051400077EEC77A84ED217AE6EE276A84ED207A3D
:10515000F0EE667AC4ED236AC4ED226A03F03E8164
:10516000D4F8A410B4F928E0A36E4A1C07EE90EA24
:105170007344012AC4F8A420A366F8EEE77A02F08B
:10518000FD85D4ED255AD4ED276A07EE102A37EEB7
:10519000E56AB8EEC75A012E86EE057A37EE257A13
:1051A00077EEC77A84ED267AE6EE276A84ED257AD3
:1051B000F0EE667AC4ED286AC4ED276A03F0308108
:1051C000F880B4F8A8309BF80080013BA4F8A83020
:1051D00004990023B8F1070F4B608B60CB607FF41C
:1051E00023ADF9F7F5FA394F9AF828310593A0EB7A
:1051F00009003880002B3FF41DAD013B8AF82831AF
:1052000019B0BDEC0C8BBDE8F08F9AF8683163B132
:10521000022D04F0A9822E4B06932E4A03EB450380
:1052200032F91510B3F90A30B3E52B4B234493ED53
:10523000000A019BD3ED01DA009B29EE000A38EE4B
:105240006DDA022D20EE0D0A83ED000A7FF4CEAD5B
:10525000224A234B10681B689847224B99ED007A2D
:10526000D3ED007A204BD6ED006A1A781F4B83ED00
:10527000020A1F4B67EE277A234467EEA87A93ED64
:10528000006A67EE867AB0EE667AA7EE8D7A012A1A
:10529000F0EE477A02D0192A7FF4BFADB4EECBDA34
:1052A000F1EE10FACCBF01230023C1E534500020F9
:1052B0002C50002028500020445000200000000006
:1052C000284F00209C5E0020D4660020DC51002086
:1052D000F836002090540020DC490020104F0020B8
:1052E000244F00202C000020D849002074360020D4
:1052F000E8490020DAED576A9AED587AB2F900E0F1
:10530000B2F90270B4EEE67AF1EE10FA8EEAEE70BF
:1053100087EAE77C4CBFB7EE007AF7EE006AA0EBB5
:10532000EE70ACEBE77C4CBF77EE665A76EEC75A70
:10533000604540F32387BEF1000FD6BFCEF10000D9
:1053400007EE10EA07EE100A274FB8EEC77A3F784B
:1053500027EE297A002F00F02187244F97ED005A7D
:10536000B5EEC05AF1EE10FA41F33686204FD7ED74
:10537000004AF5EEC04AF1EE10FA41F32D8634EE04
:10538000C77AB7EE006AC7EE246A75EEC65AF4EE25
:10539000C66A65EEAA5AF1EE10FA85EE857A88BFE4
:1053A000F0EE466AF5EEC06AF1EE10FA37EE067AD4
:1053B000B8BFF0EE6C6A66EE876AF4EEC66AF1EE8C
:1053C00010FA88BFF0EE466AF5EEC06AF1EE10FA08
:1053D000B8BFF0EE6C6A074F97ED007A67EE877AF8
:1053E000A7EEA68AD2E400BF144A0020104A00208B
:1053F000184A00200C4A0020E24B03935B8BE249E1
:10540000079107EE903AE14B91ED037AE04993ED75
:10541000004AE04BD1ED004AD3ED006ADE4B8AED45
:10542000624AF8EEE77A029377EE677ACAED614A4C
:10543000C7EEA62AD949DA4B91ED008AD949DFEDAA
:10544000DA6A91ED005AD9499FEDD96AD1ED005A37
:1054500093ED007AF7EE007AF4EEE72A38EE058A4B
:10546000F1EE10FA88BFF0EE672A38EE258AF4EEE6
:10547000E62AF1EE10FA28EE066AB8BFF0EE662AC8
:10548000F1EE476A34EEC43AB4EEE66AF1EE10FA91
:10549000CAED632A8AED653A00F16B85B4EEC76AFE
:1054A000F1EE10FA88BFB0EE476ABC4BDFEDC07A70
:1054B000D3ED018ABB4B93ED015ABC4B78EE858A44
:1054C000D3ED015A78EEA58A68EEA77AF4EEE76A82
:1054D000F1EE10FA08DCB4EEE77AF1EE10FA8CBFC8
:1054E000F0EE676AF0EE476AAC4BDFEDB17A93ED10
:1054F000029AAC4BD3ED025AAE4B39EE259A93ED9E
:10550000007A69EE277AF1EE475AF4EEE57AF1EE89
:1055100010FA08D4F4EEC77AF1EE10FA8CBFF0EE70
:10552000475AF0EE675A002A41F08982F7EE007A76
:10553000A14B5A789AF89831002AA04AFFEE003A17
:10554000B7EE007A127814BFB0EE472AB0EE632AA5
:10555000002B14BFB0EE635AB0EE475A002A02F097
:105560005B84F4EEC77AF1EE10FA65EE825A944B42
:1055700041F3128393ED027A93ED011AD3ED031AEE
:105580009FED892A26EE877A67EE853AA6EE017AA4
:10559000A5EEA17A27EE237AB4EEC27AF1EE10FAE4
:1055A000B4BFF0EE427AF0EE477A8DED0C7A88BF08
:1055B000B0EE427A012A00F0BE8193ED065AD3ED97
:1055C000051A93ED072A26EE855AA6EE215AA5EE76
:1055D000825A25EE235AB4EEC57AF1EE10FAF4EEB3
:1055E000C57A8CBFB0EE452AB0EE472AF1EE10FA2C
:1055F00058BFB0EE427AB8BFF0EE457A022A8DED80
:105600000D5A00F0988193ED0A5AD3ED091A93EDE3
:105610000B2A26EE855AA6EE215AA5EE825A25EED1
:10562000235AB4EEC57AF1EE10FAF4EEC57A8CBFC7
:10563000B0EE452AB0EE472AF1EE10FA58BFB0EEB0
:10564000427AB8BFF0EE457A032A8DED0E5A00F08B
:10565000728193ED0E5AD3ED0D1A93ED0F2A26EEBB
:10566000855AA6EE215AA5EE825A25EE235AB4EEAB
:10567000C57AF1EE10FAF4EEC57A8CBFB0EE452A89
:10568000B0EE472AF1EE10FA58BFB0EE427AB8BF3A
:10569000F0EE457A042A8DED0F5A00F04C8193ED1F
:1056A000125AD3ED111A93ED132A26EE855AA6EE5F
:1056B000215AA5EE825A25EE235AB4EEC57AF1EEB0
:1056C00010FAF4EEC57A8CBFB0EE452AB0EE472A48
:1056D000F1EE10FA58BFB0EE427AB8BFF0EE457A5C
:1056E000052A8DED105A00F0268193ED165AD3ED60
:1056F000151A93ED172A26EE855AA6EE215AA5EE25
:10570000825A25EE235AB4EEC57AF1EE10FAF4EE81
:10571000C57A8CBFB0EE452AB0EE472AF1EE10FAFA
:1057200058BFB0EE427AB8BFF0EE457A062A8DED4A
:10573000115A00F0008193ED1A5AD3ED191A93ED26
:105740001B2A26EE855AA6EE215AA5EE825A25EE90
:10575000235AB4EEC57AF1EE10FAF4EEC57A8CBF96
:10576000B0EE452AB0EE472AF1EE10FA58BFB0EE7F
:10577000427AB8BFF0EE457A072A8DED125A00F052
:10578000DA801FE0B0720020C8520020F0370020FD
:10579000285000203C500020C451002074360020C6
:1057A0002C4F002080360020000000008C360020A6
:1057B0006F12833A304F002090390020C9510020E9
:1057C000684F002093ED1E5AD3ED1D1A93ED1F2A4A
:1057D00026EE855AA6EE215AA5EE825A25EE235AC8
:1057E000B4EEC57AF1EE10FAF4EEC57A8CBFB0EEE5
:1057F000452AB0EE472AF1EE10FA58BFB0EE427AD1
:10580000B8BFF0EE457A082A8DED135A00F0938068
:1058100093ED225AD3ED211A93ED232A26EE855AD1
:10582000A6EE215AA5EE825A25EE235AB4EEC57A89
:10583000F1EE10FAF4EEC57A8CBFB0EE452AB0EE68
:10584000472AF1EE10FA58BFB0EE427AB8BFF0EE38
:10585000457A092A8DED145A6DD093ED265AD3ED71
:10586000251A93ED272A26EE855AA6EE215AA5EE93
:10587000825A25EE235AB4EEC57AF1EE10FAF4EE10
:10588000C57A8CBFB0EE452AB0EE472AF1EE10FA89
:1058900058BFB0EE427AB8BFF0EE457A0A2A8DEDD5
:1058A000155A48D093ED2A5AD3ED291A93ED2B2A95
:1058B00026EE855AA6EE215AA5EE825A25EE235AE7
:1058C000B4EEC57AF1EE10FAF4EEC57A8CBFB0EE04
:1058D000452AB0EE472AF1EE10FA8DED165A58BF60
:1058E000B0EE427AA8BFB0EE675A0B2A02F0F184FC
:1058F000D3ED2E7AD3ED2D1A93ED2F2A66EEA77AEB
:10590000E1EE867AE2EE257A67EEA37AF4EEC77AC4
:10591000F1EE10FAF4EEC57A8CBFF0EE476AF0EEC5
:10592000676AF1EE10FACDED177A98BFB0EE667A9D
:10593000B8BFF0EE457A77EEC77AF7EE006AF4EE7C
:10594000E67AF1EE10FACAED4C7A42F3B28486EEB2
:10595000A77A012ADDED0C7A67EE877ACDED0C7A15
:1059600055D0DDED0D7A67EE877A022ACDED0D7AFE
:105970004DD0DDED0E7A67EE877A032ACDED0E7AF3
:1059800045D0DDED0F7A67EE877A042ACDED0F7AE8
:105990003DD0DDED107A67EE877A052ACDED107ADD
:1059A00035D0DDED117A67EE877A062ACDED117AD2
:1059B0002DD0DDED127A67EE877A072ACDED127AC7
:1059C00025D0DDED137A67EE877A082ACDED137ABC
:1059D0001DD0DDED147A67EE877A092ACDED147AB1
:1059E00015D0DDED157A67EE877A0A2ACDED157AA6
:1059F0000DD0DDED167A67EE877A0B2ACDED167A9B
:105A000005D0DDED177A27EE877A8DED177AE14B19
:105A1000196811F0805100F0AC834FF07C53CAF844
:105A20008C31002A02F0F281029BDB4E1F78DB4CA6
:105A3000DB48DC4DD6ED005A9AF89031039EE478AD
:105A40000078B5F90650DAED636A768B07F0010C41
:105A5000019F07F0100E07F48007002B40F0AB8287
:105A6000BEF1000F00F0AE85BCF1000F42F07E8366
:105A7000002C42F05A84CC4BDDED0C7A93ED007A89
:105A8000CA48E7EE267ABDEEE47A17EE101AB0EEB9
:105A9000447AA3EE277A0D46F0EE477AFDEEE77AD8
:105AA000BDEEC47A17EE906A17EE104AB142A8BF55
:105AB0003546B442C8BF254607EE905AF8EEE77A5D
:105AC000012AC0ED007A00F04D8193ED047ADDEDFE
:105AD0000D7AE7EE267AB0EE447AA3EE277AFDEE51
:105AE000C77A17EE906A17EE905A8E42A8BF0D46FD
:105AF000A642B8BF254607EE905AF8EEE77A022A8A
:105B0000C0ED017A00F02E8193ED087ADDED0E7A7A
:105B1000E7EE267AB0EE447AA3EE277AFDEEC77A56
:105B200017EE906A17EE905A8E42A8BF0D46A64215
:105B3000B8BF254607EE905AF8EEE77A032AC0ED83
:105B4000027A00F00F8193ED0C7ADDED0F7AE7EE2B
:105B5000267AB0EE447AA3EE277AFDEEC77A17EEE6
:105B6000906A17EE905A8E42A8BF0D46A642B8BF63
:105B7000254607EE905AF8EEE77A042AC0ED037A3C
:105B800000F0F08093ED107ADDED107AE7EE267AE2
:105B9000B0EE447AA3EE277AFDEEC77A17EE906A4C
:105BA00017EE905A8E42A8BF0D46A642B8BF2546B2
:105BB00007EE905AF8EEE77A052AC0ED047A00F075
:105BC000D18093ED147ADDED117AE7EE267AB0EE0E
:105BD000447AA3EE277AFDEEC77A17EE906A17EEA5
:105BE000905A8E42A8BF0D46A642B8BF254607EE82
:105BF000905AF8EEE77A062AC0ED057A00F0B280F6
:105C000093ED187ADDED127AE7EE267AB0EE447A5B
:105C1000A3EE277AFDEEC77A17EE906A17EE905A38
:105C20008E42A8BF0D46A642B8BF254607EE905A41
:105C3000F8EEE77A072AC0ED067A00F0938093ED3C
:105C40001C7ADDED137AE7EE267AB0EE447AA3EE05
:105C5000277AFDEEC77A17EE906A17EE905A8E42B9
:105C6000A8BF0D46A642B8BF254607EE905AF8EEEB
:105C7000E77A082AC0ED077A74D093ED207ADDED3B
:105C8000147AE7EE267AB0EE447AA3EE277AFDEE98
:105C9000C77A17EE906A17EE905A8E42A8BF0D464B
:105CA000A642B8BF254607EE905AF8EEE77A092AD1
:105CB000C0ED087A56D093ED247ADDED157AE7EE43
:105CC000267AB0EE447AA3EE277AFDEEC77A17EE75
:105CD000906A17EE905A8E42A8BF0D46A642B8BFF2
:105CE000254607EE905AF8EEE77A0A2AC0ED097ABF
:105CF00038D093ED287ADDED167AE7EE267AB0EE0D
:105D0000447AA3EE277AFDEEC77A17EE906A17EE73
:105D1000905A8E42A8BF0D46A642B8BF254607EE50
:105D2000905AF8EEE77A0B2AC0ED0A7A1AD093ED72
:105D30002C7ADDED177AE6EE877AA3EE274AFDEEA0
:105D4000C47A17EE903A9942A8BF19469C42D8BF30
:105D50000C4607EE904AF8EEE77AC0ED0B7A002A7F
:105D600000F0F98392001249104824F005FA114B13
:105D70001B68002B00F0F4830F4B1B78192B22D8E3
:105D800001220E4902FA03F31940002942F054831C
:105D900016E000BFDC370020344F0020489200207E
:105DA000FC6D0020B08F0020684F0020C836002016
:105DB000384F0020D4490020D84900203241300318
:105DC0001E0301F1AE86AD4DAD4E019B9C061BD569
:105DD000F37AFF2B04D0AB4A12789A4201F29C86E8
:105DE000B6F90870F37D2F80FF2B04D0A54A1278F6
:105DF0009A4201F28C86B6F914406C80082022F099
:105E0000E9F8002841F0A083B6F90600B5F900E0F2
:105E1000B5F90270B6F91210B6F91E20B5F90440B2
:105E2000B6F90430B5F906C07045A8BF7046B9424E
:105E3000A8BF3946A242A8BF22469E45A8BF034636
:105E40002B80B6F91030B5F90800BB42C8BF19461F
:105E5000B6F92A306980B6F91C10B6F9347063457A
:105E6000A8BF6346A142CCBF0C461446B6F9362003
:105E7000AC80B6F92840B5F90A108242A8BF0246A4
:105E8000A445ACBF9C46A446B6F94230B5F90C40D7
:105E9000A5F806C08B42A8BF0B468742CCBF384648
:105EA0001046B6F94E202881B6F94000B5F90E70BB
:105EB000A242A8BF22468842C8BF0346B6F95A008C
:105EC000B6F94C106B81B842B6F958306E4EA8BF87
:105ED00038469F42A8BF0346A142D8BF1146A981B8
:105EE000EB81B38923B3694FDFF8B891DFF8908174
:105EF00007F11004B7F9023000EE103A4846B8EE48
:105F0000C00AF2F7EDFB24F0ABFAB8F90430B8F9A7
:105F1000062000B2984209F12C0908F10C0803DBB5
:105F200082421346A8BF034627F8023FA742E1D1A9
:105F3000574B1B78013B182B00F2C485DFE813F0A8
:105F4000B005C205C205F00AC205C205C2051F0E92
:105F5000C205C205C205C205C2055F0EC205C20563
:105F6000C205C2050E0EF00A500EC205C2055F0E34
:105F7000B005B0EE666AFFF798BA464BDFF828A185
:105F80001968454A454F9AF80031C9691288398025
:105F90007A80002B3EF4CBAD04F014FF00238AF886
:105FA00000319BF80030072B7EF4C1ADF8F710FCF0
:105FB0008146FEF7BEBDBEF1000F00F04B81BCF183
:105FC000000F42F02181002841F03A82FDEEC47AB0
:105FD0000DF1300E17EE906AFDEEE47A0EEB8203BF
:105FE00017EE907AFDEEE57A2D48DFF8C090CDF8F7
:105FF00024A017EE905AB1EE436A84F001084FFADC
:1060000084FC08929A46034693ED007AFEEC017AEE
:10601000E7EE267A3A461030B0EE647AA6EE277A9A
:10602000FDEEC77A17EE903A9F42A8BF1A469D42EE
:10603000CCBF002104F00101002914BF11462946FC
:106040009E42CCBF002308F0010307EE901A002BFC
:1060500014BF13463346B8EEE77A07EE903AF8EEEF
:10606000E77ABCF1000F18BFF0EE477AD645E9ECAD
:10607000017AC8D1089ADDF824A070E6B83600206D
:10608000D0500020D8550020006D0020B6360020EA
:10609000D849002038940020DE330020DC51002055
:1060A000684F00209047002024220020C83600209E
:1060B000069BB2F90070B3F90A305A49F81A096818
:1060C00080EAE073A3EBE0738B42BEF67FAEB2F9D9
:1060D0000230069AB2F90C209A1A82EAE273A3EB14
:1060E000E27399427EF772AE04994F4BD1ED017A7B
:1060F00093ED007AF0EEE77AF4EEC77AF1EE10FA5B
:106100007EF564AED1ED027AF0EEE77AB4EEE77A8E
:10611000F1EE10FA7EF75AAE444B1A8800238AF843
:106120006831002A40F0EA83414A424B11781868EE
:1061300081F00101F3F74EFDFEF748BE3E4B3F4AAA
:10614000234493ED007AD2ED007A3D4B67EE277A37
:10615000F7EE006AF4EEE67AF1EE10FA93ED007ACB
:1061600088BFF0EE667A67EE877A27EE888AFEF7B8
:1061700088BE019B5F023FF550AC52E4002FD6BFB2
:10618000784207EE107A07EE100A2E4FB8EEC77A63
:106190003F7827EE297A002F7FF4DFA82A4FD7ED2A
:1061A000006AF4EEEB6AF1EE10FA40F1BE87B7EE4A
:1061B000005A35EE665A9FED256A254F3CEE477A28
:1061C00025EE065A97ED006AE7EE056A26EE867A16
:1061D000B5EEC07AF1EE10FA40F2FE86CAEE876A9A
:1061E000B7EE006A35EEC67AF0EE465AE7EE265A6A
:1061F000F0EE656AFFF7E1B801230399CAF86C1164
:10620000022A8AF868317EF46AAE084A1288002AA7
:1062100043F0E181064A074B11781868F3F7DAFC7E
:10622000FEF75DBE384A00203C4A002058A80020F6
:106230005AA800205CA8002080230020044A0020E7
:10624000004A0020144A00201C4A0020610BB63B83
:10625000104A0020D44BDDED0C7A93ED007A002833
:1062600040F09887E7EE267AD048B1EE436AB0EE68
:10627000647AA6EE277AF0EE477ABDEEE47A002C37
:1062800042F0F282FDEEE77A17EE104A17EE906ABE
:10629000FDEEC47AB44217EE901A17EE105AA8BF5A
:1062A0003546B142C8BF0D4607EE905AF8EEE77A80
:1062B000012AC0ED007A00F04A8193ED047ADDED09
:1062C0000D7AE7EE267AB0EE647AA6EE277AFDEE36
:1062D000C77A17EE906A17EE905AA642A8BF2546D5
:1062E0008E42B8BF0D4607EE905AF8EEE77A022AC2
:1062F000C0ED017A00F02B8193ED087ADDED0E7A86
:10630000E7EE267AB0EE647AA6EE277AFDEEC77A3B
:1063100017EE906A17EE905AA642A8BF25468E4205
:10632000B8BF0D4607EE905AF8EEE77A032AC0EDA3
:10633000027A00F00C8193ED0C7ADDED0F7AE7EE36
:10634000267AB0EE647AA6EE277AFDEEC77A17EECB
:10635000906A17EE905AA642A8BF25468E42B8BF53
:106360000D4607EE905AF8EEE77A042AC0ED037A5C
:1063700000F0ED8093ED107ADDED107AE7EE267AED
:10638000B0EE647AA6EE277AFDEEC77A17EE906A31
:1063900017EE905AA642A8BF25468E42B8BF0D46BA
:1063A00007EE905AF8EEE77A052AC0ED047A00F07D
:1063B000CE8093ED147ADDED117AE7EE267AB0EE19
:1063C000647AA6EE277AFDEEC77A17EE906A17EE8A
:1063D000905AA642A8BF25468E42B8BF0D4607EE8A
:1063E000905AF8EEE77A062AC0ED057A00F0AF8001
:1063F00093ED187ADDED127AE7EE267AB0EE647A44
:10640000A6EE277AFDEEC77A17EE906A17EE905A3D
:10641000A642A8BF25468E42B8BF0D4607EE905A49
:10642000F8EEE77A072AC0ED067A00F0908093ED47
:106430001C7ADDED137AE7EE267AB0EE647AA6EEEA
:10644000277AFDEEC77A17EE906A17EE905AA642A9
:10645000A8BF25468E42B8BF0D4607EE905AF8EE0B
:10646000E77A082AC0ED077A71D093ED207ADDED46
:10647000147AE7EE267AB0EE647AA6EE277AFDEE7D
:10648000C77A17EE906A17EE905AA642A8BF254623
:106490008E42B8BF0D4607EE905AF8EEE77A092A09
:1064A000C0ED087A53D093ED247ADDED157AE7EE4E
:1064B000267AB0EE647AA6EE277AFDEEC77A17EE5A
:1064C000906A17EE905AA642A8BF25468E42B8BFE2
:1064D0000D4607EE905AF8EEE77A0A2AC0ED097ADF
:1064E00035D093ED287ADDED167AE7EE267AB0EE18
:1064F000647AA6EE277AFDEEC77A17EE906A17EE59
:10650000905AA642A8BF25468E42B8BF0D4607EE58
:10651000905AF8EEE77A0B2AC0ED0A7A17D093ED7D
:106520002C7ADDED177AE6EE877AE6EE274AFDEE65
:10653000E47A17EE903A9C42A8BF1C469942D8BF15
:10654000214607EE901AF8EEE77AC0ED0B7ABCF11F
:10655000000F3FF404AC164B1B68002B7FF40CAC0F
:10656000144B1B7893B1144B187860B10F4D134E38
:106570000024E0B23368B5EC010A98470E4B187856
:1065800001348442F5DB0E4B1B6898479BF80030C2
:10659000072B00F0AB8501238AF8003119B0BDEC60
:1065A0000C8BBDE8F08F00BF684F0020C83600207C
:1065B000D449002064720020C9510020F06D0020F1
:1065C000F86D0020D24BDDED0C7A93ED007A002CB3
:1065D00041F05484E7EE267ACE48BDEEE47A17EE19
:1065E000101AB0EE447AA3EE277A0D46F0EE477A01
:1065F000FDEEE77ABDEEC47A17EE906A17EE104A08
:10660000B142A8BF3546B442C8BF254607EE905AEE
:10661000F8EEE77A012AC0ED007A98D093ED047A7B
:10662000DDED0D7AE7EE267AB0EE447AA3EE277A16
:10663000FDEEC77A17EE906A17EE905A8E42A8BF09
:106640000D46A642B8BF254607EE905AF8EEE77A07
:10665000022AC0ED017A3FF47AAF93ED087ADDEDBE
:106660000E7AE7EE267AB0EE447AA3EE277AFDEEB4
:10667000C77A17EE906A17EE905A8E42A8BF0D4661
:10668000A642B8BF254607EE905AF8EEE77A032AED
:10669000C0ED027A3FF45BAF93ED0C7ADDED0F7A3B
:1066A000E7EE267AB0EE447AA3EE277AFDEEC77ABB
:1066B00017EE906A17EE905A8E42A8BF0D46A6427A
:1066C000B8BF254607EE905AF8EEE77A042AC0EDE7
:1066D000037A3FF43CAF93ED107ADDED107AE7EEEC
:1066E000267AB0EE447AA3EE277AFDEEC77A17EE4B
:1066F000906A17EE905A8E42A8BF0D46A642B8BFC8
:10670000254607EE905AF8EEE77A052AC0ED047A9E
:106710003FF41DAF93ED147ADDED117AE7EE267AA2
:10672000B0EE447AA3EE277AFDEEC77A17EE906AB0
:1067300017EE905A8E42A8BF0D46A642B8BF254616
:1067400007EE905AF8EEE77A062AC0ED057A3FF494
:10675000FEAE93ED187ADDED127AE7EE267AB0EE12
:10676000447AA3EE277AFDEEC77A17EE906A17EE09
:10677000905A8E42A8BF0D46A642B8BF254607EEE6
:10678000905AF8EEE77A072AC0ED067A3FF4DFAEBA
:1067900093ED1C7ADDED137AE7EE267AB0EE447ABB
:1067A000A3EE277AFDEEC77A17EE906A17EE905A9D
:1067B0008E42A8BF0D46A642B8BF254607EE905AA6
:1067C000F8EEE77A082AC0ED077A3FF4C0AE93ED01
:1067D000207ADDED147AE7EE267AB0EE447AA3EE65
:1067E000277AFDEEC77A17EE906A17EE905A8E421E
:1067F000A8BF0D46A642B8BF254607EE905AF8EE50
:10680000E77A092AC0ED087A3FF4A1AE93ED247A25
:10681000DDED157AE7EE267AB0EE447AA3EE277A1C
:10682000FDEEC77A17EE906A17EE905A8E42A8BF17
:106830000D46A642B8BF254607EE905AF8EEE77A15
:106840000A2AC0ED097A3FF482AE93ED287ADDED95
:10685000167AE7EE267AB0EE447AA3EE277AFDEEBA
:10686000C77A17EE906A17EE905A8E42A8BF0D466F
:10687000A642B8BF254607EE905AF8EEE77A0B2AF3
:10688000C0ED0A7A3FF463AE93ED2C7ADDED177A12
:10689000E6EE877AA3EE274AFDEEC47A17EE903A29
:1068A0009942A8BF19469C42D8BF0C4607EE904AB1
:1068B000F8EEE77AC0ED0B7A49E607EE901AF8EEAB
:1068C000E77A1548154C90ED004AD4ED004A14487B
:1068D000CAED614A06EE903A77EE677ABCEEC77A67
:1068E000F8EEE66A17EE103A77EEE67A8AED624A3B
:1068F000AAF88031D0ED006AFEF79ABD09494A69CD
:10690000002A3EF463AA0A6813604B74FEF75EBA6D
:10691000684F0020C83600202C500020285000204E
:106920004450002060A8002007EE103A9BF8003089
:106930008E4FCAF81061B8EEC77AF7EE006A132BD3
:1069400086EE879AB7F90400BAF8145194ED080A54
:1069500001F06481864B874A93ED001A93ED093A62
:1069600093ED162A93ED1F6AD3ED0B1A93ED144A9B
:10697000D3ED015AD3ED0A3A93ED0C7A93ED155A03
:10698000D3ED172AD3ED206AD3ED044AD3ED030AE1
:1069900069EE277A69EE288A29EE088AA7EE813AFD
:1069A00002EB85060021A2EE286ACAF80411CAF893
:1069B0000811A8EE214AE7EEA53AA8EE075A93ED92
:1069C0001A7AD3ED0F5A93ED021AD3ED0E1A86ED13
:1069D000003AE2EEA86A64EEC34A27EE467A93EDE7
:1069E0000D2AD3ED192A86ED204AE3EE603A65EED2
:1069F000C45A93ED183AC3ED093AE7EE814AF0EE36
:106A0000477AA4EE615AE8EE025AE2EEC66AE3EE75
:106A1000287AC3ED0A4A83ED145AC3ED155A86ED60
:106A2000406AC3ED1F6AC3ED207ACAF80C116B1CD3
:106A300003F01F03AAF81431B880FEF7CDB84E4B0F
:106A40001A79002A3EF472AD4C4A1278002A3EF4BC
:106A50006DAD1B789FED4A2A07EE103A494B07EEC1
:106A6000902A1B88F8EEE77A05EE103AB8EE477ADE
:106A7000B8EE455A27EE277AF7EE003AC7EE057AC8
:106A8000F4EEC27AF1EE10FA88BFF0EE427AF4EE3C
:106A9000E37AF1EE10FAB8BFF0EE637AFEF748BD84
:106AA000B37B002B42F06B84029B1B7813F0010335
:106AB00042F06584344A1268002A02F0218613608D
:106AC00001230593009B1B68980633D42F4A127844
:106AD000052A2FD0D9027FF543ADF57B112D3FF666
:106AE0003FAD2B4BDDF814801C4633F9153000EE1A
:106AF000103A4046B8EEC00A6F1C05F10E0604F0CD
:106B000051F94346FFB25D1BF6B2A04600E02746AE
:106B10007C1C7819122FE4B2C0B23FF421AD38F9D1
:106B2000173000EE103AB8EEC00A04F03BF9B44258
:106B3000EDD115E5059A13460233541CDBB210461D
:106B4000E4B20593B5F9003000EE103AB8EEC00A91
:106B500004F028F9B5F9023000EE103A2046B8EEFC
:106B6000C00A04F01FF9009B1B68B3E7DC5100204A
:106B7000186A00207C6700207C540020C752002047
:106B8000713DAA3F80520020106D0020D84900209E
:106B9000B08F00200000000093ED027A93ED012AEF
:106BA000D3ED037A5FED053A26EE877AA6EE027AF8
:106BB000A5EEA77A27EE057AB4EEE37AF1EE10FAA5
:106BC000B4BFF0EE637AF0EE477A8DED0C7A88BFB1
:106BD000B0EE637A012A3EF4AEAED3ED063AD3EDC1
:106BE000051A93ED072A66EEA33AE6EE213AE5EEA2
:106BF000823A63EE853AB4EEE37AF1EE10FAF4EEFF
:106C0000E37A8CBFB0EE632AB0EE472AF1EE10FAB9
:106C100058BFB0EE427AB8BFF0EE637A022ACDEDEB
:106C20000D3A3EF488AED3ED0A3AD3ED091A93ED4E
:106C30000B2A66EEA33AE6EE213AE5EE823A63EEDF
:106C4000853AB4EEE37AF1EE10FAF4EEE37A8CBF13
:106C5000B0EE632AB0EE472AF1EE10FA58BFB0EE5C
:106C6000427AB8BFF0EE637A032ACDED0E3A3EF4D5
:106C700062AED3ED0E3AD3ED0D1A93ED0F2A66EE08
:106C8000A33AE6EE213AE5EE823A63EE853AB4EEB7
:106C9000E37AF1EE10FAF4EEE37A8CBFB0EE632AF9
:106CA000B0EE472AF1EE10FA58BFB0EE427AB8BF04
:106CB000F0EE637A042ACDED0F3A3EF43CAED3ED0C
:106CC000123AD3ED111A93ED132A66EEA33AE6EECB
:106CD000213AE5EE823A63EE853AB4EEE37AF1EEDC
:106CE00010FAF4EEE37A8CBFB0EE632AB0EE472AD6
:106CF000F1EE10FA58BFB0EE427AB8BFF0EE637A08
:106D0000052ACDED103A3EF416AED3ED163AD3ED8A
:106D1000151A93ED172A66EEA33AE6EE213AE5EE50
:106D2000823A63EE853AB4EEE37AF1EE10FAF4EECD
:106D3000E37A8CBFB0EE632AB0EE472AF1EE10FA88
:106D400058BFB0EE427AB8BFF0EE637A062ACDEDB6
:106D5000113A3EF4F0ADD3ED1A3AD3ED191A93ED92
:106D60001B2A66EEA33AE6EE213AE5EE823A63EE9E
:106D7000853AB4EEE37AF1EE10FAF4EEE37A8CBFE2
:106D8000B0EE632AB0EE472AF1EE10FA58BFB0EE2B
:106D9000427AB8BFF0EE637A072ACDED123A3EF49C
:106DA000CAADD3ED1E3AD3ED1D1A93ED1F2A66EE40
:106DB000A33AE6EE213AE5EE823A63EE853AB4EE86
:106DC000E37AF1EE10FAF4EEE37A8CBFB0EE632AC8
:106DD000B0EE472AF1EE10FA58BFB0EE427AB8BFD3
:106DE000F0EE637A082ACDED133A3EF4A4ADD3ED6C
:106DF000223AD3ED211A93ED232A66EEA33AE6EE6A
:106E0000213AE5EE823A63EE853AB4EEE37AF1EEAA
:106E100010FAF4EEE37A8CBFB0EE632AB0EE472AA4
:106E2000F1EE10FA58BFB0EE427AB8BFF0EE637AD6
:106E3000092ACDED143A3EF47EADD3ED263AD3EDDA
:106E4000251A93ED272A66EEA33AE6EE213AE5EEFF
:106E5000823A63EE853AB4EEE37AF1EE10FAF4EE9C
:106E6000E37A8CBFB0EE632AB0EE472AF1EE10FA57
:106E700058BFB0EE427AB8BFF0EE637A0A2ACDED81
:106E8000153A3EF458AD93ED2A2AD3ED291AD3EDE5
:106E90002B3A26EE822AA6EE212AA5EEA32A22EE7E
:106EA000052AB4EEC27AF1EE10FAF4EEC27A8CBF83
:106EB000F0EE423AF0EE473AF1EE10FA8DED162A76
:106EC00058BFB0EE637AA8BFB0EE672A0B2A02F073
:106ED0003A83D3ED2E7AD3ED2D1AD3ED2F3A66EE09
:106EE000A77AE6EE217AE3EEA57A67EE857AF4EEEC
:106EF000C77AF1EE10FAF4EEC27A8CBFF0EE476A70
:106F0000F0EE676AF1EE10FACDED177A98BFB0EEA9
:106F1000667AB8BFF0EE427AFEF70DBD904A049251
:106F20000025904E904FDDF81080CDF80490A946D2
:106F3000B6EC018AD4ED087AB8EEC88A28EE278A22
:106F4000B9F1000F02F0EB837BBB9BF80030082BFC
:106F50003BD005F5D260B0EE480A2044D4F88C3618
:106F6000984705F5E360D4F81437204498479BF818
:106F70000030032BB0EE408A22D0D4F8AC30D6F8E3
:106F80004406B0EE480A984708EB890309F1010965
:106F9000B9F1030F05F12C0583ED010A3DF43CAE78
:106FA000009B1B6803F00053C2E705F5F460B0EEE8
:106FB000480A2044D4F89C379847B0EE408AC4E78A
:106FC00023F04EFA27F81900D7E7B0EE480A23F06D
:106FD00047FA27F81900BCE7DFED646AFEF7FBB952
:106FE000DFF8A881DAED017A9AED006AB8F80000BE
:106FF000D8F8143077EEA77AF0EE006AB0EE677A30
:10700000A6EE267A01380AEBC002D6EE267A083AB6
:107010001033F6EE003A27EE237A67EEA37A8AED74
:10702000207ACAED217ADFF868A157460AF180017B
:1070300092ED027A92ED036AD7ED036AD7ED027AF8
:1070400053ED014A13ED025A37EE674A76EEC65AFF
:1070500077EE277AE4EE845A0138A2F10802E5EED1
:10706000047A07F1080703F1080336EE267A01F1E6
:107070000801E4EE877AE5EE475A67EEA37A25EE3B
:10708000A37AC1ED007A81ED017AD1D1142E07D116
:10709000F7F79EFB019B344FC01A7880DAF818513D
:1070A0002F4B0493324A009B013582FB0512511984
:1070B000EA17C2EBA1021B68C2EBC202AD1ACAF802
:1070C000185103F000532BE7F7F782FB9BF80030D1
:1070D000079A254F801A012B78802CD0072B7DF43E
:1070E0002AAFF7F775FB0490FDF727BFF7F770FBA2
:1070F000049A1D4B801AD880FFF74DBA1D491E48CF
:107100001E4B91ED004AD0ED004A1D491B78CAED97
:10711000614A8AED624AD1ED006A13B101238AF80F
:107120009031DAED637AFEF783B9164F97ED007A66
:10713000FFF74EB80C4FF7F74BFB134ADAF87C31E8
:1071400012680490C31A9A1ACAF87C01BB80FA80AC
:10715000FDF7F3BEF7F73CFB0790FDF77ABD00BFE4
:10716000D4660020E85E0020DC5100200000000012
:1071700093244992F037002030500020FC6D00200D
:1071800040500020104A0020883900206467002009
:1071900024220020E7EE267ADF48B1EE436AB0EE03
:1071A000647AA6EE277AF0EE477ABDEEE47A002CF8
:1071B00041F09686FDEEE77A17EE104A17EE906AD8
:1071C000FDEEC47AB44217EE901A17EE105AA8BF1B
:1071D0003546B142C8BF0D4607EE905AF8EEE77A41
:1071E000012AC0ED007A3FF4B2A993ED047ADDEDF7
:1071F0000D7AE7EE267AB0EE647AA6EE277AFDEEF7
:10720000C77A17EE906A17EE905AA642A8BF254695
:107210008E42B8BF0D4607EE905AF8EEE77A022A82
:10722000C0ED017A3FF493A993ED087ADDED0E7A73
:10723000E7EE267AB0EE647AA6EE277AFDEEC77AFC
:1072400017EE906A17EE905AA642A8BF25468E42C6
:10725000B8BF0D4607EE905AF8EEE77A032AC0ED64
:10726000027A3FF474A993ED0C7ADDED0F7AE7EE24
:10727000267AB0EE647AA7EEC37AFDEEC77A17EEEF
:10728000906A17EE905AA642A8BF25468E42B8BF14
:107290000D4607EE905AF8EEE77A042AC0ED037A1D
:1072A0003FF455A993ED107ADDED107AE7EE267ADA
:1072B000B0EE647AA7EEC37AFDEEC77A17EE906A55
:1072C00017EE905AA642A8BF25468E42B8BF0D467B
:1072D00007EE905AF8EEE77A052AC0ED047A3FF4FB
:1072E00036A993ED147ADDED117AE7EE267AB0EE49
:1072F000647AA7EEC37AFDEEC77A17EE906A17EEAE
:10730000905AA642A8BF25468E42B8BF0D4607EE4A
:10731000905AF8EEE77A062AC0ED057A3FF417A9ED
:1073200093ED187ADDED127AE7EE267AB0EE647A04
:10733000A7EEC37AFDEEC77A17EE906A17EE905A61
:10734000A642A8BF25468E42B8BF0D4607EE905A0A
:10735000F8EEE77A072AC0ED067A3FF4F8A893ED35
:107360001C7ADDED137AE6EE877A2546B0EE647A74
:10737000A6EE277AFDEEC77A17EE906AB442A8BF50
:107380003546B142C8BF0D4607EE905AF8EEE77A8F
:10739000082AC0ED077A3FF4DAA893ED207ADDEDF4
:1073A000147AE6EE877A2546B0EE647AA6EE277A5E
:1073B000FDEEC77A17EE906AB442A8BF3546B142D7
:1073C000C8BF0D4607EE905AF8EEE77A092AC0EDDD
:1073D000087A3FF4BCA893ED247ADDED157AE6EE49
:1073E000877A2546B0EE647AA6EE277AFDEEC77A54
:1073F00017EE906AB442A8BF3546B142C8BF0D46E9
:1074000007EE905AF8EEE77A0A2AC0ED097A3FF4BF
:107410009EA893ED287ADDED167AE7EE267A2546CA
:10742000B0EE647AA7EEC37AFDEEC77A17EE906AE3
:10743000B442A8BF3546B142C8BF0D46FFF767B892
:10744000FDEEC47A0CA817EE906AFDEEE47A00EB2C
:10745000820317EE907AFDEEE57ADFF8C090DFF850
:10746000B8E0089217EE905AB1EE436A84F0010832
:107470004FFA84FC1946CDF824A04B4693ED007AD0
:10748000F0EC017AE7EE267A04F0010309F1100925
:10749000B0EE647AA6EE277AB4EEC74AF1EE10FA9F
:1074A000D8BF0023002BF0EE477A18BFB0EE657A04
:1074B000BDEEC77AFDEEE77A17EE102A17EE90AA16
:1074C000BA4217EE103AA8BF3B469542CCBF002205
:1074D00004F00102002A08BF2B46574507EE103A78
:1074E0003A46A8BF52465645CCBF002308F00103D8
:1074F000002B08BF324607EE902AB8EEC77AF8EEA6
:10750000E77ABCF1000F18BFF0EE477A8842EEEC44
:10751000017AB2D1FEF7AEBDC8360020684F002018
:10752000B84BB5F908101A6802B111609B69B5F93A
:107530000A2003B11A60009B1B689A0601F1A58618
:1075400002220592FFF7C6BA9AF8BC31012B01F06E
:107550002287AD4B96F916005A8896F90AE01B88E7
:10756000AA4910FB03F31EFB02F281FB020C81FB14
:107570000301D217DB17C2EB2C12C3EB21133A44E1
:107580001C442A806C80FEF73FBCDFF8A082A04834
:10759000D8F80820B8F80C1022F00CF89BF800601E
:1075A000142E02F05880DAF818510135CAF8185133
:1075B00018E5DFF87882B8F80060D8F804E04FEA00
:1075C000560C4FEA8C020AEB8607F6080AEB020318
:1075D00000F09F80103201368E4803EB06163A44C5
:1075E00010330EF1100507F1100151ED032A51ED92
:1075F000043A10ED043A10ED032A51ED026A11ED40
:10760000016A10ED020A10ED018A12ED044A12ED32
:10761000035A53ED044A53ED035A13ED027A53ED26
:10762000017A52ED020A12ED011A73EE238A72EE0C
:10763000221A40ED048A40ED031A70EE268A78EE95
:10764000061A40ED028A40ED011A74EE848A75EE46
:10765000851A43ED048A43ED031A77EE208A77EE0C
:10766000811A43ED028A43ED011A73EE633A75EE17
:10767000655A15ED035A32EE623A74EE644A65EECD
:10768000631A15ED044A23EE052A64EE652AE3EE3B
:10769000041A1033B34224EE843AA3EE842A00F194
:1076A000100005F11005A5EE853A01F1100102F177
:1076B0001002E4EE852A41ED071A01ED082A02EDD9
:1076C000073A42ED082A55ED055A15ED065A70EEB7
:1076D000666A38EE466A30EEC77A71EE677A26EE51
:1076E000253A65EEE63A25EE674A67EE054AE6EE8C
:1076F000053AA6EE853AA7EE254AE7EEA54A01ED42
:10770000063A41ED053A02ED064A42ED054A7FF49C
:107710006CAF1FFA8CF5724629463D4816F02AFFD9
:107720002946D8F80420384616F024FF9BF800308C
